:042000006FEF6CF022
:0820080000C004F001C005F066
:1020100002C006F0076A03C008F000016F00D4FF99
:1020200009F06F00D8FF0AF06F00DCFF0BF03901F8
:1020300093A71EEF10F0A3B747EF2AF093AF24EF5A
:1020400010F0A3BF29EF2AF094A12AEF10F0A4B159
:102050005AEF25F096A530EF10F0A6B5FFEF29F066
:1020600096AD36EF10F0A6BD35EF26F098AD3CEFFB
:1020700010F0A8BD70EF26F0600027F0F5FF6000BB
:102080002BF0F6FF60002FF0F7FF04C000F005C052
:1020900001F006C002F0078E08C003F01100F76AD5
:1020A000AE0FF66E200EF7220900F5501200280C34
:1020B0000106C00FF66E200EF7220900F55012003F
:1020C0000000C1C081C1400101C3C003800241C200
:1020D00001C6C006800741C70005C1C581C44004D0
:1020E00001CCC00C800D41CD000FC1CF81CE400E80
:1020F000000AC1CA81CB400B01C9C009800841C890
:1021000001D8C018801941D9001BC1DB81DA401AFF
:10211000001EC1DE81DF401F01DDC01D801C41DCCF
:102120000014C1D481D5401501D7C017801641D6FF
:1021300001D2C012801341D30011C1D181D040100F
:1021400001F0C030803141F10033C1F381F24032FF
:102150000036C1F681F7403701F5C035803441F4CF
:10216000003CC1FC81FD403D01FFC03F803E41FE7F
:1021700001FAC03A803B41FB0039C1F981F840388F
:102180000028C1E881E9402901EBC02B802A41EAFF
:1021900001EEC02E802F41EF002DC1ED81EC402CCF
:1021A00001E4C024802541E50027C1E781E64026FF
:1021B0000022C1E281E3402301E1C021802041E00F
:1021C00001A0C060806141A10063C1A381A24062FF
:1021D0000066C1A681A7406701A5C065806441A4CF
:1021E000006CC1AC81AD406D01AFC06F806E41AE7F
:1021F00001AAC06A806B41AB0069C1A981A840688F
:102200000078C1B881B9407901BBC07B807A41BAFE
:1022100001BEC07E807F41BF007DC1BD81BC407CCE
:1022200001B4C074807541B50077C1B781B64076FE
:102230000072C1B281B3407301B1C071807041B00E
:102240000050C190819140510193C05380524192FE
:102250000196C056805741970055C19581944054CE
:10226000019CC05C805D419D005FC19F819E405E7E
:10227000005AC19A819B405B0199C059805841988E
:102280000188C04880494189004BC18B818A404AFE
:10229000004EC18E818F404F018DC04D804C418CCE
:1022A0000044C184818540450187C04780464186FE
:1022B0000182C042804341830041C181818040400E
:1022C000583220256325632563256325632563250F
:1022D000632563202020202000005831202563251D
:1022E00063256325632563256325632563202020FB
:1022F00020200000706F736963616F2020202536F5
:102300004C640000656E747261646120202020209E
:1023100020253033750020504152414D4554524FD5
:102320005320444520200000205445535445204765
:1023300052415641444F5320000020504152412009
:10234000434F4E54494E5541522000004C4942459E
:102350005245204F5320424F544F45530000414AAD
:10236000555354452020202020202025322E306631
:102370002525000053616972202020202D20202077
:10238000202B202000002020504F52544120534148
:102390004645545920200000736169722020207343
:1023A000696D2020206E616F00002020504F525434
:1023B0004120534146455459202000002020504FD1
:1023C000525441204154495641444F20000020209E
:1023D000504F52544120534146455459202000004B
:1023E000504F525441204445534154495641444F63
:1023F00000002074696D657220667265657A657289
:102400003F2000007361697220202073696D2020D5
:10241000206E616F00002074696D65722020667205
:1024200065657A657220000020202020616A75733E
:10243000746172202020202000002074696D657274
:102440002020667265657A657220000020202020B9
:102450006D616E7469646F202020200054494D45E1
:102460005220202020253375204D696E00005361D5
:102470006972202020202D20202020202B200000E9
:1024800054494D455220202020253375204D696E3A
:1024900000002045535441204E4120454550524FA5
:1024A0004D20000020415449564152202020504FD9
:1024B000525441200000465245455A455220505240
:1024C000494D4549524F000020504F52544120463B
:1024D0005245455A45522020000073616972202000
:1024E0002073696D2020206E616F000020504F52D4
:1024F000544120465245455A455220200000205460
:10250000494D4552204154495641444F2020000036
:1025100020504F52544120465245455A45522020A2
:10252000000054494D4552204445534154495641B9
:10253000444F000020504F52544120465245455AC6
:10254000455220200000204E414F205045524D4919
:102550005449444F20200000464341204455504CEC
:102560004F20504152414441000073616972202064
:102570002073696D2020206E616F0000464341206A
:102580004455504C41205041524144410000464383
:102590004120202020202020415449564F20000077
:1025A000464341204455504C412050415241444102
:1025B00000004643412020202020494E41544956E6
:1025C0004F200000425220434F4E544147454D3F5B
:1025D0002020202000007361697220202073696D23
:1025E0002020206E616F000042522020434F4E5445
:1025F0004147454D202020200000434F4E54414785
:10260000454D20204154495641200000425220208F
:10261000434F4E544147454D202020200000434F5A
:102620004E544147454D20494E41544956410000C2
:10263000515444205245544F524E4F532025337528
:10264000000053616972202020202D2020202020AE
:102650002B200000515444205245544F524E4F53AA
:102660002025337500002045535441204E4120451C
:102670004550524F4D20000044454C4159204142A5
:102680004552545552413F20000073616972202029
:102690002073696D2020206E616F000044454C411D
:1026A0005920414245525455524120200000444592
:1026B0004C41592020202020415449564F200000F1
:1026C00044454C41592041424552545552412020E5
:1026D000000044454C4159202020494E4154495660
:1026E0004F20000054502044454C4159202533755B
:1026F00020534547000053616972202020202D207F
:10270000202020202B20000054502044454C4159CB
:102710002025337520534547000020455354412060
:102720004E4120454550524F4D2000002052454C0F
:102730004553205041206520504620200000736101
:10274000697220202073696D2020206E616F000067
:102750002052454C455320504120652050462020B2
:102760000000202020204154495641444F5320204E
:10277000202000002052454C455320504120652028
:1027800050462020000020204445534154495641E2
:10279000444F532020200000504120652050462007
:1027A00050554C5345203F20000073616972202032
:1027B0002073696D2020206E616F00002050412041
:1027C000652050462050554C5345202000002020C5
:1027D00020204154495641444F53202020200000DE
:1027E00020504120652050462050554C5345202014
:1027F000000020204445534154495641444F532042
:1028000020200000504F5320444553415420464F50
:10281000544F313F00002020202020202073696D7C
:102820002020206E616F0000706F732061747561ED
:102830006C25364C6400706F73204646202020259E
:10284000364C64002020202020504F534943414FF4
:1028500020202020000020202020204752415641E7
:1028600044412020202000002020202020504F53D1
:102870004943414F20202020000020202020204DCF
:10288000414E544944412020202000002020204374
:102890004F4E5441544F5245532020200000736145
:1028A000697220202073696D2020206E616F000006
:1028B00053414944415320434F4E5441544F5220B9
:1028C0000000202020204154495641444F532020ED
:1028D0002020000053414944415320434F4E54416E
:1028E000544F522000002020444553415449564142
:1028F000444F53202020000020202020202020535F
:10290000696D20204E616F20000020202020436F41
:102910006E6669726D613F2020200000202020201B
:1029200020202053692020204E6F202000002020EE
:102930002020436F6E6669726D613F202020000089
:102940002020202020205965732020204E6F202039
:102950000000202020436F6E6669726D203F2020AA
:1029600020200000205041524120434F4E54494EF8
:10297000554152200000205041524120434F4E54B7
:10298000494E55415220000020464F522053455495
:1029900054494E472055502000004C49424552456D
:1029A000204F5320424F544F45530000204C494282
:1029B00045524520424F544F4E455320000052454A
:1029C0004C454153452020425554544F4E5300002E
:1029D00020202020202020202020202020202020F7
:1029E0000000202020202020202020202020202027
:1029F00020200000204449474954452041205345A8
:102A00004E4841200000454E54524520434F4E54FD
:102A1000524153454E41000020454E5445522050EE
:102A2000415353574F52442000004F6B2020202029
:102A30002020253175202020202025317520000000
:102A40002044494749544520412053454E484120A0
:102A50000000454E54524520434F4E545241534579
:102A60004E41000020454E5445522050415353578B
:102A70004F52442000004F6B202020202020253181
:102A80007520202020202531752000002044494752
:102A900049544520412053454E4841200000454EB1
:102AA00054524520434F4E54524153454E4100002D
:102AB00020454E5445522050415353574F524420C5
:102AC00000004F6B20202020202025317520202061
:102AD0002020253175200000202020202020534573
:102AE0004E48412020202020200020202020494E38
:102AF000434F5252455441212020200020202043A2
:102B00004F4E54524153454E41202020200020205A
:102B100020494E434F52524543544121202020002A
:102B2000202020202057524F4E47202020202020B8
:102B300020002020202050415353574F5244212041
:102B400020202000204C41444F204D4F544F522014
:102B50003F2020200000204C41444F204D4F544F37
:102B600052203F2020200000204D4F544F52205330
:102B7000494445203F202020000053696D2020203B
:102B80002020256320202020202563200000536979
:102B900020202020202025632020202020256320A5
:102BA000000059657320202020202563202020204C
:102BB000202563200000204C41444F204D4F544FAE
:102BC00052203F2020200000204C41444F204D4FF8
:102BD000544F52203F2020200000204D4F544F5290
:102BE0002053494445203F202020000053696D2098
:102BF0002020202025632020202020256320000085
:102C000053692020202020202563202020202025FB
:102C10006320000059657320202020202563202098
:102C200020202025632000002020204D4F544F52AB
:102C30002053494445202020000020204C41444F8F
:102C40002020204D4F544F522020000073616972A4
:102C50002020206573712020206469720000736158
:102C60006C69722020697A712020206465720000EE
:102C70004578697420204C656674205269676874D1
:102C80000000204D4F544F5220455351554552445A
:102C90004F3F00006772617661722065737120207A
:102CA0006469722000004D4F544F5220495A5155CB
:102CB000494552444F3F000067726162617220696A
:102CC0007A71202064657220000020204D4F544FFF
:102CD00052202020204C4546543F0000536574206C
:102CE000204C656674202052696768740000204D8E
:102CF0004F544F52204449524549544F203F000001
:102D00006772617661722065737120206469722038
:102D10000000204D4F544F52204445524543484FE8
:102D2000203F000067726162617220697A71202021
:102D300064657220000020204D4F544F52202052D5
:102D400049474854203F000053657420204C656675
:102D50007420205269676874000020204643204197
:102D600042455254555241203F20000053696D2086
:102D70002020202025632020202020256320000003
:102D800020204643204150455254555241203F2077
:102D900000005369202020202020256320202020AF
:102DA00020256320000020204C494D495420204F0D
:102DB00050454E203F2000005965732020202020E0
:102DC0002563202020202025632000006772617683
:102DD00061646F20202025364C64000053616972C5
:102DE0002020446573636520536F6265000067723D
:102DF000616261646F20202025364C6400005361BD
:102E00006C6972204162616A6F20537562650000CF
:102E10005365745F6F6B2020202025364C640000C2
:102E20004578697420202020446F776E20205570EB
:102E30000000706F7320617475616C2025364C64DE
:102E40000000477261766120446573636520536FAB
:102E500062650000706F732061637475616C253664
:102E60004C6400004772616261204162616A6F20B8
:102E7000537562650000706F732061637475616CD7
:102E800025364C6400004578697420202020446F6A
:102E9000776E202055700000464320414245525431
:102EA00055524120494E543F000053696D20202067
:102EB0002020256320202020202563200000464379
:102EC00020415045525455524120494E543F000034
:102ED0005369202020202020256320202020202529
:102EE00063200000494E54204F50454E20204C494D
:102EF0004D49543F00005965732020202020256350
:102F00002020202020256320000067726176616404
:102F10006F20202025364C64000053616972202008
:102F2000446573636520536F626500006772616278
:102F300061646F20202025364C64000053616C6969
:102F400072204162616A6F205375626500005365AB
:102F5000745F6F6B2020202025364C64000045787C
:102F6000697420202020446F776E20205570000067
:102F7000706F7320617475616C2025364C6400009D
:102F8000477261766120446573636520536F6265A3
:102F90000000706F732061637475616C25364C643A
:102FA00000004772616261204162616A6F2053755F
:102FB00062650000706F732061637475616C253603
:102FC0004C6400004578697420202020446F776E9F
:102FD0002020557000002046432046454348414D7F
:102FE000454E544F203F000053696D202020202083
:102FF000256320202020202563200000202020465B
:1030000043204349455252453F2020200000536948
:103010002020202020202563202020202025632020
:10302000000020204C494D49542020434C4F53452B
:103030003F20000059657320202020202563202098
:1030400020202025632000006772617661646F2074
:10305000202025364C6400005361697220204465AD
:1030600073636520536F626500006772616261641B
:103070006F20202025364C64000053616C6972205B
:103080004162616A6F205375626500005365745F29
:103090006F6B2020202025364C6400004578697431
:1030A00020202020446F776E202055700000706F24
:1030B0007320617475616C2025364C640000477282
:1030C00061766120446573636520536F626500001B
:1030D000706F732061637475616C25364C640000F9
:1030E0004772616261204162616A6F205375626557
:1030F0000000706F732061637475616C25364C64D9
:1031000000004578697420202020446F776E2020CD
:103110005570000020414A205245442056454C201D
:103120004645203F000053696D2020202020256364
:103130002020202020256320000020414A205245E5
:10314000442056454C204345203F00005369202031
:10315000202020202563202020202025632000001F
:1031600053455420534C4F2053504420434C203F50
:103170000000596573202020202025632020202076
:103180002025632000007265647563616F20202034
:1031900025357525250053616972202020202D20BA
:1031A000202020202B200000726564756363696F06
:1031B0006E2025357525250053616C69722020200D
:1031C0002D20202020202B200000736C6F207261A6
:1031D00074652020253575252500457869742020E3
:1031E00020202D20202020202B20000072656475D7
:1031F00063616F2020202535752525004772617693
:10320000617220202D20202020202B2000007265BC
:1032100064756363696F6E202535752525004772D7
:103220006162617220202D20202020202B200000B0
:10323000736C6F207261746520202535752525001B
:103240005365745F6F6B20202D20202020202B20C1
:103250000000677261766F752071756174726F20FE
:103260002020000020414A205245442056454C2051
:103270004142203F000053696D202020202025631B
:103280002020202020256320000020414A20524594
:10329000442056454C204150203F000053692020D7
:1032A00020202020256320202020202563200000CE
:1032B00053455420534C4F20535044204F50203FEF
:1032C0000000596573202020202025632020202025
:1032D0002025632000007265647563616F202020E3
:1032E00025357525250053616972202020202D2069
:1032F000202020202B200000726564756363696FB5
:103300006E2025357525250053616C6972202020BB
:103310002D20202020202B200000736C6F20726154
:103320007465202025357525250045786974202091
:1033300020202D20202020202B2000007265647585
:1033400063616F2020202535752525004772617641
:10335000617220202D20202020202B20000072656B
:1033600064756363696F6E20253575252500477286
:103370006162617220202D20202020202B2000005F
:10338000736C6F20726174652020253575252500CA
:1033900053657420202020202D20202020202B2049
:1033A0000000414A555354452020204C4F4F50496E
:1033B0004E470000414A555354452020204C4F4F62
:1033C00050494E470000204C4F4F50494E47202057
:1033D000534554555020000053696D202020202073
:1033E0002563202020202025632000005369202011
:1033F000202020202563202020202025632000007D
:10340000596573202020202025632020202020259E
:1034100063200000414A555354452020202020209D
:103420002025322E30662525000053616972202048
:1034300020202D202020202B20200000414A555301
:1034400054452020202020202025322E306625259E
:10345000000053616C69722020202D202020202B39
:1034600020200000536574202056616C7565202073
:103470002025322E306625250000457869742020ED
:1034800020202D202020202B20200000414A5553B1
:1034900054452020202020202025322E306625254E
:1034A000000047726176617220202D202020202BA1
:1034B00020200000414A5553544520202020202040
:1034C0002025322E30662525000047726162617228
:1034D00020202D202020202B202000005365742048
:1034E0002056616C756520202025322E30662525FA
:1034F000000053657420202020202D202020202B28
:103500002020000020434D44204D414E55414C2089
:103510003F202020000053696D20202020202563BB
:103520002020202020256320000053692020202017
:1035300020202563202020202025632000005965BD
:103540007320202020202563202020202025632098
:10355000000020434D44202020204D414E55414C39
:1035600020200000736169722066656368612061D4
:1035700062726520000073616C6972206162616A29
:103580006F207375626500004578697420202020E3
:10359000446F776E202055700000414A2054454DFD
:1035A000504F204645434841203F000053696D205D
:1035B00020202020256320202020202563200000BB
:1035C000414A205449454D50204349455252453FB8
:1035D0000000536920202020202025632020202067
:1035E00020256320000041444A20434C4F5345208E
:1035F00054494D45203F000059657320202020206C
:1036000025632020202020256320000054504645BB
:10361000434841202533752073656773000053616B
:103620006972202020202D20202020202B20000027
:1036300054504349455252452025337520736567E0
:10364000000053616C69722020202D202020202052
:103650002B2000005443434C4F5345202025337505
:1036600020736563000045786974202020202D2098
:10367000202020202B200000545046454348412064
:103680002533752073656773000047726176617238
:1036900020202D20202020202B20000054504349A2
:1036A00045525245202533752073656700004772E7
:1036B000616261722020202D20202020202B2000FC
:1036C0005443434C4F534520202533752073656385
:1036D00000005365742020202020202D2020202051
:1036E000202B20002054454D504F52495A41444F01
:1036F00052203F2000002054454D504F52495A411E
:10370000444F52203F200000202020202054494DCB
:103710004552203F20202020000053696D202020AA
:1037200020202563202020202025632000005369CD
:1037300020202020202025632020202020256320F9
:1037400000005965732020202020256320202020A0
:103750002025632000002054454D504F52495A41C6
:10376000444F52203F2000002054454D504F5249B5
:103770005A41444F52203F20000020202020205456
:10378000494D4552203F202020200000736169727E
:1037900020202073696D2020206E616F000073610E
:1037A0006C697220207369202020206E6F20000039
:1037B000457869742020796573202020206E6F2061
:1037C00000002054454D504F52495A41444F522019
:1037D000202000002054454D504F52495A41444F3B
:1037E000522020200000202020202054494D455206
:1037F0002020202020200000736169722020207387
:10380000696D2020206E616F000073616C69722009
:10381000207369202020206E6F2000004578697495
:103820002020796573202020206E6F200000205416
:10383000454D504F52495A41444F522020200000DC
:103840002054454D504F52495A41444F5220202058
:103850000000202020202054494D455220202020C7
:10386000202000006772617661722073696D2020EC
:103870006E616F200000677261626172207369205F
:1038800020206E6F20200000736574202020796551
:10389000732020206E6F202000002054454D504F93
:1038A00052495A41444F5220202000002054454D97
:1038B000504F52495A41444F5220202000002020AE
:1038C00020202054494D4552202020202020000057
:1038D0006772617661722073696D20206E616F205E
:1038E00000006772616261722073692020206E6F30
:1038F000202000007365742020207965732020202B
:103900006E6F202000004944494F4D412F4C414EDD
:1039100047554147453F0000532F59202020202084
:103920002563202020202025632000004944494FA2
:103930004D412F4C414E4755414745200000454ED3
:1039400047202020204553502020504F5254000043
:103950004944494F4D412F4C414E47554147452021
:103960000000454E47202020204553502020504F36
:10397000525400004944494F4D412F4C414E475548
:1039800041474520000020202020454E474C495308
:1039900048202020202000004944494F4D412F4C11
:1039A000414E4755414745200000202020204553E7
:1039B00050414E4F4C202020202000004944494FC8
:1039C0004D412F4C414E4755414745200000202096
:1039D00020504F5254554755455320202020000079
:1039E000202020444947494C494E4B203F2020206D
:1039F000000053696D2020202020256320202020F6
:103A0000202563200000202020444947494C494E8E
:103A10004B203F2020200000536920202020202020
:103A20002563202020202025632000002020204422
:103A30004947494C494E4B203F2020200000596502
:103A40007320202020202563202020202025632093
:103A5000000020202020444947494C494E4B20205B
:103A6000202000007361697220202073696D20207E
:103A7000206E616F000020202020444947494C49B6
:103A80004E4B20202020000073616C69722020734F
:103A900069202020206E6F20000020202020444933
:103AA00047494C494E4B202020200000457869743E
:103AB0002020796573202020206E6F200000204395
:103AC0004F4D2020444947494C494E4B202000008F
:103AD0006772617661722073696D20206E616F205C
:103AE000000020434F4D2020444947494C494E4B4C
:103AF00020200000677261626172207369202020BB
:103B00006E6F2020000020574954482044494749FF
:103B10004C494E4B202000007365742020207965AD
:103B2000732020206E6F202000002053454D202060
:103B3000444947494C494E4B20200000677261764A
:103B400061722073696D20206E616F200000205328
:103B5000454D2020444947494C494E4B2020000008
:103B60006772616261722073692020206E6F20206D
:103B70000000574954484F555420444947494C493F
:103B80004E4B00007365742020207965732020203F
:103B90006E6F2020000020202020205361697220B9
:103BA0003F2020202020000053696D20202020206D
:103BB00025632020202020256320000020202020B5
:103BC0002053616C6972203F20202020000053693F
:103BD0002020202020202563202020202025632055
:103BE0000000202020202045786974203F202020DC
:103BF00020200000596573202020202025632020EC
:103C00002020202563200000202020204154454E04
:103C100043414F2120202020000020564F434520C3
:103C200056414920454E5452415200002020202048
:103C30004154454E43494F4E202020200000202073
:103C4000555354454420454E5452415241200000A2
:103C5000202020205741524E494E4720202020202E
:103C6000000020202020454E544552494E47202038
:103C7000202000002020454D2054524F4341204435
:103C8000452020200000202020504152414D455425
:103C9000524F5320202000002020412043414D421C
:103CA000494F204445202020000020202050415230
:103CB000414D4554524F5320202000002020202009
:103CC0004348414E47494E472020202000002020F5
:103CD0002020202053455455502020202020000033
:103CE0002020434F4E5452412D53454E48412020F1
:103CF00000004F6B2020202020202531752020201F
:103D000020202531752000002020434F4E54524181
:103D10002D53454E4841202000004F6B202020208D
:103D200020202531752020202020253175200000FD
:103D30002020434F4E5452412D53454E48412020A0
:103D400000004F6B202020202020253175202020CE
:103D500020202531752000002020202020205345E0
:103D60004E48412020202020200020202020494EA5
:103D7000434F525245544121202020004147554194
:103D80005244414E444F204645434841000054456B
:103D90004D504F204645434841522025334C750035
:103DA0004553504552414E444F2043455252415293
:103DB00000005449454D504F204345525241202563
:103DC000334C750057414954494E4720544F2043C6
:103DD0004C4F5345000054494D452020434C4F5310
:103DE00045202025334C75004245202020202020EE
:103DF00020202020202020200000424120202020C0
:103E000020202020202020202020000042452F427A
:103E1000412020202020202020202020000042526D
:103E200020202020202020202020202020200000D2
:103E300042452F42522020202020202020202020D8
:103E4000000042412F42522020202020202020200C
:103E50002020000020504152414441202041424551
:103E600052544120000042452F42412F425220200F
:103E7000202020202020000046312020202020204B
:103E80002020202020202020000042452F463120E5
:103E900020202020202020202020000042412F46EA
:103EA00031202020202020202020202000004245FA
:103EB0002F42412F463120202020202020200000AA
:103EC00042522F4631202020202020202020202058
:103ED000000042452F42522F463120202020202032
:103EE0002020000042412F42522F46312020202026
:103EF00020202020000042452F42412F42522F46D1
:103F000031202020202000004632202020202020A8
:103F10002020202020202020000042452F46322053
:103F200020202020202020202020000042412F4659
:103F30003220202020202020202020200000424568
:103F40002F42412F46322020202020202020000018
:103F500042522F46322020202020202020202020C6
:103F6000000042452F42522F4632202020202020A0
:103F70002020000042412F42522F46322020202094
:103F800020202020000042452F42412F42522F4640
:103F9000322020202020000046312F4632202020D1
:103FA0002020202020202020000042452F46312FB5
:103FB00046322020202020202020000042412F4691
:103FC000312F463220202020202020200000424592
:103FD0002F42412F46312F46322020202020000042
:103FE00042522F46312F46322020202020202020F0
:103FF000000042452F42522F46312F4632202020CA
:104000002020200042412F42522F46312F4632209D
:1040100020202020000042452F42412F42522F46AF
:10402000312F4632202000004C202020202020204C
:104030002020202020202020000042452F4C20203E
:1040400020202020202020202020000042412F4C32
:104050002020202020202020202020200000424559
:104060002F42412F4C202020202020202020000003
:1040700042522F4C202020202020202020202020B1
:10408000000042452F42522F4C202020202020208B
:104090002020000042412F42522F4C20202020207F
:1040A00020202020000042452F42412F42522F4C19
:1040B000202020202020000046312F4C20202020CE
:1040C0002020202020202020000042452F46312F94
:1040D0004C202020202020202020000042412F467C
:1040E000312F4C202020202020202020000042457D
:1040F0002F42412F46312F4C20202020202000002D
:1041000042522F46312F4C202020202020202020DA
:10411000000042452F42522F46312F4C20202020B4
:104120002020000042412F42522F46312F4C2020A8
:1041300020202020000042452F42412F42522F468E
:10414000312F4C202020000046322F4C20202020F0
:104150002020202020202020000042452F46322F02
:104160004C202020202020202020000042412F46EB
:10417000322F4C20202020202020202000004245EB
:104180002F42412F46322F4C20202020202000009B
:1041900042522F46322F4C20202020202020202049
:1041A000000042452F42522F46322F4C0000424120
:1041B0002F42522F46322F4C20202020202000005A
:1041C00042452F42412F42522F46322F4C20202071
:1041D000000046312F46322F4C2020202020202066
:1041E0002020000042452F46312F46322F4C202000
:1041F00020202020000042412F46312F46322F4CF4
:10420000202020202020000042452F42412F46310F
:104210002F46322F4C202020000042522F46312FB3
:1042200046322F4C202020202020000042452F42E3
:10423000522F46312F46322F4C2020200000424181
:104240002F42522F46312F46322F4C20200042451C
:104250002F42412F42522F46312F46322F4C000021
:104260004E414F20434845474F55204E4120202086
:104270000000253275202020202020202020202012
:1042800020202000205041524144412020414245FD
:1042900052544120000020504152414441202041CD
:1042A0004249455254410000202020204F50454EA5
:1042B0002053544F50202020000020504F52544192
:1042C0002020504152414441202000002020204520
:1042D0004D204D4F444F2053544F20200000583163
:1042E00020256325632563256325632563256325D1
:1042F00063204C5020256300583120256325632519
:104300006325632563256325632563202020202002
:104310000000454D455247454E43494120424F54C8
:10432000414F00004150502020444953504F4E49C6
:1043300056454C200000454D455247454E434941A6
:1043400020424F54414F00002020202020202020D8
:1043500020202020202020200000454D45524745A8
:104360004E43494120424F544F4E00002020202010
:104370002020202020202020202020200000454D2B
:10438000455247454E435920425554544F4E000024
:10439000202020202020202020202020202020201D
:1043A00000004D414E4F504C412041434F504C4135
:1043B000444100004445534C4947415220502F523C
:1043C0004553455400005831202563256325632556
:1043D000632563256325632563204C5020256300F6
:1043E00020504F52544120464543484144412020EB
:1043F00000002020494E54455254524156414441F8
:10440000202000002050554552544120434552522F
:104410004144412000002020494E5445525452410D
:104420005641444120200000202020434C4F53455A
:104430004420444F4F5220200000202020494E5459
:1044400045524C4F434B45442020000020454E43ED
:104450004F444552205245515545522000002020DE
:10446000205245494E494349415220202020000016
:1044700020202020504F53534956454C20202020C7
:10448000000053455249414C20494E56455254492B
:104490004441000020202020202020202020202017
:1044A000202020200000656D657267656E6369617C
:1044B0002020206C636400006261206163696F6E7C
:1044C00061646F2020202020000041475541524464
:1044D000414E444F204645434841000054454D500D
:1044E0004F204645434841522025334C75004553E3
:1044F000504552414E444F204345525241520000D4
:104500005449454D504F2043455252415220253287
:104510004C75000057414954494E4720544F2043A1
:104520004C4F5345000054494D4520544F20434CB7
:104530004F53452025324C75000074656D706F2017
:1045400066656368616D656E746F00007469656DA2
:10455000706F2064652063696572726500002020B9
:10456000636C6F7365202074696D652020002020C6
:10457000202020202020202020202020202000007B
:10458000202020202020202020202020202020202B
:10459000000020202020202020202020202020205B
:1045A0002020000045422032345F302056434F44E3
:1045B00045522020000056455253414F20202020D4
:1045C0002025730056455253494F4E202020202568
:1045D00073004D4F544F5220534944452020202012
:1045E000202000004C41444F20204D4F544F52207A
:1045F000202020200000455351554552444F202093
:1046000020202020202000004449524549544F20BA
:1046100020202020202020200000495A51554945C3
:1046200052444F20202020202020000044455245A5
:1046300043484F20202020202020202000004C45EF
:104640004654202020202020202020202020000050
:10465000524947485420202020202020202020207C
:10466000000054494D4552202020202020202020A9
:104670002020000054454D504F52495A41444F525A
:1046800020202020000046454348415220454D202F
:1046900025324C75207365670000434552524152E4
:1046A00020454E2025324C75207365670000434C31
:1046B0004F534520494E202025324C7520736563A9
:1046C00000004349434C4F5320444120504F525423
:1046D000412000004349434C4F53202020202025F7
:1046E000354C75004349434C4F53204441205055AD
:1046F0004552544100004349434C4F532020202051
:104700002025354C7500202020444F4F522043591E
:10471000434C4553202000004359434C455320202F
:1047200020202025354C7500504F52544120202028
:10473000465245455A455220000054494D455220A5
:104740004154495641444F202020000050554552C5
:10475000544120465245455A4552202000005449B4
:104760004D455220414354495641444F20200000BA
:104770002020465245455A455220444F4F52202052
:10478000000020202054494D4552204F4E2020202B
:1047900020200000504F52544120202046524545D1
:1047A0005A455220000054494D455220444553413A
:1047B00054495641444F00005055455254412046FB
:1047C0005245455A45522020000054494D4552203B
:1047D0004E4F414354495641444F00002020465219
:1047E00045455A455220444F4F522020000020207A
:1047F0002054494D4552204F46462020202000009D
:10480000414A555354452020204C4F4F50494E4764
:10481000000053454E5349422020202020202025CF
:10482000322E306625250000204C4F4F50494E4710
:104830002041444A55535420000053454E53495497
:104840002020202020202025322E30662525000023
:104850002052454C45532050412065205046202091
:104860000000202020204154495641444F5320202D
:10487000202000002052454C455320504120652007
:10488000504320200000202020204143544956411D
:10489000444F5320202000002052454C41595320C2
:1048A000444F2026204443200000202020202020A8
:1048B000204F4E202020202020200000494E54452B
:1048C000522D424C4F5155454F20202000002020B2
:1048D00020204154495641444F20202020200000F0
:1048E000494E5445522D424C4F5155454F202020A2
:1048F000000020202020414354495641444F2020AD
:1049000020200000202020494E5445524C4F434B5C
:104910002020202000002020202020204F4E20207A
:1049200020202020202000002020202020204D4F6B
:10493000444F202020202020000020202020205331
:1049400041464554592020202020000020202020CE
:1049500020204D4F444F20202020202000002020E8
:104960002020204E4F524D414C202020202000007E
:104970002020564D4F5445204D4F44425553202042
:104980000000202020204154495641444F2020203F
:10499000202000002020564D4F5445204D4F4442CA
:1049A0005553202000002020202020204F4E202082
:1049B0002020202020200000202020202020202037
:1049C0002020202020202020000020202020202027
:1049D0002020202020202020202000000101D95369
:1049E0000CE0010E006ED851016E04E0D890003644
:1049F000012EFCD7005082130DD0010E006ED8514D
:104A0000016E04E0D8900036012EFCD70050FF0A5A
:104A10008217836B00011200D8B204D0010EEA6E37
:104A2000E30EE96E006A016A026A036A0101E36B40
:104A3000E46BE56BE66BE251E111E011DF112CE074
:104A4000200EE76FD890DB37DC37DD37DE37E33712
:104A5000E437E537E637E251E65D08E1E151E55D2F
:104A600005E1E051E45D02E1DF51E35D0FE3DF5179
:104A7000E35FE051D8A0E03DE45FE151D8A0E13D23
:104A8000E55FE251D8A0E23DE65FD880003601360E
:104A900002360336E72FD6D760008FF7EFFF6000AE
:104AA00093F7ECFF600097F7ECFF60009BF7ECFFDB
:104AB0000001120000010101D86B02C1D9F100010F
:104AC0008DDF010E0101D86F00C1D9F1000186DF31
:104AD000020E0101D86FFEC0D9F100017FDF000E88
:104AE000CAB2010E0101D76F030ED86FD7C1D9F139
:104AF000000174DF000ECAB4010E0101D76F040E6D
:104B0000D86FD7C1D9F1000169DF000ECAB6010E16
:104B10000101D76F050ED86FD7C1D9F100015EDF53
:104B2000000ECAB8010E0101D76F060ED86FD7C1AB
:104B3000D9F1000153DF000ECABA010E0101D76F8F
:104B4000070ED86FD7C1D9F1000148DF3901949120
:104B5000C3C01CF1C2C01BF1000E000188B5010EDC
:104B600001011D6F1E6B000E000188B7010E0101CF
:104B70001F6F206B0001AA5306E1AB5304E1AC5355
:104B800002E1AD5328E088A526D0AA51AE5D01010F
:104B9000D76F0001AB51AF590101D86F0001AC5183
:104BA000B0590101D96F0001AD51B1590101DA6F5E
:104BB000D892DE6FD9C1DDF1D8C1DCF1D7C1DBF10C
:104BC000E26BE16BE06B0A0EDF6F000125DF01C0D5
:104BD00022F100C021F1000E010116B7010E236F72
:104BE000246B000E16B9010E256F266BB7C028F195
:104BF000B6C027F1BBC02AF1BAC029F1CCC02BF155
:104C0000CDC02CF1DB6BCAC02DF10001CBC02EF161
:104C1000010183C130F182C12FF1000E17BD010ED9
:104C2000010A179DE8B0178D000E000169B5010E4D
:104C3000010A6995E8B06985662BD8B4672B67BF10
:104C400008D0675303E16651020803E2676B666BA5
:104C5000BB943C0EB16EB00EB06E00003901A49151
:104C60009481A49100013CEF10F000018E2B8E5135
:104C700009080AE2000E88B1010E010A8891E8B025
:104C800088818E6BDE2BDF2B010EAA27D8B0AB2BD1
:104C9000D8B4AC2BD8B4AD2BB151AD5D15E30BE15D
:104CA000B051AC5D11E307E1AF51AB5D0DE303E142
:104CB000AA51AE5D09E2AD6BAC6BAB6BAA6BB56B89
:104CC000B46BB36B010EB26FE02B3C0EA56EB00E51
:104CD000A46E00003901A69DA69D00013CEF10F0D6
:104CE0000001CDB806D0CDAA04D0CCAE02D0010EC2
:104CF000956FCDB806D0CDBA04D0CCBE02D0020E8E
:104D0000956FCDA806D0CDBA04D0CCAE02D0030E9C
:104D1000956FCDA806D0CDAA04D0CCBE02D0040E8B
:104D2000956FCDA806D0CDAA04D0CCAE02D0050E8A
:104D3000956FCDB806D0CDBA04D0CCAE02D0060E59
:104D4000956FCDB806D0CDAA04D0CCBE02D0070E48
:104D5000956FCDA806D0CDBA04D0CCBE02D0080E37
:104D6000956FCC9C0A0E0101D76F020ED725D86F24
:104D7000000187BF95D0F05327E1B7AF03D0C3AF91
:104D80000CD002D0C3BF07D0B751C35D04E305E127
:104D9000C251B65D02E3CAA205D0F497010116978D
:104DA00000018885C3AF03D0B7AF0AD002D0B7BF28
:104DB0000AD0C351B75D07E303E1B651C25D03E218
:104DC000CAB201D0889515D0B7AF03D0C3AF0AD00F
:104DD00002D0C3BF0DD0B751C35D0AE303E1C25196
:104DE000B65D06E2F497010116970001888501D0AF
:104DF0008895C3AF03D0BBAF0AD002D0BBBF0FD0E2
:104E0000C351BB5D0CE303E1BA51C25D08E201018D
:104E100016A906D0169B169D1699000188870101D8
:104E20000001BBAF03D0C3AF0AD002D0C3BF0ED0C6
:104E3000BB51C35D0BE303E1C251BA5D07E201015F
:104E400016B702D0000102D000018897BDAF03D091
:104E5000C3AF0AD002D0C3BF0DD0BD51C35D0AE3BA
:104E600003E1C251BC5D06E2010116A702D0169D06
:104E7000168B0001C3AF03D0C1AF0AD002D0C1BFAF
:104E80000FD0C351C15D0CE303E1C051C25D08E224
:104E9000010116A904D016BB02D0168B168D000195
:104EA000010116B71ED016B91CD00001E06B69973E
:104EB000C56BC46BC769C6690101126B169B169D51
:104EC0000001C3AF03D0BBAF0AD002D0BBBF08D034
:104ED000C351BB5D05E303E1BA51C25D01E28887BE
:104EE000010116A707D0000187AF02D0010102D04F
:104EF0000101169D16B702D016A924D0122B12510B
:104F0000320807E21251340804E3C3C0C5F0C2C03E
:104F1000C4F01251640807E21251660804E3C3C0EA
:104F2000C7F0C2C0C6F01251C8080CE20001C4515B
:104F3000C65D05E1C551C75D02E1698701D069978A
:104F40000101126BBA9C0C5301E1BA8CCAA00DD0BE
:104F50000001FF2BFF510101D75D06E2010E0001A8
:104F6000FE6FD8C1FFF0010104D00001FE6BFF6BA2
:104F700001010001F53D12D0CAB60AD001010D2B86
:104F80000D51D75D03E20C6BD8C10DF105D00001C6
:104F9000010E01010C6F0D6B11D00001CAA60BD0E0
:104FA0000101112B1151D75D04E2010E106FD8C120
:104FB00011F104D000010101106B116B0001E853E5
:104FC00022E1CBB819D00101032B0351D75D12E2C6
:104FD000D8C103F1132BD8B4142B145303E113518C
:104FE000050807E2010E146FF50E136F010E026F34
:104FF00001D0026B07D00001010E0101026F036BAB
:10500000146B136B0001E83D11D0CBB80AD001013D
:10501000032B0351D75D03E2026BD8C103F105D026
:105020000001010E0101026F036B0001CBBA0AD02F
:105030000101012B0151D75D03E2006BD8C101F1E1
:1050400005D00001010E0101006F016B0001F53D6B
:1050500012D0010E01010E6FCAB408D0052B055104
:10506000D75D03E2046BD8C105F103D0010E046FD4
:10507000056B11D00001010E0101046FCAB408D004
:105080000F2B0F51D75D03E20E6BD8C10FF103D088
:10509000010E0E6F0F6BCAA223D016A921D00001FA
:1050A000C3AF03D0BDAF12D004D0BDAF02D0010159
:1050B00017D0C351BD5DD8B002D0010111D006E1B7
:1050C000BC51C25DD8A002D001010AD00101072B5A
:1050D0000751010804E2010E066F030E076F02D0AC
:1050E000066B076B0001C851BA25016EC951BB217F
:1050F000036E015003AE03D0C3AF0AD002D0C3BFCA
:1051000014D00350C35D11E303E1C251015C0DE211
:10511000CAA80BD00101092B0951010804E2010EB4
:10512000086F030E096F04D000010101086B096BC1
:10513000CAAA09D00B2B0B51010804E2010E0A6F19
:10514000030E0B6F02D00A6B0B6B0001FE2D01D01A
:1051500069D0F53D67D0F1534DE101011691000191
:10516000F4AF03D0010116810001F23D11D001011D
:105170001693000188A503D00101168300010101E7
:105180001695000188A703D001011685000131D0D2
:10519000010116A703D00001888F0101000169AB4E
:1051A00007D0010116B902D0000102D00001F4813C
:1051B00088AF0ED088A50CD0F32B01011683000117
:1051C000F351320805E2889F010116930001F36B49
:1051D000F4A10FD088A70DD0F32B01011685000193
:1051E000F351320806E2F491699B01011695000122
:1051F000F36B18D0010116910001F4AF03D0010147
:1052000016810001010116930001F4AF03D00101E2
:1052100016830001010116950001F4AF03D00101CE
:1052200016850001F53D05D0EF3D01D002D0F4898F
:10523000F49B0101025309E10001EF3D03D001019C
:1052400004D00001F48BF4990101025308E100013C
:10525000EF3D02D0010103D0010116B90FD0005378
:1052600010E10001F53D01D002D001010AD0EF3D6F
:1052700002D0010106D0010116A903D00001F48D6E
:1052800001010001F55355E1FE531CE101011053EA
:10529000D8B402D0000116D00653D8B402D0000111
:1052A00011D00853D8B402D000010CD00A53D8B49E
:1052B00002D0000107D017A302D0000103D017A528
:1052C00003D000010101169F0001FE531FE10101FF
:1052D0001053D8B402D0000119D00653D8B402D06C
:1052E000000114D00853D8B402D000010FD00A53E3
:1052F000D8B402D000010AD017A302D0000106D012
:1053000017A502D0000102D0168F0001FE5304E160
:105310000101105303E00001010117910001FE5348
:1053200008E101011053D8B402D0000102D0178166
:105330000001F63D2ED0F53D0FD0BE90F4BFBE80EB
:10534000BE92010116B1BE82BE9416B3BE84BA9E4F
:1053500016B5BA8E10D00001BE90010117B1BE8003
:10536000BE9216BFBE82BE94000188B5BE84BA9EAE
:1053700088B7BA8E0101BC9616B7BC86BC9416B924
:10538000BC84BC9216BBBC82BC9016BDBC802AD02B
:105390000001F53D09D0BE90010116B3BE80BE925A
:1053A00016B5BE820DD00001BE90010116BFBE80B1
:1053B000006A16BF002A010E001ABE9200B0BE821B
:1053C000BE9416B7BE84BA9E16B9BA8EBC9616B7EE
:1053D000BC86BC9416B9BC84BC9216BBBC82BC9083
:1053E00016BDBC800001F55300E13C0E996EB00E75
:1053F000986E00003901A89D00013CEF10F00001FB
:10540000CC8C3D01E1B71BD0E1B319D0E1AD08D0A0
:105410006F0040F794F00001889D879B05D03D0107
:105420006F0040F7A9F00001A9C0C3F094C0C2F01A
:1054300088B903D0FF0EC21BC31B03D03D01E1930B
:105440000001E06B3D01D0513901A69500013CEF10
:1054500010F000016983B8A802D0CF0EB76E2C0EF1
:10546000B66E3901A39F00013CEF10F03901A3A7EC
:10547000FED73D01F9511A6EE851016E1AA204D00F
:10548000F299F783F993F289000149EF2AF00001BC
:10549000EDD701C0D7F1625315E161513F0812E326
:1054A00062C003F06151612BD8B4622B0101D86F47
:1054B000210ED825E96E000E0320EA6E60005FF72A
:1054C000EFFF0001646B636B3901A39700013CEFB0
:1054D00010F0202020444554454354414E444F2071
:1054E000202000002020204C4F4F50494E47202EB6
:1054F0002E2E2E2E0000202020204C4F4F50494EA3
:105500004720202020200000202020204445544512
:1055100043544544202020200000202020204C4FD0
:105520004F50494E472020202020000020202020DE
:1055300050524553454E5445202020200000202045
:1055400020204C4F4F50494E472020202020000063
:1055500020204E4F54204445544543544544202078
:105560000000202020204C4F4F50494E4720202043
:105570002020000020202020415553454E54452036
:10558000202020200000202020434845434B494E46
:1055900047202020202000002020504C454153452A
:1055A00020574149542E2E2E0000202056455249A6
:1055B000464943414E444F202020000020202045F2
:1055C00053504552452E2E2E202020200000202012
:1055D00056455249464943414E444F202020000041
:1055E000202020414755415244452E2E2E20202078
:1055F0000000564D5425303258253032582530326F
:105600005825303258253032582530325800202065
:10561000564D4F5445202020204F46462020000064
:1056200044494725303258253032582530325825E4
:1056300030325825303258253032580020444947FE
:10564000494C494E4B20204F46462020000020491F
:105650004E564552534F522020204F4B20200000E1
:10566000202020202020202020202020202020203A
:10567000000020494E564552534F5220204F464677
:10568000202000002020202020202020202020205A
:1056900020202020000020504F5254412020464519
:1056A00043484144412000004349434C4F53202587
:1056B000394C7500205055455254412043455252B3
:1056C0004144412000004349434C4F532025394C6D
:1056D00075002020434C4F53454420444F4F5220E7
:1056E000202000004359434C45532025394C750078
:1056F00020504F52544120204645434841444120C8
:1057000000004349434C4F532025394C750020502D
:1057100055455254412043455252414441200000D6
:105720004349434C4F532025394C75002020434CAE
:105730004F53454420444F4F5220202000004359EE
:10574000434C45532025394C7500504F525441204D
:105750004645434841444125334C75004349434C39
:105760004F532025394C75005055455254414345FF
:10577000525241444125334C75004349434C4F53E9
:105780002025394C7500444F4F5220434C4F534510
:1057900044202025334C75004359434C4553202564
:1057A000394C750058312025632563256325632511
:1057B00063256325632563204C502025630020204A
:1057C00020555341522042462020000020202050E6
:1057D000415241205245534554415220000020205F
:1057E00020555341522042462020000020202050C6
:1057F000415241205245534554415220000020203F
:1058000055534152202042412020202020200000DA
:1058100020205041524120464543484152202020FB
:105820000000583120256325632563256325632502
:105830006325632563204C502025630058312025C3
:10584000632563256325632563256325632563201D
:105850004C50202563004359434C45532025394C77
:1058600075004349434C4F532025394C750058313E
:10587000202563256325632563256325632563252B
:1058800063204C502025630020504F52544120206B
:10589000464543484144412000004349434C4F534F
:1058A0002025394C75002050554552544120434520
:1058B00052524144412000004349434C4F5320255C
:1058C000394C75002020434C4F53454420444F4FE2
:1058D0005220202000004359434C45532025394C89
:1058E00075005831202563256325632563256325CD
:1058F0006325632563204C50202563002020454EFE
:105900005452454142455254412020200000434911
:10591000434C4F532025394C75002020454E54529E
:10592000454142494552544F202000004349434CD1
:105930004F532025394C7500202020444F4F5220D2
:10594000414A41522020202000004359434C4553F6
:105950002025394C750058312025632563256325A2
:10596000632563256325632563204C502025630050
:1059700020504F5254412020414252494E444F2022
:1059800000005055455254412041425249454E4431
:105990004F2000002020444F4F52204F50454E4989
:1059A0004E4720200000524544555A2020204142B5
:1059B00045525455524100005245445543495220E6
:1059C000415045525455524100002020534C4F57EE
:1059D000204F50454E494E47202000005831202589
:1059E000632563256325632563256325632563207C
:1059F0004C502025630020504F52544120464543CF
:105A000048414E444F2000005055455254412043D8
:105A1000455252414E444F2000002020444F4F52E7
:105A200020434C4F53494E472020000052454455D7
:105A30005A2046454348414D454E544F000052457B
:105A40004455434520454E204349455252450000A8
:105A50002020534C4F5720434C4F53494E47202052
:105A600000004552524F2032202020202020434F5A
:105A70004D4D0000434F4E53554C544152204D4123
:105A80004E55414C00004552524F203120202020DD
:105A90002020434F4D4D0000434F4E53554C544131
:105AA00052204D414E55414C00004552524F20323C
:105AB000202020202020434F4D4D0000434F4E53C7
:105AC000554C544152204D414E55414C00006F0001
:105AD00048FF91F1D29E3901E16B0F0EE06FE59D19
:105AE000E59FE581E351E59DE58F010191BFD28EF0
:105AF0000001906F6F0048FF91F1D29E3901E16B78
:105B0000100EE06FE59DE59FE581E351E59DE58F92
:105B1000010191BFD28E0001916F6F0048FF91F19A
:105B2000D29E3901E16B110EE06FE59DE59FE581A5
:105B3000E351E59DE58F010191BFD28E0001926F87
:105B40006F0048FF91F1D29E3901E16B120EE06FB8
:105B5000E59DE59FE581E351E59DE58F010191BF5D
:105B6000D28E0001936F93C0CDF092C0CCF091C063
:105B7000CBF090C0CAF03EEF6DF00101A9B102D0A8
:105B8000BD9601D0BD86C596A9B302D0BD9401D003
:105B9000BD84C594A9B502D0BD9201D0BD82C59285
:105BA000A9B702D0BD9001D0BD80C5900000C498B7
:105BB000BC880400020E006E002EFED7C498BC986C
:105BC00000011200C49ABC9A04004F0E006E002E11
:105BD000FED700000101A65303E0C49ABC8A02D09C
:105BE000C49ABC9A0000C498BC98A739A86F0F0E3D
:105BF000A817A8C1A9F10001C0DF0101A7510F0B2F
:105C0000A86FA96F0001B9DF1200010EEA6ECE0E77
:105C1000E96EEF5011E0050E016EBF0E006E04003C
:105C2000002EFDD7012EF9D72E0E006E002EFED7C6
:105C300000000400EF2EEFD712000101A32D01D0C8
:105C400003D0400EA46F01D0A46B010EA25DA42767
:105C5000A4518009A56FA66BA76F0001B3DF1200E6
:105C60000101A1510C0A000107E0060A11E0070A30
:105C700017E0050A1CE022D00101A66B010EA76FF8
:105C80000001A0DF020E0101CE6F0001BEDF1DD0BA
:105C9000010E0101A26F020EA36F0001CEDF15D02D
:105CA000010E0101A26FA36F0001C7DF0ED0010139
:105CB000A66B100EA76F000185DF07D0010E010152
:105CC000A66FA1C1A7F100017DDF12000C0E01013A
:105CD000A16F0001C5DF1200C49ABC9AC498BC9899
:105CE0000F0E0101CE6F000190DF0101916B915108
:105CF00002080CE3030EA96F00013FDF050E01014E
:105D0000CE6F000182DF0101912BF1D7020EA96F46
:105D1000000133DF0101916B915103080EE3036A27
:105D2000915100014FEC10F00101926FA66BA76F2B
:105D3000000148DF0101912BEFD7000112000101A2
:105D4000925194036F00CCFF01F06F00D0FF00F080
:105D50009503F350002693519403F3500020026EF4
:105D6000000112008E0E006E94C101F093C102F08A
:105D7000036A015209E102C001F0026A080E005EE6
:105D8000015202E1006A08D0D89001BE04D0023668
:105D900001360006F9D7019E120001019351D8B4D3
:105DA000A5D09F6F9751D8B4A1D09F5F05E37F0E18
:105DB0009F27D8B09BD006D0810E9F5FD8A096D0E9
:105DC000D8B494D09FC100F0016A026A036A9E6B46
:105DD00094C19DF19D8F95C19CF196C19BF1190EC7
:105DE0009F6F9A519B5F0DE2010E9C5F0AE29D5FDF
:105DF00008E29E5F06E29E2B9D2B9C2B9A519B27CF
:105E000028D099519C5F12E2010E9D5F0FE29E5FC8
:105E10000DE29E2B9D2B99519C279A519B2719E3AC
:105E20009C2B17E19D2B15E19E2B13D098518009D7
:105E30009D5F0EE2010E9E5F0BE29E2B9851800942
:105E40009D2799519C27E9E39D2BE7E19E2BE5D700
:105E500003809F2F01D00BD0D8909B379C379D3764
:105E60009E37D890033602360136A037BAD7A0A1A4
:105E700006D0D890013202320332A03302D000069D
:105E800035E0A0BF1ED0D8909B379C379D379E37FA
:105E90009A519B5F07E2010E9C5F04E29D5F02E264
:105EA0009E5F1AE399519C5F05E2010E9D5F02E23D
:105EB0009E5F12E3985180099D5F03E2010E9E5F91
:105EC0000BE3032A09E1022A07E1012A05E1002A7E
:105ED0000DE001320232033294C19FF198519F1BB1
:105EE0009FAF02D0018E06D0019E04D0006A016AE5
:105EF000026A036A000130EF30F001019E51D8B40C
:105F000074D0006EA251D8B470D0002604E3810E84
:105F100000266BE204D07F0E005E67E366E09FC15F
:105F2000A6F1A351A61B9F8FA38FA151A5036F00BC
:105F3000D0FFA8F1A051A4036F00D0FF03F06F00C1
:105F4000CCFFA7F1A503F350A827F450A723000E18
:105F50000322A151A403F350A827F450A723000E55
:105F6000026A032202229F51A503F350A727F4508F
:105F70000322000E02229F51A403F3500326F45083
:105F80000222000E016A0122A151A303F350A727A8
:105F9000F4500322000E02220122A051A303F35069
:105FA0000326F4500222000E01229F51A303F35056
:105FB0000226F4500122002A01BE05D0A73703367D
:105FC000023601360006000EA7AF0AD0032A0222CD
:105FD0000122015005E1025003E1035001E1002AD2
:105FE000A6BF018EA6AF019E04D0006A016A026AB4
:105FF000036A000112008E0E006E01019351005ED3
:1060000094C102F095C101F0028E005209E0D890CF
:10601000025202E1015204E002320132002EF7D7AF
:1060200094AF05D0011E021E012AD8B4022A000135
:106030005FEF30F092C194F191C193F193DE03C010
:1060400096F102C095F101C094F100C093F10101F5
:106050009A6B996B480E986F850E976F00019DD6CD
:1060600003C0D2F002C0D1F001C0D0F000C0CFF028
:10607000BA51B65D006EBB51B75900C0D3F0D46FB2
:10608000D4C094F1D3C093F16DDE03C0A1F102C07E
:10609000A0F101C09FF100C09EF1D2C0A5F1D1C016
:1060A000A4F1D0C0A3F1CFC0A2F127DF03C096F1C5
:1060B00002C095F101C094F100C093F19CD702C0D9
:1060C000D4F001C0D3F0D3C001F0D4C002F012006C
:1060D0000A0E0101CE6F000198DD010E0101A26FD1
:1060E000A36F0001AADD12000900F55211E06F0054
:1060F000D8FF95F16F00DCFF96F16F00D4FFA1F19E
:10610000AFDD600057F6F6FF60005BF6F7FFECD7F7
:1061100012000A0E0101CE6F000177DD010E0101B0
:10612000A26F020EA36F000188DD1200C39CBB9C0E
:10613000080E016E00D00000018E10D0019E0101FA
:1061400091330001D8B0BB8CD8A0BB9C018C06D089
:10615000019C012EF4D700D00000BB8C840EE96EA8
:10616000E92EFED700D0000001BEE8D701BCF0D771
:1061700012000B0EA56EDC0EA46E000096C1ADF0F1
:1061800095C1ACF094C1ABF093C1AAF09AC1B1F043
:1061900099C1B0F098C1AFF097C1AEF0B56BB46BD8
:1061A000B36BB26B39015B51040000011200016650
:1061B00003D0026602D008D0022A600003F0EEFF8E
:1061C000012EFBD7022EF9D739EF31F00101D46946
:1061D000D369D051D007000A28E060003FF7EAFFFA
:1061E000CE51CE2BD8B4CF2BE96EEF50D319D16F4F
:1061F000D4C1D2F1D4C1D3F1D46BD1C1D5F1D66B16
:10620000D890D135026ED635036E025060000FF083
:10621000F7FF000159EC10F009006F00D4FF03F004
:106220000101D31B0350D41BD4D7D3C101F0D4C177
:1062300002F0000112003901A3A9FED73D01EA6F67
:10624000000112000101AF5303E1000E016EA1D164
:10625000D890AF35030F020FB46FB56BD8B0B52B24
:10626000EA6A7C0EE96E006A026A0A0E016E00019B
:106270009ED7ACC17CF0030E7D6FAEC17EF00001F5
:10628000ADC17FF000010001806BAFC181F0000162
:106290000101CF6B7C0ECE6F060ED06F000196DF32
:1062A00002C0B3F101C0B2F1B2C182F00001B3C1CA
:1062B00083F000010101BA6BBA510408D8A067D17C
:1062C0000001626B616B646B636BBB84050E010143
:1062D000CE6F00019ADC0101B76BB66BB75314E1C6
:1062E000B651070811E37C0EB625E96E000EB72102
:1062F000EA6E6F00BCFFC0F1C05100019CDF0101DC
:10630000B62BD8B4B72BEAD73D01F9AFFED7F98F3A
:1063100039019387BB940001626B616B050E01012B
:10632000B96FDC0EB86FB851B91118E000016251B5
:106330000101B55D13E308E1B4510001615DD8A02E
:1063400002D001010BD00101010ECE6F00015DDC16
:106350000101B851D8B4B907B807E5D73901939707
:10636000000162510101B55D0AE308E1B451000189
:10637000615DD8A002D0010102D0010106D1B55162
:106380000001625D12E305E10101B4510001615DAC
:106390000CE30101B4510001615D006E0101B551D2
:1063A00000016259036E005002D0036A000E010121
:1063B000BD6F03C0BEF1BF6BBC6BBB6BBC51BE5DA0
:1063C000D8A0DDD004E1BB51BD5DD8A0D8D0210E4E
:1063D000BB25E96E000EBC21EA6EAC51EF5CD8A47F
:1063E000CAD0010EBB25C06F000EBC21C16F210EAB
:1063F000C025E96E000EC121EA6EEF500308D8A453
:10640000BAD0020EBB25C06F000EBC21C16F210E99
:10641000C025E96E000EC121EA6E6F00BCFFC2F11B
:10642000D890AF35C25DD8A4A6D0210EBB25016E91
:10643000000EBC21036E01C0C0F1C16F020EB45D3D
:10644000C26F000EB559C36F03C0CFF101C0CEF1CA
:10645000C2C1D0F10001BADE02C0B3F101C0B2F195
:10646000B2C1C0F10101B451BB25C16FB551BC210E
:10647000C26F020EC15F000EC25B210EC125E96E24
:10648000000EC221EA6EEF50B25DD8A474D0B3C141
:10649000C0F1B451BB25C16FB551BC21C26F010E13
:1064A000C15F000EC25B210EC125E96E000EC22144
:1064B000EA6EEF50C05DD8A45ED0B051B11154E087
:1064C000B76BB66BB75350E1AF51B65D4DE2D890A4
:1064D000B635026EB735036E0250B025016EB1516C
:1064E000032203C0C1F1030EBB25C26F000EBC2105
:1064F000C36FD890B635026EB735036E0250C2270F
:106500000350C323210EC225E96E000EC321EA6E9B
:106510006F00BCFFC4F1040EBB25C56F000EBC218B
:10652000C66FD890B635026EB735036E0250C527D8
:106530000350C623210EC525E96E000EC621EA6E62
:106540006F00BCFFC7F1600007F7EAFF600007F0CB
:10655000E9FF600013F7ECFFED5260001FF7EFFF5B
:10656000B62BD8B4B72BAED7010EBF6F0001626B4C
:10657000616B010104D0BB2BD8B4BC2B1FD7BF5318
:10658000D8B403D0010E016E04D0BA2B95D6000EFC
:10659000016E0001120001017FA3E4D00F0EAB6F6A
:1065A000AB5126080DE3D890AB35036A1B0FE96E9B
:1065B000010E0320EA6EEC6AED52EF6AAB2BF0D7C6
:1065C000010EAC6F030EAE6FE80EAD6F090EAF6F2C
:1065D000010EB16F910EB06F000134DE015214E074
:1065E00092C13AF191C139F198C13CF197C13BF1A7
:1065F0009EC13EF19DC13DF1A0C140F19FC13FF15F
:10660000A2C142F1A1C141F1010E0101AC6F040E22
:10661000AE6FAD6B060EAF6F010EB16F910EB06F26
:10662000000110DE015210E092C144F191C143F12A
:1066300094C146F193C145F196C148F195C147F126
:106640009CC14AF19BC149F1010E0101AC6F040EDE
:10665000AE6F230EAD6F0D0EAF6F010EB16F910EC9
:10666000B06F0001EFDD015210E092C14CF191C119
:106670004BF1A6C14EF1A5C14DF1A8C150F1A7C182
:106680004FF1AAC152F1A9C151F1010E0101AC6F44
:10669000040EAE6F360EAD6F0C0EAF6F010EB16F04
:1066A000910EB06F0001CEDD01521CE092C154F199
:1066B00091C153F194C156F193C155F196C158F16E
:1066C00095C157F198C15AF197C159F19AC15CF13E
:1066D00099C15BF19CC15EF19BC15DF1A8C160F104
:1066E000A7C15FF1010E0101AC6F040EAE6FA70EE2
:1066F000AD6F010EAF6FB16F910EB06F0001A2DDF3
:10670000015204E092C162F191C161F1010E0101F7
:10671000AC6F040EAE6FE00EAD6F010EAF6FB16FD8
:10672000910EB06F00018EDD015204E092C164F160
:1067300091C163F1010E0101AC6F070EAE6F4F0EF8
:10674000AD6F010EAF6FB16F910EB06F00017ADDCA
:10675000015209E092C166F191C165F10101686BD6
:10676000010E676F0001120001017FA301D07FA716
:1067700095D0050E916F100E926F936B120E946F61
:10678000956B180E966F300E976F070ECB6F0F0E2E
:10679000CA6FCA51260845E3036ACB51910F016EB7
:1067A000010E032203C0CFF1D890CA35036A1B0F34
:1067B000E96E010E0320EA6E6F00B0FFD1F1ED52D9
:1067C0006F00BCFFD0F160003FF7EAFF600007F008
:1067D000E9FF600047F7EFFF010ECB25036A910F39
:1067E000016E010E032203C0CFF1D890CA35036AAF
:1067F0001B0FE96E010E0320EA6E6F00B0FFD1F1AE
:10680000ED526F00BCFFD0F160003FF7EAFF60007F
:1068100007F0E9FF600043F7EFFF020ECB27CA2B1A
:10682000B8D7010ECF6F910ECE6F370ED06F00012B
:10683000CDDC02C0CDF101C0CCF10101CCC1C8F169
:10684000CDC1C9F1010E0001656FBB843D01F98F17
:106850000101CA6BCA51380810E3036ACA51910F8B
:10686000E96E010E0320EA6E6F00BCFFCEF1CE513F
:106870000001E1DC0101CA2BEDD73D01F9AFFED7E4
:10688000F98FBB940001626B616B140E0101CE6F36
:10689000000105EC2EF0626B616B0101000112003A
:1068A000955105084CE0A82D39D0D93D07D010DC12
:1068B000640EF66E290EF76E17DC13D0D95307E17C
:1068C00007DC760EF66E290EF76E0EDC0AD0D95173
:1068D0007F0807E168EC30F0880EF66E290EF76E3F
:1068E00003DCD93D07D015DC9A0EF66E290EF76E43
:1068F00074EC30F0D95307E10CDCAC0EF66E290EC7
:10690000F76E74EC30F0D9517F0807E102DCBE0E5F
:10691000F66E290EF76E74EC30F010D068EC30F0A3
:10692000D00EF66E290EF76E74EC30F089EC30F074
:10693000E20EF66E290EF76E74EC30F0B1D712004D
:1069400009006F00D8FF96F16F00DCFF97F16F0030
:10695000D4FFA1F130EC2EF060005BF6F6FF600092
:106960005FF6F7FF0101952F01D002D00001E8D7B3
:106970000001120001019551016A945D03E294C186
:1069800000F00CD0006A080E966F943700369551CF
:10699000005CD8B0006E0136962FF7D700011200C8
:1069A000015092C194F1640E0101956F0001E2DF84
:1069B00000C092F10150300E08E1010193A310D004
:1069C00093B70ED093B9200E04D0010193979399F9
:1069D0009381012601C0A1F1000130EC2EF00101EC
:1069E00092C194F10A0E956F0001C4DF00C092F1CC
:1069F0000150300E08E1010193B70BD093A109D0EB
:106A000093B9200E0001012601C0A1F130EC2EF057
:106A10000101300E922792C1A1F1000130EC2EF05D
:106A200012003EDFF96BFA6B010191910001955163
:106A30000308D8B47DD068EC30F0780EF66E260EE0
:106A4000F76E74EC30F089EC30F08A0EF66E260E9C
:106A5000F76E74EC30F0952D31D068EC30F09C0E70
:106A6000F66E260EF76E74EC30F089EC30F0AE0E58
:106A7000F66E260EF76E74EC30F06F0048FF92F160
:106A8000D29E3901E16B330EE06FE59DE59FE58114
:106A9000E351E59DE58F010192BFD28E0001FD6FAC
:106AA00001019181080E926FFA0ECE6F000105EC84
:106AB0002EF00101922FF8D700013AD09551040829
:106AC00036E168EC30F0C00EF66E260EF76E74EC10
:106AD00030F089EC30F0D20EF66E260EF76E74ECC4
:106AE00030F0FD69D250006ED29E3901E16B330E59
:106AF000E06F6000F7F3E3F9E59DE59FE585550E4E
:106B0000E66FAA0EE66FE583E5B3FED7E595E59D52
:106B1000E58F0050D212080E0101926FFA0ECE6F6F
:106B2000000105EC2EF00101922FF8D700017FD76C
:106B3000010191A1A1D0000168EC30F0E40EF66EE5
:106B4000260EF76E090E0101956F0001F9DEFDC0FA
:106B500092F1130E0101936F000122DFF00EF66E29
:106B6000260EF76E040E0101956F0001E9DE89EC37
:106B700030F0F60EF66E260EF76E74EC30F0640E02
:106B80000101CE6F000105EC2EF09551040801E1E2
:106B9000FD2B640E0101CE6F000105EC2EF0952D4A
:106BA00001D0FD079551030865E1FF0EFD1BD25092
:106BB000006ED29E3901E16B330EE06F6000F7F397
:106BC000E3F9E59DE59FE585550EE66FAA0EE66FB4
:106BD000E583E5B3FED7E595E59DE58F0050D2123C
:106BE0000400840E006E002EFED700D06F0048FF18
:106BF00092F1D29EE16B330EE06FE59DE59FE5815A
:106C0000E351E59DE58F010192BFD28E0001FD6F3A
:106C1000FF0EFD1B68EC30F0080EF66E270EF76EC7
:106C2000090E0101956F00018BDEFDC092F1130E7C
:106C30000101936F0001B4DE140EF66E270EF76E9D
:106C4000040E0101956F00017BDE89EC30F01A0E15
:106C5000F66E270EF76E74EC30F0080E0101926F9D
:106C6000FA0ECE6F000105EC2EF00101922FF8D73D
:106C7000919100015DD701010001CDEF42F010DEDE
:106C8000F96BFA6B95510308D8B482D068EC30F0F8
:106C90008C0EF66E280EF76E74EC30F089EC30F046
:106CA0009E0EF66E280EF76E74EC30F0952D36D0F1
:106CB00068EC30F0B00EF66E280EF76E74EC30F023
:106CC00089EC30F0C20EF66E280EF76E74EC30F0E0
:106CD000F66BD250006ED29E3901E16B370EE06F39
:106CE0006000DBF3E3F9E59DE59FE585550EE66F72
:106CF000AA0EE66FE583E5B3FED7E595E59DE58F42
:106D00000050D212080E0101916FFA0ECE6F0001F1
:106D100005EC2EF00101912FF8D7000195510408E0
:106D200036E168EC30F0D40EF66E280EF76E74EC97
:106D300030F089EC30F0E60EF66E280EF76E74EC4B
:106D400030F0F669D250006ED29E3901E16B370EF9
:106D5000E06F6000DBF3E3F9E59DE59FE585550E07
:106D6000E66FAA0EE66FE583E5B3FED7E595E59DF0
:106D7000E58F0050D212080E0101916FFA0ECE6F0E
:106D8000000105EC2EF00101912FF8D700017AD710
:106D9000D4EF42F085DDF96BFA6B010191910001AE
:106DA00095510308D8B47DD068EC30F0C40EF66E6F
:106DB000250EF76E74EC30F089EC30F0D60EF66EDE
:106DC000250EF76E74EC30F0952D31D068EC30F074
:106DD000E80EF66E250EF76E74EC30F089EC30F0AC
:106DE000FA0EF66E250EF76E74EC30F06F0048FF69
:106DF00092F1D29E3901E16B320EE06FE59DE59F85
:106E0000E581E351E59DE58F010192BFD28E00013E
:106E1000FB6F01019181080E926FFA0ECE6F000197
:106E200005EC2EF00101922FF8D700013AD09551D0
:106E3000040836E168EC30F00C0EF66E260EF76EA4
:106E400074EC30F089EC30F01E0EF66E260EF76E04
:106E500074EC30F0FB69D250006ED29E3901E16BC8
:106E6000320EE06F6000EFF3E3F9E59DE59FE58505
:106E7000550EE66FAA0EE66FE583E5B3FED7E595FE
:106E8000E59DE58F0050D212080E0101926FFA0EB7
:106E9000CE6F000105EC2EF00101922FF8D7000112
:106EA0007FD7010191A18BD0000168EC30F0300E4A
:106EB000F66E260EF76E0D0E0101956F000140DD96
:106EC000FBC092F1130E0101936F000169DD89ECA3
:106ED00030F0420EF66E260EF76E74EC30F0640E53
:106EE0000101CE6F000105EC2EF09551040801E17F
:106EF000FB2B640E0101CE6F000105EC2EF0952DE9
:106F000001D0FB079551030858E1D250006ED29E84
:106F10003901E16B320EE06F6000EFF3E3F9E59DBC
:106F2000E59FE585550EE66FAA0EE66FE583E5B3AE
:106F3000FED7E595E59DE58F0050D2120400840E42
:106F4000006E002EFED700D06F0048FF92F1D29E57
:106F5000E16B320EE06FE59DE59FE581E351E59D34
:106F6000E58F010192BFD28E0001FB6F68EC30F01B
:106F7000540EF66E260EF76E0D0E0101956F000190
:106F8000DFDCFBC092F1130E0101936F000108DDFD
:106F900089EC30F0660EF66E260EF76E74EC30F06B
:106FA000080E0101926FFA0ECE6F000105EC2EF073
:106FB0000101922FF8D79191000173D701010001CF
:106FC000DBEF42F06DDCF96BFA6B95510308D8B436
:106FD00082D068EC30F0580EF66E250EF76E74EC29
:106FE00030F089EC30F06A0EF66E250EF76E74EC18
:106FF00030F0952D36D068EC30F07C0EF66E250E14
:10700000F76E74EC30F089EC30F08E0EF66E250ED3
:10701000F76E74EC30F0EF6BD250006ED29E3901F7
:10702000E16B310EE06F6000BFF3E3F9E59DE59F92
:10703000E585550EE66FAA0EE66FE583E5B3FED74C
:10704000E595E59DE58F0050D212080E0101916F84
:10705000FA0ECE6F000105EC2EF00101912FF8D74A
:1070600000019551040836E168EC30F0A00EF66E90
:10707000250EF76E74EC30F089EC30F0B20EF66E3F
:10708000250EF76E74EC30F0EF69D250006ED29E90
:107090003901E16B310EE06F6000BFF3E3F9E59D6C
:1070A000E59FE585550EE66FAA0EE66FE583E5B32D
:1070B000FED7E595E59DE58F0050D212080E01013F
:1070C000916FFA0ECE6F000105EC2EF00101912FA9
:1070D000F8D700017AD7E2EF42F050EC34F0F96BC8
:1070E000FA6B95510308D8B482D068EC30F02C0EBE
:1070F000F66E270EF76E74EC30F089EC30F03E0E31
:10710000F66E270EF76E74EC30F0952D36D068ECE5
:1071100030F0500EF66E270EF76E74EC30F089ECFE
:1071200030F0620EF66E270EF76E74EC30F0F16BF5
:10713000D250006ED29E3901E16B2F0EE06F6000DD
:10714000C7F3E3F9E59DE59FE585550EE66FAA0EC9
:10715000E66FE583E5B3FED7E595E59DE58F005045
:10716000D212080E0101916FFA0ECE6F000105ECEC
:107170002EF00101912FF8D700019551040836E156
:1071800068EC30F0740EF66E270EF76E74EC30F08B
:1071900089EC30F0860EF66E270EF76E74EC30F048
:1071A000F169D250006ED29E3901E16B2F0EE06F73
:1071B0006000C7F3E3F9E59DE59FE585550EE66FB1
:1071C000AA0EE66FE583E5B3FED7E595E59DE58F6D
:1071D0000050D212080E0101916FFA0ECE6F00011D
:1071E00005EC2EF00101912FF8D700017AD7E9EFD5
:1071F00042F050EC34F0F96BFA6B95510308D8B4B7
:1072000082D068EC30F0980EF66E270EF76E74ECB4
:1072100030F089EC30F0AA0EF66E270EF76E74ECA3
:1072200030F0952D36D068EC30F0BC0EF66E270E9F
:10723000F76E74EC30F089EC30F0CE0EF66E270E5F
:10724000F76E74EC30F0F26BD250006ED29E3901C2
:10725000E16B380EE06F6000CBF3E3F9E59DE59F4D
:10726000E585550EE66FAA0EE66FE583E5B3FED71A
:10727000E595E59DE58F0050D212080E0101916F52
:10728000FA0ECE6F000105EC2EF00101912FF8D718
:1072900000019551040836E168EC30F0E00EF66E1E
:1072A000270EF76E74EC30F089EC30F0F20EF66ECB
:1072B000270EF76E74EC30F0F269D250006ED29E59
:1072C0003901E16B380EE06F6000CBF3E3F9E59D27
:1072D000E59FE585550EE66FAA0EE66FE583E5B3FB
:1072E000FED7E595E59DE58F0050D212080E01010D
:1072F000916FFA0ECE6F000105EC2EF00101912F77
:10730000F8D700017AD7F0EF42F06F00A8FF99F1AB
:107310006F00A4FF98F1010192AF08D0988F98A94F
:10732000982B911F921F912BD8B4922B9239F00970
:10733000946F9427E20F956F320F976F92510F0B56
:10734000952795279727E90F966F962796279139C6
:107350000F0B9627972796379737971F9737915197
:107360000F0B97279437070E936F0A0E96079727F0
:10737000FDE395079627FDE394079527FDE3930723
:107380009427FDE3010EEA6E930EE96E070E981541
:10739000989DED52981507E198B9EE5298B903D02F
:1073A000200E006E20D0E926000EEA22E950970850
:1073B00003E1EA2C01D0988DEF50006E08E198BDF2
:1073C00006D098B922D098B702D0200E0BD098AF33
:1073D00006D02D0E006EED50989D989F04D0988792
:1073E0009899300E00266F00A8FF92F16F00A4FF5D
:1073F00091F100C0A1F1000130EC2EF060004BF6DD
:10740000EAFF600047F6E9FF0101EE5098ADCED7E4
:1074100000011200966BCAB0962B976BCBBA972BD4
:10742000986BCBB8982B996BCAB4992B9A6BCAB24C
:107430009A2B9B6BCAB89B2B9C6BCABA9C2B9D6BDF
:10744000CAB69D2B9D51800DF3500101916F000133
:107450009C51400DF3500101912700019B51200DDB
:10746000F3500101912700019A51100DF3500101D1
:10747000912700019951080DF35001019127000156
:107480009851040DF35001019127D89000019735D0
:107490000101912500019625A76FB4EF3AF0C80EBF
:1074A0000101CE6F000105EC2EF0010ECD6EC80E6D
:1074B0000101CE6F000105EC2EF0020ECD6EC80E5C
:1074C0000101CE6F000105EC2EF0040ECD6EC80E4A
:1074D0000101CE6F000105EC2EF0080ECD6EC80E36
:1074E0000101CE6F000105EC2EF0100ECD6EC80E1E
:1074F0000101CE6F000105EC2EF0200ECD6EC80EFE
:107500000101CE6F000105EC2EF0CD6A1200C00E15
:10751000D21239019387000168EC30F0F40EF66E58
:10752000220EF76E0A0E0101956F0001A0EC34F0F7
:10753000000EE96EC3C092F1C2C091F1E6DE89ECA3
:1075400030F0040EF66E230EF76E0D0E0101956FEE
:107550000001A0EC34F095C092F1030E0101936F8D
:107560000001D0EC34F056D7A751FE0A0FE0030A11
:107570000FE0060A0FE00C0A0FE0180A0FE0300ACD
:107580000FE0600A0FE0C00A0FE010D088DF0FD0D4
:1075900086DF0DD084DF0BD082DF09D080DF07D0FB
:1075A0007EDF05D07CDF03D07ADF01D0CD6AB4D78F
:1075B000F7EF42F0CD6BCC6BCB6BCA6B878DCAC03B
:1075C00090F0CBC091F0CCC092F0CDC093F0D250EF
:1075D000006ED29E3901E16B0F0EE06F600043F246
:1075E000E3F9E59DE59FE585550EE66FAA0EE66F8A
:1075F000E583E5B3FED7E595E59DE58F0050D21212
:10760000D250006ED29EE16B100EE06F600047F228
:10761000E3F9E59DE59FE585550EE66FAA0EE66F59
:10762000E583E5B3FED7E595E59DE58F0050D212E1
:10763000D250006ED29EE16B110EE06F60004BF2F3
:10764000E3F9E59DE59FE585550EE66FAA0EE66F29
:10765000E583E5B3FED7E595E59DE58F0050D212B1
:10766000D250006ED29EE16B120EE06F60004FF2BE
:10767000E3F9E59DE59FE585550EE66FAA0EE66FF9
:10768000E583E5B3FED7E595E59DE58F0050D21281
:107690006F0048FF95F1D29EE16B0F0EE06FE59D04
:1076A000E59FE581E351E59DE58F010195BFD28E10
:1076B0000001906F6F0048FF95F1D29E3901E16B98
:1076C000100EE06FE59DE59FE581E351E59DE58FB7
:1076D000010195BFD28E0001916F6F0048FF95F1B7
:1076E000D29E3901E16B110EE06FE59DE59FE581CA
:1076F000E351E59DE58F010195BFD28E0001926FA8
:107700006F0048FF95F1D29E3901E16B120EE06FD8
:10771000E59DE59FE581E351E59DE58F010195BF7D
:10772000D28E0001936F93C0CDF092C0CCF091C087
:10773000CBF090C0CAF0A1EF3CF08889000E88B968
:10774000010E0101956FD250006ED29E3901E16B9E
:10775000140EE06F600057F6E3F9E59DE59FE585BF
:10776000550EE66FAA0EE66FE583E5B3FED7E59505
:10777000E59DE58F0050D212050E0001CE6FD2506C
:10778000006ED29E3901E16B050EE06F60003BF3A5
:10779000E3F9E59DE59FE585550EE66FAA0EE66FD8
:1077A000E583E5B3FED7E595E59DE58F0050D21260
:1077B000050E0101926F140E916F91C195F1D25097
:1077C000006ED29E3901E16B060EE06F600047F655
:1077D000E3F9E59DE59FE585550EE66FAA0EE66F98
:1077E000E583E5B3FED7E595E59DE58F0050D21220
:1077F00092C195F1D250006ED29EE16B070EE06F00
:1078000060004BF6E3F9E59DE59FE585550EE66FD3
:10781000AA0EE66FE583E5B3FED7E595E59DE58F16
:107820000050D212FE0E0101946FD40E936F93C1DB
:1078300095F1D250006ED29E3901E16B080EE06FD7
:1078400060004FF6E3F9E59DE59FE585550EE66F8F
:10785000AA0EE66FE583E5B3FED7E595E59DE58FD6
:107860000050D21294C195F1D250006ED29EE16BBD
:10787000090EE06F600053F6E3F9E59DE59FE585AD
:10788000550EE66FAA0EE66FE583E5B3FED7E595E4
:10789000E59DE58F0050D2120001E869D250006EDC
:1078A000D29E3901E16B150EE06F6000A3F3E3F99E
:1078B000E59DE59FE585550EE66FAA0EE66FE5832B
:1078C000E5B3FED7E595E59DE58F0050D212140E85
:1078D0000001F76FD250006ED29E3901E16B0D0EA0
:1078E000E06F6000DFF3E3F9E59DE59FE585550E68
:1078F000E66FAA0EE66FE583E5B3FED7E595E59D55
:10790000E58F0050D212140E0001F86FD250006EB5
:10791000D29E3901E16B0B0EE06F6000E3F3E3F9F7
:10792000E59DE59FE585550EE66FAA0EE66FE583BA
:10793000E5B3FED7E595E59DE58F0050D212000135
:1079400039D668EC30F0160EF66E230EF76E74EC36
:1079500030F089EC30F0280EF66E230EF76E74ECE2
:1079600030F0080E0101956FFA0ECE6F000105ECA4
:107970002EF00101952FF8D70001FEEF42F050ECF8
:1079800034F0F96BFA6B50EC34F095510308D8B42D
:10799000B1D068EC30F0040EF66E280EF76E74EC81
:1079A00030F089EC30F0160EF66E280EF76E74EC9F
:1079B00030F0878F952D7DD0BA51C25D006EBB51DE
:1079C000C35900C0C8F0C96F68EC30F0280EF66EDD
:1079D000280EF76E090E0101956F0001A0EC34F03E
:1079E000000EE96EC3C092F1C2C091F18EDC89EC49
:1079F00030F0360EF66E280EF76E090E0101956F07
:107A00000001A0EC34F0000EE96EBBC092F1BAC0E8
:107A100091F17BDC600023F3E3F9D250006ED29E3B
:107A20003901E16B390EE06FE59DE59FE585550E67
:107A3000E66FAA0EE66FE583E5B3FED7E595E59D13
:107A4000E58F0050D212600027F3E3F9D250006EA8
:107A5000D29EE16B3A0EE06FE59DE59FE585550E00
:107A6000E66FAA0EE66FE583E5B3FED7E595E59DE3
:107A7000E58F0050D212000168EC30F0440EF66E33
:107A8000280EF76E74EC30F089EC30F0560EF66E7E
:107A9000280EF76E74EC30F0080E0101916FFA0EAB
:107AA000CE6F000105EC2EF00101912FF8D70001F7
:107AB00021D0955104081DE168EC30F0680EF66E97
:107AC000280EF76E74EC30F089EC30F07A0EF66E1A
:107AD000280EF76E74EC30F0080E0101916FFA0E6B
:107AE000CE6F000105EC2EF00101912FF8D70001B7
:107AF00001D04BD706EF43F001019E51B6089E6FAF
:107B0000036A9FC1A2F19F8FD8909F33A033A13306
:107B100003320232013200329E2FF6D7A2AF0BD0D1
:107B2000001E011E021E031E002AD8B4012AD8B46A
:107B3000022AD8B4032A0001CAEF3DF0E95001013E
:107B4000966F9551986F1CE094C1A1F193C1A0F17B
:107B500092C19FF191C19EF1A56BA46B200EA36F02
:107B6000820EA26F00017DEC2FF003C094F102C0E1
:107B700093F101C092F100C091F10101982FE4D777
:107B800094C1A1F193C1A0F192C19FF191C19EF165
:107B90000001B2D703C094F102C093F101C092F189
:107BA00000C091F1010194AF0DD09607968B911F03
:107BB000921F931F941F912BD8B4922BD8B4932B60
:107BC000D8B4942B3B0E9D6F9A0E9C6FCA0E9B6F80
:107BD0009A6B0A0E986F9551D8B4962BD882010EE5
:107BE000EA6E910EE96E196AD2BE198ED29E94C1C8
:107BF000DEF193C1DDF192C1DCF191C1DBF19DC1F8
:107C0000E2F19CC1E1F19BC1E0F19AC1DFF1000119
:107C10000CEC25F019BED28E0150005213E1010187
:107C20009529985DD8A402D000010CD096510DE0A2
:107C30000F0B985D01E044E296BF42D096BD05D09F
:107C4000200E37D0200E0101961796AB0FD0969BD1
:107C50009551D8A496070050966F2D0EA16F000184
:107C600030EC2EF001019651006E966B9551985DA7
:107C70000DE10050966F2E0EA16F000130EC2EF03A
:107C800001019651006E200E9617000E300E96AB35
:107C900010D0969B9551D8A496070050966F2D0E44
:107CA000A16F000130EC2EF001019651006E966B31
:107CB000300E002600C0A1F1000130EC2EF00101D1
:107CC000D892196AD2BE198ED29E9DC1DEF19CC196
:107CD000DDF19BC1DCF19AC1DBF1E26BE16BE06BA2
:107CE0000A0EDF6F00010CEC25F019BED28E03C026
:107CF0009DF102C09CF101C09BF100C09AF101010D
:107D0000982F6CD7000112009551030811E168EC1F
:107D100030F03A0EF66E230EF76E74EC30F089EC0C
:107D200030F04C0EF66E230EF76E74EC30F0ECD79C
:107D30009551030875E0EDC0EEF0ED51FF0AEE6FCE
:107D40000101946BEEC093F10001B2EC2EF003C080
:107D5000A1F102C0A0F101C09FF100C09EF1550E3B
:107D60000101A56FC10EA46F480EA36F7D0EA26F17
:107D700000017DEC2FF003C0ECF002C0EBF001C07D
:107D8000EAF000C0E9F068EC30F05E0EF66E230E0B
:107D9000F76E0D0E0101956F0001A0EC34F0010E9D
:107DA000E96EECC094F1EBC093F1EAC092F1E9C046
:107DB00091F10101956B0001C1DE250E0101A16F5A
:107DC000000130EC2EF089EC30F0740EF66E230ECC
:107DD000F76E74EC30F0952D0BD0ED2B0A0E0101EF
:107DE000CE6F000105EC2EF0EDC091F196EC30F075
:107DF000955104080BE1ED070A0E0101CE6F000159
:107E000005EC2EF0EDC091F196EC30F0955105089F
:107E100006E1010116971699169B169D000188D759
:107E2000020E0101916FFA0ECE6F000105EC2EF0EB
:107E30000101912FF8D700010DEF43F050EC34F021
:107E4000F96BFA6B6F0048FF92F1D29E3901E16B3A
:107E50003D0EE06FE59DE59FE581E351E59DE58FF2
:107E6000010192BFD28E0001E26FF053D8A423D15A
:107E70009551030850E068EC30F0F20EF66E230ED8
:107E8000F76E74EC30F089EC30F0040EF66E240ED0
:107E9000F76E74EC30F0952D1ED068EC30F0160EB5
:107EA000F66E240EF76E74EC30F089EC30F0280E8C
:107EB000F66E240EF76E74EC30F001019181080E1D
:107EC000926FFA0ECE6F000105EC2EF00101922F99
:107ED000F8D7000120D0955104081CE168EC30F07F
:107EE0003A0EF66E240EF76E74EC30F089EC30F03A
:107EF0004C0EF66E240EF76E74EC30F0080E010195
:107F0000926FFA0ECE6F000105EC2EF00101922F58
:107F1000F8D70001ADD76F0048FF92F1D29E39012A
:107F2000E16B3D0EE06FE59DE59FE581E351E59D49
:107F3000E58F010192BFD28E0001E26F010191A194
:107F4000B8D00001E2515A0801E2E26B68EC30F06F
:107F50005C0EF66E240EF76E090E0101956F00019E
:107F6000A0EC34F0E2C092F1130E0101936F000116
:107F7000D0EC34F0680EF66E240EF76E040E01019C
:107F8000956F0001A0EC34F089EC30F06E0EF66EC7
:107F9000240EF76E74EC30F0640E0101CE6F000118
:107FA00005EC2EF09551040801E1E22B640E01016D
:107FB000CE6F000105EC2EF0952D01D0E207955112
:107FC000030875E1D250006ED29E3901E16B3D0E7F
:107FD000E06F60008BF3E3F9E59DE59FE585550EC5
:107FE000E66FAA0EE66FE583E5B3FED7E595E59D5E
:107FF000E58F0050D2120400840E006E002EFED7D2
:1080000000D06F0048FF92F1D29EE16B3D0EE06F11
:10801000E59DE59FE581E351E59DE58F010192BF77
:10802000D28E0001E26F68EC30F0800EF66E240E06
:10803000F76E090E0101956F0001A0EC34F0E2C06B
:1080400092F1130E0101936F0001D0EC34F08C0E0D
:10805000F66E240EF76E040E0101956F0001A0EC80
:1080600034F089EC30F0920EF66E240EF76E74EC5C
:1080700030F00101936BE2C092F1020E956F580E41
:10808000946F00019FEC2EF0E66BE56B02C0E4F00C
:1080900001C0E3F0080E0101926FFA0ECE6F0001ED
:1080A00005EC2EF00101922FF8D79191000146D7EF
:1080B00001011CD0000168EC30F0A40EF66E240E15
:1080C000F76E74EC30F089EC30F0B60EF66E240EDC
:1080D000F76E74EC30F0080E0101926FFA0ECE6F5D
:1080E000000105EC2EF00101922FF8D7000114EFEA
:1080F00043F050EC34F0F96BFA6B95510308D8B4A7
:10810000A7D0F53D94D068EC30F0C80EF66E240E82
:10811000F76E74EC30F089EC30F0DA0EF66E240E67
:10812000F76E74EC30F0952D48D068EC30F0EC0E22
:10813000F66E240EF76E74EC30F089EC30F0FE0E23
:10814000F66E240EF76E74EC30F0F06BD250006EC9
:10815000D29E3901E16B2D0EE06F6000C3F3E3F9AD
:10816000E59DE59FE585550EE66FAA0EE66FE58372
:10817000E5B3FED7E595E59DE58F0050D2126F007F
:1081800048FF91F1D29EE16B2D0EE06FE59DE59FDA
:10819000E581E351E59DE58F010191BFD28E00019C
:1081A000F06F080E0101916FFA0ECE6F000105EC21
:1081B0002EF00101912FF8D700019551040836E106
:1081C00068EC30F0100EF66E250EF76E74EC30F0A1
:1081D00089EC30F0220EF66E250EF76E74EC30F05E
:1081E000F069D250006ED29E3901E16B2D0EE06F26
:1081F0006000C3F3E3F9E59DE59FE585550EE66F65
:10820000AA0EE66FE583E5B3FED7E595E59DE58F1C
:108210000050D212080E0101916FFA0ECE6F0001CC
:1082200005EC2EF00101912FF8D7000110D068EC79
:1082300030F0340EF66E250EF76E74EC30F089ECEB
:1082400030F0460EF66E250EF76E74EC30F055D712
:108250001AEF43F050EC34F0F96BFA6B95510308C8
:10826000D8B482D068EC30F0860EF66E230EF76E2E
:1082700074EC30F089EC30F0980EF66E230EF76E49
:1082800074EC30F0952D36D068EC30F0AA0EF66E16
:10829000230EF76E74EC30F089EC30F0BC0EF66E05
:1082A000230EF76E74EC30F0F56BD250006ED29E58
:1082B0003901E16B300EE06F6000D7F3E3F9E59D23
:1082C000E59FE585550EE66FAA0EE66FE583E5B3FB
:1082D000FED7E595E59DE58F0050D212080E01010D
:1082E000916FFA0ECE6F000105EC2EF00101912F77
:1082F000F8D700019551040836E168EC30F0CE0E55
:10830000F66E230EF76E74EC30F089EC30F0E00E70
:10831000F66E230EF76E74EC30F0F569D250006EF5
:10832000D29E3901E16B300EE06F6000D7F3E3F9C4
:10833000E59DE59FE585550EE66FAA0EE66FE583A0
:10834000E5B3FED7E595E59DE58F0050D212080E06
:108350000101916FFA0ECE6F000105EC2EF00101C4
:10836000912FF8D700017AD720EF43F050EC34F08A
:10837000F96BFA6B95510308D8B4BBD0F9510908D1
:1083800001E2F96BFA51090801E2FA6B68EC30F08E
:10839000E00EF66E3C0EF76E74EC30F089EC30F0C7
:1083A000F20EF66E3C0EF76E080E0101956F00019D
:1083B000A0EC34F0F9C092F1180E0101936F0001A6
:1083C000D0EC34F0FD0EF66E3C0EF76E050E01019A
:1083D000956F0001A0EC34F0FAC092F1180E010183
:1083E000936F0001D0EC34F0200E0101A16F000169
:1083F00030EC2EF0955104083DE1FA2B955104081C
:1084000039E1FA51090801E2FA6B68EC30F0080E24
:10841000F66E3D0EF76E74EC30F089EC30F01A0E0B
:10842000F66E3D0EF76E080E0101956F0001A0EC8F
:1084300034F0F9C092F1180E0101936F0001D0ECF5
:1084400034F0250EF66E3D0EF76E050E0101956FA8
:108450000001A0EC34F0FAC092F1180E0101936F04
:108460000001D0EC34F0200E0101A16F000130ECCE
:108470002EF0C4D7952D3CD0F92B952D39D0F9513C
:10848000090801E2F96B68EC30F0300EF66E3D0E33
:10849000F76E74EC30F089EC30F0420EF66E3D0E63
:1084A000F76E080E0101956F0001A0EC34F0F9C0E1
:1084B00092F1180E0101936F0001D0EC34F04D0ED3
:1084C000F66E3D0EF76E050E0101956F0001A0ECF2
:1084D00034F0FAC092F1180E0101936F0001D0EC54
:1084E00034F0200E0101A16F000130EC2EF0C5D751
:1084F00041D7F951040802E1FA5348E0F95105085F
:1085000002E1FA5343E0F951060802E1FA533EE072
:10851000F951060803E1FA51060838E0F951070855
:1085200002E1FA5333E0F951070803E1FA51050873
:108530002DE0F951080802E1FA5328E0F951090841
:1085400002E1FA5323E0F951090803E1FA2D01D0C1
:108550001DD0F951030802E1FA5318E0F95102085D
:1085600002E1FA5313E0F951020803E1FA2D01D0B8
:108570000DD0F951050803E1FA2D01D007D0F951CA
:108580000808D8A45ED0FA5109085BE1F951020845
:1085900004E1FA53D8B411EF35F0F951020804E1BF
:1085A000FA2D02D03FEF36F0F951030804E1FA53F7
:1085B000D8B4CAEF36F0F951040804E1FA53D8B43C
:1085C000E2EF37F0F951050804E1FA53D8B46DEF42
:1085D00038F0F951050804E1FA2D02D0F9EF38F02E
:1085E000F951060804E1FA53D8B487EF3AF0F9518B
:1085F000070804E1FA53D8B49DEF3BF0F95107089E
:1086000005E1FA510508D8B4BFEF3CF0F95108086C
:1086100004E1FA53D8B484EF3EF0F951080804E1BC
:10862000FA510908D8B40AD4F951090803E1FA53F8
:10863000D8B45FD5F951090803E1FA2D01D00AD663
:108640001DD068EC30F0580EF66E3D0EF76E74ECEF
:1086500030F089EC30F06A0EF66E3D0EF76E74EC79
:1086600030F0020E0101916FFA0ECE6F000105ECA1
:108670002EF00101912FF8D7FF0000017BD6E9EF22
:1086800044F00A0E0101CE6F000105EC2EF0D93D39
:1086900010D089EC30F0F80EF66E280EF76E74EC00
:1086A00030F068EC30F00A0EF66E290EF76E74ECBE
:1086B00030F0D95310E189EC30F01C0EF66E290E23
:1086C000F76E74EC30F068EC30F02E0EF66E290E7A
:1086D000F76E74EC30F0D9517F0810E189EC30F07E
:1086E000400EF66E290EF76E74EC30F068EC30F048
:1086F000520EF66E290EF76E74EC30F01200CBECD1
:1087000032F0140E0101CE6F000105EC2EF0B4EC36
:1087100033F0010EA86F50EC34F0F96BFA6BA851EE
:10872000010A35E0030AD8B49DD1010AD8B483EF19
:1087300047F0070AD8B472EF49F0010AD8B463EFE2
:108740004BF0030AD8B44FEF4DF0010AD8B4B4EFA0
:108750004FF00F0AD8B40FEF52F0010AD8B459EF16
:1087600054F0030AD8B44FEF55F0010AD8B46DEFB6
:1087700057F0070AD8B480EF59F0010AD8B494EF43
:108780005AF0030AD8B435EF5CF0DEEF5CF050EC41
:1087900034F095510308D8B400D1F951090801E229
:1087A000F96BFA51090801E2FA6BD93D08D068EC7F
:1087B00030F0F40EF66E290EF76E74EC30F0D953EB
:1087C00008E168EC30F0060EF66E2A0EF76E74ECD7
:1087D00030F0D9517F0808E168EC30F0180EF66EE1
:1087E0002A0EF76E74EC30F089EC30F02A0EF66E3B
:1087F0002A0EF76E080E0101956F0001A0EC34F00F
:10880000F9C092F1180E0101936F0001D0EC34F021
:10881000350EF66E2A0EF76E050E0101956F0001FA
:10882000A0EC34F0FAC092F1180E0101936F000130
:10883000D0EC34F0200E0101A16F000130EC2EF0DD
:108840009551040854E1FA2B9551040850E1FA516E
:10885000090801E2FA6BD93D08D068EC30F0400E0F
:10886000F66E2A0EF76E74EC30F0D95308E168EC1E
:1088700030F0520EF66E2A0EF76E74EC30F0D951CD
:108880007F0808E168EC30F0640EF66E2A0EF76E91
:1088900074EC30F089EC30F0760EF66E2A0EF76E3E
:1088A000080E0101956F0001A0EC34F0F9C092F1BF
:1088B000180E0101936F0001D0EC34F0810EF66EBA
:1088C0002A0EF76E050E0101956F0001A0EC34F041
:1088D000FAC092F1180E0101936F0001D0EC34F050
:1088E000200E0101A16F000130EC2EF0ADD7952DC7
:1088F00053D0F92B952D50D0F951090801E2F96BAD
:10890000D93D08D068EC30F08C0EF66E2A0EF76E6A
:1089100074EC30F0D95308E168EC30F09E0EF66E3E
:108920002A0EF76E74EC30F0D9517F0808E168EC3C
:1089300030F0B00EF66E2A0EF76E74EC30F089EC63
:1089400030F0C20EF66E2A0EF76E080E0101956F1A
:108950000001A0EC34F0F9C092F1180E0101936F00
:108960000001D0EC34F0CD0EF66E2A0EF76E050E37
:108970000101956F0001A0EC34F0FAC092F1180EDD
:108980000101936F0001D0EC34F0200E0101A16FC2
:10899000000130EC2EF0AED7FCD6640E0101CE6F94
:1089A000000105EC2EF0F951090803E1FA5109081C
:1089B0000AE0F92D03D0FA51030805E0F9530BE161
:1089C000FA51040808E1F95304E1FA510408D8B453
:1089D000CDD4A82B45D0D93D10D068EC30F0D80EBE
:1089E000F66E2A0EF76E74EC30F089EC30F0EA0E79
:1089F000F66E2A0EF76E74EC30F0D95310E168EC85
:108A000030F0FC0EF66E2A0EF76E74EC30F089EC46
:108A100030F00E0EF66E2B0EF76E74EC30F0D9516E
:108A20007F0810E168EC30F0200EF66E2B0EF76E2A
:108A300074EC30F089EC30F0320EF66E2B0EF76EDF
:108A400074EC30F0020E0101916FFA0ECE6F00014E
:108A500005EC2EF00101912FF8D7E6EF5CF0000154
:108A6000DEEF5CF0F92D06D0FA51030803E1A82BE4
:108A7000DEEF5CF050EC34F0D93D09D068EC30F01A
:108A8000440EF66E2B0EF76E74EC30F016D0D95300
:108A900009E168EC30F0560EF66E2B0EF76E74ECB2
:108AA00030F00BD0D9517F0808E168EC30F0680E47
:108AB000F66E2B0EF76E74EC30F0D93D29D089ECB0
:108AC00030F07A0EF66E2B0EF76E080E0101956FE0
:108AD0000001A0EC34F07F0E0101A16F000130EC29
:108AE0002EF0840EF66E2B0EF76E050E0101956FBB
:108AF0000001A0EC34F07E0E0101A16F000130EC0A
:108B00002EF0200E0101A16F000130EC2EF056D0A6
:108B1000D95329E189EC30F08E0EF66E2B0EF76EEC
:108B2000080E0101956F0001A0EC34F07F0E0101E9
:108B3000A16F000130EC2EF0980EF66E2B0EF76E42
:108B4000050E0101956F0001A0EC34F07E0E0101CD
:108B5000A16F000130EC2EF0200E0101A16F000189
:108B600030EC2EF02BD0D9517F0828E189EC30F081
:108B7000A20EF66E2B0EF76E080E0101956F000126
:108B8000A0EC34F07F0E0101A16F000130EC2EF05B
:108B9000AC0EF66E2B0EF76E050E0101956F0001FF
:108BA000A0EC34F07E0E0101A16F000130EC2EF03C
:108BB000200E0101A16F000130EC2EF09551040848
:108BC00001E1A82B952D01D0A807A85302E1010EC1
:108BD000A86F95510308D8A494D1D93D09D068EC69
:108BE00030F0B60EF66E2B0EF76E74EC30F016D039
:108BF000D95309E168EC30F0C80EF66E2B0EF76E13
:108C000074EC30F00BD0D9517F0808E168EC30F0FB
:108C1000DA0EF66E2B0EF76E74EC30F0D93D29D0DB
:108C200089EC30F0EC0EF66E2B0EF76E080E01019B
:108C3000956F0001A0EC34F07F0E0101A16F0001DF
:108C400030EC2EF0F60EF66E2B0EF76E050E0101CF
:108C5000956F0001A0EC34F07E0E0101A16F0001C0
:108C600030EC2EF0200E0101A16F000130EC2EF04F
:108C700056D0D95329E189EC30F0000EF66E2C0E57
:108C8000F76E080E0101956F0001A0EC34F07F0E25
:108C90000101A16F000130EC2EF00A0EF66E2C0ED1
:108CA000F76E050E0101956F0001A0EC34F07E0E09
:108CB0000101A16F000130EC2EF0200E0101A16F27
:108CC000000130EC2EF02BD0D9517F0828E189EC3F
:108CD00030F0140EF66E2C0EF76E080E0101956F33
:108CE0000001A0EC34F07F0E0101A16F000130EC17
:108CF0002EF01E0EF66E2C0EF76E050E0101956F0E
:108D00000001A0EC34F07E0E0101A16F000130ECF7
:108D10002EF0200E0101A16F000130EC2EF050EC7E
:108D200034F095510308D8B4BDD0D9517F0809E17A
:108D300068EC30F0280EF66E2C0EF76E74EC30F006
:108D400008D068EC30F03A0EF66E2C0EF76E74EC2C
:108D500030F0D93D08D089EC30F04C0EF66E2C0E78
:108D6000F76E74EC30F0D95308E189EC30F05E0E08
:108D7000F66E2C0EF76E74EC30F0D9517F0808E1D6
:108D800089EC30F0700EF66E2C0EF76E74EC30F04D
:108D900095510308D8B4B2D0952D40D050EC34F0A2
:108DA000955105083BE1D93D11D068EC30F0820EB9
:108DB000F66E2C0EF76E74EC30F089EC30F0940EF9
:108DC000F66E2C0EF76E74EC30F026D0D95311E10C
:108DD00068EC30F0A60EF66E2C0EF76E74EC30F0E8
:108DE00089EC30F0B80EF66E2C0EF76E74EC30F0A5
:108DF00013D0D9517F0810E168EC30F0CA0EF66E3E
:108E00002C0EF76E74EC30F089EC30F0DC0EF66E60
:108E10002C0EF76E74EC30F08889C2D79551040897
:108E200040E150EC34F0955105083BE1D93D11D0BB
:108E300068EC30F0EE0EF66E2C0EF76E74EC30F03F
:108E400089EC30F0000EF66E2D0EF76E74EC30F0FB
:108E500026D0D95311E168EC30F0120EF66E2D0ECB
:108E6000F76E74EC30F089EC30F0240EF66E2D0EB7
:108E7000F76E74EC30F013D0D9517F0810E168EC34
:108E800030F0360EF66E2D0EF76E74EC30F089EC85
:108E900030F0480EF66E2D0EF76E74EC30F08899B7
:108EA000C2D73FD741EC43F0952D21D0000E88B9B1
:108EB000010E0101916FD250006ED29E3901E16B1B
:108EC000140EE06F600047F6E3F9E59DE59FE58548
:108ED000550EE66FAA0EE66FE583E5B3FED7E5957E
:108EE000E59DE58F0050D2120AD006D000019551C1
:108EF000040803E1390103D00001D4D7390100018E
:108F0000A82BDEEF5CF0F92D06D0FA51030803E13F
:108F1000A82BDEEF5CF050EC34F0D93D31D068EC9A
:108F200030F05A0EF66E2D0EF76E74EC30F089ECC0
:108F300030F06C0EF66E2D0EF76E080E0101956F77
:108F40000001A0EC34F07F0E0101A16F000130ECB4
:108F50002EF0760EF66E2D0EF76E050E0101956F52
:108F60000001A0EC34F07E0E0101A16F000130EC95
:108F70002EF0200E0101A16F000130EC2EF066D022
:108F8000D95331E168EC30F0800EF66E2D0EF76E9D
:108F900074EC30F089EC30F0920EF66E2D0EF76E18
:108FA000080E0101956F0001A0EC34F07F0E010165
:108FB000A16F000130EC2EF09C0EF66E2D0EF76EB8
:108FC000050E0101956F0001A0EC34F07E0E010149
:108FD000A16F000130EC2EF0200E0101A16F000105
:108FE00030EC2EF033D0D9517F0830E168EC30F00E
:108FF000A60EF66E2D0EF76E74EC30F089EC30F0A4
:10900000B80EF66E2D0EF76E080E0101956F000179
:10901000A0EC34F07F0E0101A16F000130EC2EF0C6
:10902000C20EF66E2D0EF76E050E0101956F000152
:10903000A0EC34F07E0E0101A16F000130EC2EF0A7
:10904000200E0101A16F000130EC2EF095510408B3
:1090500001E1A82B952D01D0A807A85302E1010E2C
:10906000A86F95510308D8A43BD150EC34F0699D0A
:1090700095510308D8B4E6D0878F69BD5ED0D93D3D
:109080001DD068EC30F0CC0EF66E2D0EF76E0A0E89
:109090000101956F0001A0EC34F0000EE96EB7C03D
:1090A00092F1B6C091F185EC39F089EC30F0DC0E2C
:1090B000F66E2D0EF76E74EC30F03ED0D9531DE1F4
:1090C00068EC30F0EE0EF66E2D0EF76E0A0E010112
:1090D000956F0001A0EC34F0000EE96EB7C092F17C
:1090E000B6C091F185EC39F089EC30F0FE0EF66EE9
:1090F0002D0EF76E74EC30F01FD0D9517F081CE1B3
:1091000068EC30F0100EF66E2E0EF76E0A0E0101AE
:10911000956F0001A0EC34F0000EE96EB7C092F13B
:10912000B6C091F185EC39F089EC30F0200EF66E86
:109130002E0EF76E74EC30F05DD0D93D1DD068EC8A
:1091400030F0320EF66E2E0EF76E0A0E0101956F9C
:109150000001A0EC34F0000EE96EC3C092F1C2C071
:1091600091F185EC39F089EC30F0420EF66E2E0E5E
:10917000F76E74EC30F03ED0D9531DE168EC30F05E
:10918000540EF66E2E0EF76E0A0E0101956F000159
:10919000A0EC34F0000EE96EC3C092F1C2C091F1B0
:1091A00085EC39F089EC30F0640EF66E2E0EF76E19
:1091B00074EC30F01FD0D9517F081CE168EC30F01E
:1091C000760EF66E2E0EF76E0A0E0101956F0001F7
:1091D000A0EC34F0000EE96EC3C092F1C2C091F170
:1091E00085EC39F089EC30F0860EF66E2E0EF76EB7
:1091F00074EC30F0952D06D001011689168B169D62
:109200000001698D9551040806E101011687168B4E
:10921000169D0001698D9551050813E1010116970E
:109220001699169B169D0001AD6BAC6BAB6BAA6BD0
:10923000B16BB06BAF6B030EAE6FB56BB46BB36B52
:10924000B26B16D7640E0101CE6F000105EC2EF053
:1092500069AD43D041EC43F0952D38D0C3C0B7F091
:10926000C2C0B6F06000DBF2E3F9D250006ED29ECD
:109270003901E16B060EE06FE59DE59FE585550E32
:10928000E66FAA0EE66FE583E5B3FED7E595E59DAB
:10929000E58F0050D2126000DFF2E3F9D250006E89
:1092A000D29EE16B070EE06FE59DE59FE585550ECB
:1092B000E66FAA0EE66FE583E5B3FED7E595E59D7B
:1092C000E58F0050D2120AD006D000019551040853
:1092D00003E1390103D00001BDD739010001A82BFA
:1092E000DEEF5CF0F92D03D0FA51030802E0EF3D08
:1092F00003D0A82BDEEF5CF050EC34F0D93D31D038
:1093000068EC30F0980EF66E2E0EF76E74EC30F0BE
:1093100089EC30F0AA0EF66E2E0EF76E080E0101E3
:10932000956F0001A0EC34F07F0E0101A16F0001E8
:1093300030EC2EF0B40EF66E2E0EF76E050E010117
:10934000956F0001A0EC34F07E0E0101A16F0001C9
:1093500030EC2EF0200E0101A16F000130EC2EF058
:1093600066D0D95331E168EC30F0BE0EF66E2E0EA9
:10937000F76E74EC30F089EC30F0D00EF66E2E0EF5
:10938000F76E080E0101956F0001A0EC34F07F0E1E
:109390000101A16F000130EC2EF0DA0EF66E2E0EF8
:1093A000F76E050E0101956F0001A0EC34F07E0E02
:1093B0000101A16F000130EC2EF0200E0101A16F20
:1093C000000130EC2EF033D0D9517F0830E168EC49
:1093D00030F0E40EF66E2E0EF76E74EC30F089EC81
:1093E00030F0F60EF66E2E0EF76E080E0101956F38
:1093F0000001A0EC34F07F0E0101A16F000130EC00
:109400002EF0000EF66E2F0EF76E050E0101956F11
:109410000001A0EC34F07E0E0101A16F000130ECE0
:109420002EF0200E0101A16F000130EC2EF09551BD
:10943000040801E1A82B952D01D0A807A85302E14B
:10944000010EA86F95510308D8A43BD150EC34F01D
:10945000699D95510308D8B4E6D0878F69BD5ED069
:10946000D93D1DD068EC30F00A0EF66E2F0EF76E67
:109470000A0E0101956F0001A0EC34F0000EE96EB8
:10948000B9C092F1B8C091F185EC39F089EC30F0B7
:109490001A0EF66E2F0EF76E74EC30F03ED0D953E4
:1094A0001DE168EC30F02C0EF66E2F0EF76E0A0EF2
:1094B0000101956F0001A0EC34F0000EE96EB9C017
:1094C00092F1B8C091F185EC39F089EC30F03C0EA6
:1094D000F66E2F0EF76E74EC30F01FD0D9517F0866
:1094E0001CE168EC30F04E0EF66E2F0EF76E0A0E91
:1094F0000101956F0001A0EC34F0000EE96EB9C0D7
:1095000092F1B8C091F185EC39F089EC30F05E0E43
:10951000F66E2F0EF76E74EC30F05DD0D93D1DD095
:1095200068EC30F0700EF66E2F0EF76E0A0E010129
:10953000956F0001A0EC34F0000EE96EC3C092F10B
:10954000C2C091F185EC39F089EC30F0800EF66EF6
:109550002F0EF76E74EC30F03ED0D9531DE168EC5D
:1095600030F0920EF66E2F0EF76E0A0E0101956F17
:109570000001A0EC34F0000EE96EC3C092F1C2C04D
:1095800091F185EC39F089EC30F0A20EF66E2F0ED9
:10959000F76E74EC30F01FD0D9517F081CE168ECF5
:1095A00030F0B40EF66E2F0EF76E0A0E0101956FB5
:1095B0000001A0EC34F0000EE96EC3C092F1C2C00D
:1095C00091F185EC39F089EC30F0C40EF66E2F0E77
:1095D000F76E74EC30F0952D06D001011689168BCC
:1095E000169D0001698D9551040806E10101168759
:1095F000168B169D0001698D9551050813E1010137
:1096000016971699169B169D0001AD6BAC6BAB6B54
:10961000AA6BB16BB06BAF6B030EAE6FB56BB46B77
:10962000B36BB26B16D7640E0101CE6F000105EC6F
:109630002EF069AD43D041EC43F0952D38D0C3C036
:10964000B9F0C2C0B8F06000E3F2E3F9D250006EA6
:10965000D29E3901E16B280EE06FE59DE59FE5851F
:10966000550EE66FAA0EE66FE583E5B3FED7E595E6
:10967000E59DE58F0050D2126000E7F2E3F9D25089
:10968000006ED29EE16B290EE06FE59DE59FE585BA
:10969000550EE66FAA0EE66FE583E5B3FED7E595B6
:1096A000E59DE58F0050D2120AD006D000019551F9
:1096B000040803E1390103D00001BDD739010001DD
:1096C000A82BDEEF5CF0F92D06D0FA51030803E178
:1096D000A82BDEEF5CF050EC34F0D93D31D068ECD3
:1096E00030F0D60EF66E2F0EF76E74EC30F089EC7B
:1096F00030F0E80EF66E2F0EF76E080E0101956F32
:109700000001A0EC34F07F0E0101A16F000130ECEC
:109710002EF0F20EF66E2F0EF76E050E0101956F0C
:109720000001A0EC34F07E0E0101A16F000130ECCD
:109730002EF0200E0101A16F000130EC2EF066D05A
:10974000D95331E168EC30F0FC0EF66E2F0EF76E57
:1097500074EC30F089EC30F00E0EF66E300EF76ED1
:10976000080E0101956F0001A0EC34F07F0E01019D
:10977000A16F000130EC2EF0180EF66E300EF76E71
:10978000050E0101956F0001A0EC34F07E0E010181
:10979000A16F000130EC2EF0200E0101A16F00013D
:1097A00030EC2EF033D0D9517F0830E168EC30F046
:1097B000220EF66E300EF76E74EC30F089EC30F05D
:1097C000340EF66E300EF76E080E0101956F000133
:1097D000A0EC34F07F0E0101A16F000130EC2EF0FF
:1097E0003E0EF66E300EF76E050E0101956F00010C
:1097F000A0EC34F07E0E0101A16F000130EC2EF0E0
:10980000200E0101A16F000130EC2EF095510408EB
:1098100001E1A82B952D09D0A807F92D03D0FA5105
:10982000030802E0EF3D01D0A807A85302E1010EB2
:10983000A86F95510308D8A430D150EC34F0699F3B
:1098400095510308D8B4DBD0878F69BF5ED0D93D6E
:109850001DD068EC30F0480EF66E300EF76E0A0E32
:109860000101956F0001A0EC34F0000EE96EBBC061
:1098700092F1BAC091F185EC39F089EC30F0580ED4
:10988000F66E300EF76E74EC30F03ED0D9531DE119
:1098900068EC30F06A0EF66E300EF76E0A0E0101BB
:1098A000956F0001A0EC34F0000EE96EBBC092F1A0
:1098B000BAC091F185EC39F089EC30F07A0EF66E91
:1098C000300EF76E74EC30F01FD0D9517F081CE1D8
:1098D00068EC30F08C0EF66E300EF76E0A0E010159
:1098E000956F0001A0EC34F0000EE96EBBC092F160
:1098F000BAC091F185EC39F089EC30F09C0EF66E2F
:10990000300EF76E74EC30F05DD0D93D1DD068ECB0
:1099100030F0AE0EF66E300EF76E0A0E0101956F46
:109920000001A0EC34F0000EE96EC3C092F1C2C099
:1099300091F185EC39F089EC30F0BE0EF66E300E08
:10994000F76E74EC30F03ED0D9531DE168EC30F086
:10995000D00EF66E300EF76E0A0E0101956F000103
:10996000A0EC34F0000EE96EC3C092F1C2C091F1D8
:1099700085EC39F089EC30F0E00EF66E300EF76EC3
:1099800074EC30F01FD0D9517F081CE168EC30F046
:10999000F20EF66E300EF76E0A0E0101956F0001A1
:1099A000A0EC34F0000EE96EC3C092F1C2C091F198
:1099B00085EC39F089EC30F0020EF66E310EF76E60
:1099C00074EC30F0952D07D001011689168B168D99
:1099D0000001698F13D09551040807E10101168732
:1099E000168B169D0001698F09D09551050806E177
:1099F000010116971699169B169D000121D7640E3A
:109A00000101CE6F000105EC2EF069AF43D041ECAF
:109A100043F0952D38D0C3C0BBF0C2C0BAF060008F
:109A2000EBF2E3F9D250006ED29E3901E16B080EE1
:109A3000E06FE59DE59FE585550EE66FAA0EE66FA2
:109A4000E583E5B3FED7E595E59DE58F0050D2129D
:109A50006000EFF2E3F9D250006ED29EE16B090E86
:109A6000E06FE59DE59FE585550EE66FAA0EE66F72
:109A7000E583E5B3FED7E595E59DE58F0050D2126D
:109A80000AD006D000019551040803E1390103D042
:109A90000001BDD739010001A82BDEEF5CF0F92DE4
:109AA00006D0FA51030803E1A82BDEEF5CF050EC7E
:109AB00034F0D93D31D068EC30F0140EF66E310E32
:109AC000F76E74EC30F089EC30F0260EF66E310E45
:109AD000F76E080E0101956F0001A0EC34F07F0EC7
:109AE0000101A16F000130EC2EF0300EF66E310E48
:109AF000F76E050E0101956F0001A0EC34F07E0EAB
:109B00000101A16F000130EC2EF0200E0101A16FC8
:109B1000000130EC2EF066D0D95331E168EC30F022
:109B20003A0EF66E310EF76E74EC30F089EC30F0D0
:109B30004C0EF66E310EF76E080E0101956F0001A6
:109B4000A0EC34F07F0E0101A16F000130EC2EF08B
:109B5000560EF66E310EF76E050E0101956F00017F
:109B6000A0EC34F07E0E0101A16F000130EC2EF06C
:109B7000200E0101A16F000130EC2EF033D0D9513D
:109B80007F0830E168EC30F0600EF66E310EF76E53
:109B900074EC30F089EC30F0720EF66E310EF76E28
:109BA000080E0101956F0001A0EC34F07F0E010159
:109BB000A16F000130EC2EF07C0EF66E310EF76EC8
:109BC000050E0101956F0001A0EC34F07E0E01013D
:109BD000A16F000130EC2EF0200E0101A16F0001F9
:109BE00030EC2EF09551040801E1A82B952D01D001
:109BF000A8076F0048FF91F1D29E3901E16B0B0E6F
:109C0000E06FE59DE59FE581E351E59DE58F01016D
:109C100091BFD28E0001F86F95510308D8A4A2D14C
:109C200050EC34F0879195510308D8B462D187B1D4
:109C3000B2D0D93D2DD068EC30F0860EF66E310EE4
:109C4000F76E0A0E0101956F0001A0EC34F0020ED0
:109C50000101916F200EA16F000130EC2EF0010187
:109C6000912FF8D7F8C092F1130E936F0001D0EC4A
:109C700034F0250E0101A16F000130EC2EF089ECCB
:109C800030F0960EF66E310EF76E74EC30F05ED05A
:109C9000D9532DE168EC30F0A80EF66E310EF76E58
:109CA0000A0E0101956F0001A0EC34F0020E0101D3
:109CB000916F200EA16F000130EC2EF00101912F69
:109CC000F8D7F8C092F1130E936F0001D0EC34F086
:109CD000250E0101A16F000130EC2EF089EC30F06F
:109CE000B80EF66E310EF76E74EC30F02FD0D951FD
:109CF0007F082CE168EC30F0CA0EF66E310EF76E7C
:109D00000A0E0101956F0001A0EC34F0020E010172
:109D1000916F200EA16F000130EC2EF00101912F08
:109D2000F8D7F8C092F1130E936F0001D0EC34F025
:109D3000250E0101A16F000130EC2EF089EC30F00E
:109D4000DA0EF66E310EF76E74EC30F00101926BA4
:109D5000F8C091F100011AEC30F002C0DDF001C052
:109D6000DCF0010E0101CE6F000105EC2EF09551E3
:109D7000040802E1F82B8781010E0101CE6F00017A
:109D800005EC2EF0952D02D0F8078781F851630875
:109D900001E2F86BADD0D93D2CD068EC30F0EC0E80
:109DA000F66E310EF76E0A0E0101956F0001A0EC00
:109DB00034F0020E0101916F200EA16F000130EC12
:109DC0002EF00101912FF8D7F8C092F1130E936F86
:109DD0000001D0EC34F0250E0101A16F000130EC40
:109DE0002EF089EC30F0FC0EF66E310EF76E74EC4E
:109DF00030F0D9532CE168EC30F00E0EF66E320ED6
:109E0000F76E0A0E0101956F0001A0EC34F0020E0E
:109E10000101916F200EA16F000130EC2EF00101C5
:109E2000912FF8D7F8C092F1130E936F0001D0EC88
:109E300034F0250E0101A16F000130EC2EF089EC09
:109E400030F01E0EF66E320EF76E74EC30F0D95113
:109E50007F082CE168EC30F0300EF66E320EF76EB3
:109E60000A0E0101956F0001A0EC34F0020E010111
:109E7000916F200EA16F000130EC2EF00101912FA7
:109E8000F8D7F8C092F1130E936F0001D0EC34F0C4
:109E9000250E0101A16F000130EC2EF089EC30F0AD
:109EA000400EF66E320EF76E74EC30F00101926BDC
:109EB000F8C091F100011AEC30F002C0DDF001C0F1
:109EC000DCF0320E0101CE6F000105EC2EF0955151
:109ED000040801E1F82B320E0101CE6F000105EC00
:109EE0002EF0952D01D0F807F851630801E2F86BC8
:109EF0009AD668EC30F0520EF66E320EF76E74ECB5
:109F000030F087A127D041EC43F0952D1CD0D250E2
:109F1000006ED29E3901E16B0B0EE06F6000E3F33F
:109F2000E3F9E59DE59FE585550EE66FAA0EE66F20
:109F3000E583E5B3FED7E595E59DE58F0050D212A8
:109F40000AD006D000019551040803E1390103D07D
:109F50000001D9D73901640E0101CE6F000105EC73
:109F60002EF0A82BDEEF5CF0F92D06D0FA51030895
:109F700003E1A82BDEEF5CF050EC34F0D93D31D09A
:109F800068EC30F0640EF66E320EF76E74EC30F062
:109F900089EC30F0760EF66E320EF76E080E010187
:109FA000956F0001A0EC34F07F0E0101A16F00015C
:109FB00030EC2EF0800EF66E320EF76E050E0101BB
:109FC000956F0001A0EC34F07E0E0101A16F00013D
:109FD00030EC2EF0200E0101A16F000130EC2EF0CC
:109FE00066D0D95331E168EC30F08A0EF66E320E4D
:109FF000F76E74EC30F089EC30F09C0EF66E320E99
:10A00000F76E080E0101956F0001A0EC34F07F0E91
:10A010000101A16F000130EC2EF0A60EF66E320E9B
:10A02000F76E050E0101956F0001A0EC34F07E0E75
:10A030000101A16F000130EC2EF0200E0101A16F93
:10A04000000130EC2EF033D0D9517F0830E168ECBC
:10A0500030F0B00EF66E320EF76E74EC30F089EC24
:10A0600030F0C20EF66E320EF76E080E0101956FDB
:10A070000001A0EC34F07F0E0101A16F000130EC73
:10A080002EF0CC0EF66E320EF76E050E0101956FB6
:10A090000001A0EC34F07E0E0101A16F000130EC54
:10A0A0002EF0200E0101A16F000130EC2EF0955131
:10A0B000040801E1A82B952D01D0A8076F0048FFE7
:10A0C00091F1D29E3901E16B0D0EE06FE59DE59FA8
:10A0D000E581E351E59DE58F010191BFD28E00013D
:10A0E000F76F95510308D8A498D150EC34F08793BA
:10A0F00095510308D8B460D187B3B0D0D93D2CD0E6
:10A1000068EC30F0D60EF66E320EF76E0A0E0101D4
:10A11000956F0001A0EC34F0020E0101916F200E4A
:10A12000A16F000130EC2EF00101912FF8D7F7C09C
:10A1300092F1130E936F0001D0EC34F0250E010163
:10A14000A16F000130EC2EF089EC30F0E60EF66ED7
:10A15000320EF76E74EC30F0D9532CE168EC30F02D
:10A16000F80EF66E320EF76E0A0E0101956F0001C1
:10A17000A0EC34F0020E0101916F200EA16F0001DE
:10A1800030EC2EF00101912FF8D7F7C092F1130EA9
:10A19000936F0001D0EC34F0250E0101A16F000196
:10A1A00030EC2EF089EC30F0080EF66E330EF76EC0
:10A1B00074EC30F0D9517F082CE168EC30F01A0EC5
:10A1C000F66E330EF76E0A0E0101956F0001A0ECDA
:10A1D00034F0020E0101916F200EA16F000130ECEE
:10A1E0002EF00101912FF8D7F7C092F1130E936F63
:10A1F0000001D0EC34F0250E0101A16F000130EC1C
:10A200002EF089EC30F02A0EF66E330EF76E74ECF9
:10A2100030F00101926BF7C091F100011AEC30F0BF
:10A2200002C0DDF001C0DCF0010E0101CE6F0001C3
:10A2300005EC2EF09551040802E1F72B8783010EFF
:10A240000101CE6F000105EC2EF0952D02D0F7072D
:10A250008783F751630801E2F76BADD0D93D2CD06D
:10A2600068EC30F03C0EF66E330EF76E0A0E01010C
:10A27000956F0001A0EC34F0020E0101916F200EE9
:10A28000A16F000130EC2EF00101912FF8D7F7C03B
:10A2900092F1130E936F0001D0EC34F0250E010102
:10A2A000A16F000130EC2EF089EC30F04C0EF66E10
:10A2B000330EF76E74EC30F0D9532CE168EC30F0CB
:10A2C0005E0EF66E330EF76E0A0E0101956F0001F9
:10A2D000A0EC34F0020E0101916F200EA16F00017D
:10A2E00030EC2EF00101912FF8D7F7C092F1130E48
:10A2F000936F0001D0EC34F0250E0101A16F000135
:10A3000030EC2EF089EC30F06E0EF66E330EF76EF8
:10A3100074EC30F0D9517F082CE168EC30F0800EFD
:10A32000F66E330EF76E0A0E0101956F0001A0EC78
:10A3300034F0020E0101916F200EA16F000130EC8C
:10A340002EF00101912FF8D7F7C092F1130E936F01
:10A350000001D0EC34F0250E0101A16F000130ECBA
:10A360002EF089EC30F0900EF66E330EF76E74EC32
:10A3700030F00101926BF7C091F100011AEC30F05E
:10A3800002C0DBF001C0DAF0320E0101CE6F000135
:10A3900005EC2EF09551040801E1F72B320E010176
:10A3A000CE6F000105EC2EF0952D01D0F707F75187
:10A3B000630801E2F76B9CD687A327D041EC43F0FA
:10A3C000952D1CD0D250006ED29E3901E16B0D0E3E
:10A3D000E06F6000DFF3E3F9E59DE59FE585550E4D
:10A3E000E66FAA0EE66FE583E5B3FED7E595E59D3A
:10A3F000E58F0050D2120AD006D000019551040812
:10A4000003E1390103D00001D9D73901640E0101FC
:10A41000CE6F000105EC2EF0A82BDEEF5CF069B9E1
:10A4200003D0A82BDEEF5CF050EC34F0D93D09D01E
:10A4300068EC30F0A20EF66E330EF76E74EC30F06E
:10A4400016D0D95309E168EC30F0B40EF66E330E35
:10A45000F76E74EC30F00BD0D9517F0808E168EC4E
:10A4600030F0C60EF66E330EF76E74EC30F0D93D58
:10A4700029D089EC30F0D80EF66E330EF76E080E48
:10A480000101956F0001A0EC34F07F0E0101A16F76
:10A49000000130EC2EF0E20EF66E330EF76E050E74
:10A4A0000101956F0001A0EC34F07E0E0101A16F57
:10A4B000000130EC2EF0200E0101A16F000130EC04
:10A4C0002EF056D0D95329E189EC30F0EC0EF66E1F
:10A4D000330EF76E080E0101956F0001A0EC34F009
:10A4E0007F0E0101A16F000130EC2EF0F60EF66E2A
:10A4F000330EF76E050E0101956F0001A0EC34F0EC
:10A500007E0E0101A16F000130EC2EF0200E010142
:10A51000A16F000130EC2EF02BD0D9517F0828E13B
:10A5200089EC30F0000EF66E340EF76E080E010165
:10A53000956F0001A0EC34F07F0E0101A16F0001C6
:10A5400030EC2EF00A0EF66E340EF76E050E010199
:10A55000956F0001A0EC34F07E0E0101A16F0001A7
:10A5600030EC2EF0200E0101A16F000130EC2EF036
:10A570009551040801E1A82B952D01D0A80795510C
:10A580000308D8A494D150EC34F087979551030870
:10A59000D8B45CD1EDC0EEF0ED51FF0AEE6F0101D1
:10A5A000946BEEC093F10001B2EC2EF003C0A1F168
:10A5B00002C0A0F101C09FF100C09EF1550E010143
:10A5C000A56FC10EA46F480EA36F7D0EA26F000190
:10A5D0007DEC2FF003C0ECF002C0EBF001C0EAF01C
:10A5E00000C0E9F087B785D0D93D2AD068EC30F0BB
:10A5F000140EF66E340EF76E0D0E0101956F00010C
:10A60000A0EC34F0010EE96EECC094F1EBC093F1D4
:10A61000EAC092F1E9C091F10101956B00019EEC55
:10A620003DF0250E0101A16F000130EC2EF089EC08
:10A6300030F02A0EF66E340EF76E74EC30F058D00F
:10A64000D9532AE168EC30F03C0EF66E340EF76E0A
:10A650000D0E0101956F0001A0EC34F0010EE96EC2
:10A66000ECC094F1EBC093F1EAC092F1E9C091F132
:10A670000101956B00019EEC3DF0250E0101A16FDB
:10A68000000130EC2EF089EC30F0520EF66E340EF4
:10A69000F76E74EC30F02CD0D9517F0829E168ECCA
:10A6A00030F0640EF66E340EF76E0D0E0101956FEC
:10A6B0000001A0EC34F0010EE96EECC094F1EBC0A7
:10A6C00093F1EAC092F1E9C091F10101956B0001AB
:10A6D0009EEC3DF0250E0101A16F000130EC2EF043
:10A6E00089EC30F07A0EF66E340EF76E74EC30F0C2
:10A6F00084D0D93D2AD068EC30F08C0EF66E340E42
:10A70000F76E0D0E0101956F0001A0EC34F0010E03
:10A71000E96EECC094F1EBC093F1EAC092F1E9C0AC
:10A7200091F10101956B00019EEC3DF0250E0101B8
:10A73000A16F000130EC2EF089EC30F0A20EF66E25
:10A74000340EF76E74EC30F058D0D9532AE168EC2F
:10A7500030F0B40EF66E340EF76E0D0E0101956FEB
:10A760000001A0EC34F0010EE96EECC094F1EBC0F6
:10A7700093F1EAC092F1E9C091F10101956B0001FA
:10A780009EEC3DF0250E0101A16F000130EC2EF092
:10A7900089EC30F0CA0EF66E340EF76E74EC30F0C1
:10A7A0002CD0D9517F0829E168EC30F0DC0EF66E30
:10A7B000340EF76E0D0E0101956F0001A0EC34F020
:10A7C000010EE96EECC094F1EBC093F1EAC092F196
:10A7D000E9C091F10101956B00019EEC3DF0250E61
:10A7E0000101A16F000130EC2EF089EC30F0F20E87
:10A7F000F66E340EF76E74EC30F0952D0DD0878721
:10A80000ED2B640E0101CE6F000105EC2EF0EDC0C2
:10A8100091F196EC30F019D0955104080DE187873D
:10A82000ED07640E0101CE6F000105EC2EF0EDC0C6
:10A8300091F196EC30F009D09551050806E101013F
:10A8400016971699169B169D0001A0D6640E01015D
:10A85000CE6F000105EC2EF087A728D041EC43F025
:10A86000952D1FD0D250006ED29E3901E16B0C0E97
:10A87000E06F6000B7F3E3F9E59DE59FE585550ED0
:10A88000E66FAA0EE66FE583E5B3FED7E595E59D95
:10A89000E58F0050D212EDC091F1000196EC30F03E
:10A8A00005D09551040801E101D0D8D7A82BDEEFDF
:10A8B0005CF0879F50EC34F068EC30F0040EF66EDC
:10A8C000350EF76E74EC30F0D93D28D089EC30F0BD
:10A8D000160EF66E350EF76E080E0101956F00012B
:10A8E000A0EC34F07F0E0101A16F000130EC2EF0DE
:10A8F000200EF66E350EF76E050E0101956F000104
:10A90000A0EC34F07E0E0101A16F000130EC2EF0BE
:10A91000200E0101A16F000130EC2EF0D95328E187
:10A9200089EC30F02A0EF66E350EF76E080E010136
:10A93000956F0001A0EC34F07F0E0101A16F0001C2
:10A9400030EC2EF0340EF66E350EF76E050E01016A
:10A95000956F0001A0EC34F07E0E0101A16F0001A3
:10A9600030EC2EF0200E0101A16F000130EC2EF032
:10A97000D9517F0828E189EC30F03E0EF66E350E95
:10A98000F76E080E0101956F0001A0EC34F07F0E08
:10A990000101A16F000130EC2EF0480EF66E350E6D
:10A9A000F76E050E0101956F0001A0EC34F07E0EEC
:10A9B0000101A16F000130EC2EF0200E0101A16F0A
:10A9C000000130EC2EF09551040801E1A82B952DE3
:10A9D00003D0CBAE01D0A807952D04D0CBBE02D0BA
:10A9E000A807A807952D09D0F92D07D0FA5103081B
:10A9F00004E1020EA86FDEEF5CF0955103084CE114
:10AA000050EC34F09551030846E068EC30F0520EFB
:10AA1000F66E350EF76E74EC30F0D93D09D089EC46
:10AA200030F0640EF66E350EF76E74EC30F016D022
:10AA3000D95309E189EC30F0760EF66E350EF76EDB
:10AA400074EC30F00BD0D9517F0808E189EC30F07C
:10AA5000880EF66E350EF76E74EC30F0952D07D03B
:10AA600088B705D001011689168B168D0001955106
:10AA7000040807E188B505D001011687168B169DDD
:10AA800000019551050806E1010116971699169BDC
:10AA9000169D0001B7D7A82B878FDEEF5CF0E85337
:10AAA00003E1A82BDEEF5CF050EC34F06F0048FFC0
:10AAB00091F1D29E3901E16B050EE06FE59DE59FB6
:10AAC000E581E351E59DE58F010191BFD28E000143
:10AAD000CE6FCE515A0802E2050ECE6FD66BCEC0B5
:10AAE000D5F0D93D31D068EC30F09A0EF66E350EC7
:10AAF000F76E74EC30F089EC30F0AC0EF66E350E7B
:10AB0000F76E080E0101956F0001A0EC34F07F0E86
:10AB10000101A16F000130EC2EF0B60EF66E350E7D
:10AB2000F76E050E0101956F0001A0EC34F07E0E6A
:10AB30000101A16F000130EC2EF0200E0101A16F88
:10AB4000000130EC2EF066D0D95331E168EC30F0E2
:10AB5000C00EF66E350EF76E74EC30F089EC30F006
:10AB6000D20EF66E350EF76E080E0101956F0001DC
:10AB7000A0EC34F07F0E0101A16F000130EC2EF04B
:10AB8000DC0EF66E350EF76E050E0101956F0001B5
:10AB9000A0EC34F07E0E0101A16F000130EC2EF02C
:10ABA000200E0101A16F000130EC2EF033D0D951FD
:10ABB0007F0830E168EC30F0E60EF66E350EF76E89
:10ABC00074EC30F089EC30F0F80EF66E350EF76E5E
:10ABD000080E0101956F0001A0EC34F07F0E010119
:10ABE000A16F000130EC2EF0020EF66E360EF76EFD
:10ABF000050E0101956F0001A0EC34F07E0E0101FD
:10AC0000A16F000130EC2EF0200E0101A16F0001B8
:10AC100030EC2EF09551040801E1A82B952D01D0C0
:10AC2000A807A85302E1010EA86F95510308D8A404
:10AC300052D150EC34F0879595510308D8B414D113
:10AC400087B57CD0D93D27D068EC30F00C0EF66E7D
:10AC5000360EF76E080E0101956F0001A0EC34F07E
:10AC6000CEC092F1130E0101936F0001D0EC34F0CD
:10AC7000170EF66E360EF76E050E0101956F000188
:10AC8000A0EC34F089EC30F01E0EF66E360EF76E46
:10AC900074EC30F052D0D95327E168EC30F0300E2C
:10ACA000F66E360EF76E090E0101956F0001A0ECED
:10ACB00034F0CEC092F1130E0101936F0001D0EC7D
:10ACC00034F03C0EF66E360EF76E040E0101956FF1
:10ACD0000001A0EC34F089EC30F0420EF66E360E36
:10ACE000F76E74EC30F029D0D9517F0826E168EC7A
:10ACF00030F0540EF66E360EF76E090E0101956FA8
:10AD00000001A0EC34F0CEC092F1130E0101936F5C
:10AD10000001D0EC34F0600EF66E360EF76E040EC5
:10AD20000101956F0001A0EC34F089EC30F0660E63
:10AD3000F66E360EF76E74EC30F07BD0D93D27D02E
:10AD400068EC30F0780EF66E360EF76E080E0101E4
:10AD5000956F0001A0EC34F0CEC092F1130E01010A
:10AD6000936F0001D0EC34F0830EF66E360EF76E62
:10AD7000050E0101956F0001A0EC34F089EC30F074
:10AD80008A0EF66E360EF76E74EC30F052D0D95350
:10AD900027E168EC30F09C0EF66E360EF76E090E69
:10ADA0000101956F0001A0EC34F0CEC092F1130EBA
:10ADB0000101936F0001D0EC34F0A80EF66E360E50
:10ADC000F76E040E0101956F0001A0EC34F089ECE0
:10ADD00030F0AE0EF66E360EF76E74EC30F029D011
:10ADE000D9517F0826E168EC30F0C00EF66E360EC1
:10ADF000F76E090E0101956F0001A0EC34F0CEC092
:10AE000092F1130E0101936F0001D0EC34F0CC0EDF
:10AE1000F66E360EF76E040E0101956F0001A0EC80
:10AE200034F089EC30F0D20EF66E360EF76E74EC1C
:10AE300030F0640E0101CE6F000105EC2EF095514B
:10AE4000040805E18785CE51590801E3CE2B640E35
:10AE50000101CE6F000105EC2EF0952D04D0878501
:10AE6000CE5301E0CE07E8D6640E0101CE6F00019B
:10AE700005EC2EF087A52ED041EC43F00A0E01011F
:10AE8000CE6F000105EC2EF0952D1FD0D250006E34
:10AE9000D29E3901E16B050EE06F60003BF3E3F9F0
:10AEA000E59DE59FE585550EE66FAA0EE66FE58305
:10AEB000E5B3FED7E595E59DE58F0050D212000180
:10AEC000D66BCEC0D5F006D004D09551040801E170
:10AED00001D0D2D7A82BDEEF5CF0F92D06D0FA51C5
:10AEE000030803E1A82BDEEF5CF050EC34F0D93D11
:10AEF00009D068EC30F0E40EF66E360EF76E74ECA6
:10AF000030F016D0D95309E168EC30F0F60EF66E49
:10AF1000360EF76E74EC30F00BD0D9517F0808E193
:10AF200068EC30F0080EF66E370EF76E74EC30F009
:10AF3000D93D29D089EC30F01A0EF66E370EF76E37
:10AF4000080E0101956F0001A0EC34F07F0E0101A5
:10AF5000A16F000130EC2EF0240EF66E370EF76E66
:10AF6000050E0101956F0001A0EC34F07E0E010189
:10AF7000A16F000130EC2EF0200E0101A16F000145
:10AF800030EC2EF056D0D95329E189EC30F02E0E5A
:10AF9000F66E370EF76E080E0101956F0001A0ECFA
:10AFA00034F07F0E0101A16F000130EC2EF0380E5D
:10AFB000F66E370EF76E050E0101956F0001A0ECDD
:10AFC00034F07E0E0101A16F000130EC2EF0200E56
:10AFD0000101A16F000130EC2EF02BD0D9517F0878
:10AFE00028E189EC30F0420EF66E370EF76E080E4F
:10AFF0000101956F0001A0EC34F07F0E0101A16FFB
:10B00000000130EC2EF04C0EF66E370EF76E050E8A
:10B010000101956F0001A0EC34F07E0E0101A16FDB
:10B02000000130EC2EF0200E0101A16F000130EC88
:10B030002EF09551040801E1A82B952D07D0A80703
:10B04000F92D04D0FA51030801E1A807A85302E141
:10B05000010EA86F95510308D8A451D1D93D09D04C
:10B0600068EC30F0560EF66E370EF76E74EC30F07A
:10B0700016D0D95309E168EC30F0680EF66E370E41
:10B08000F76E74EC30F00BD0D9517F0808E168EC12
:10B0900030F07A0EF66E370EF76E74EC30F0D93D64
:10B0A00009D089EC30F08C0EF66E370EF76E74EC2A
:10B0B00030F016D0D95309E189EC30F09E0EF66ECF
:10B0C000370EF76E74EC30F00BD0D9517F0808E1E1
:10B0D00089EC30F0B00EF66E370EF76E74EC30F08F
:10B0E00050EC34F095510308D8B4DFD0D93D09D0E5
:10B0F00068EC30F0C20EF66E370EF76E74EC30F07E
:10B1000016D0D95309E168EC30F0D40EF66E370E44
:10B11000F76E74EC30F00BD0D9517F0808E168EC81
:10B1200030F0E60EF66E370EF76E74EC30F0D93D67
:10B1300009D089EC30F0F80EF66E370EF76E74EC2D
:10B1400030F01BD0D95309E189EC30F00A0EF66ECD
:10B15000380EF76E74EC30F010D0D9517F0809E149
:10B1600089EC30F01C0EF66E380EF76E74EC30F091
:10B1700004D095510308D8B4BFD0952D49D050ECD8
:10B1800034F09551050844E1D93D09D068EC30F020
:10B190002E0EF66E380EF76E74EC30F016D0D953D2
:10B1A00009E168EC30F0400EF66E380EF76E74EC84
:10B1B00030F00BD0D9517F0808E168EC30F0520E26
:10B1C000F66E380EF76E74EC30F0D93D09D089EC8C
:10B1D00030F0640EF66E380EF76E74EC30F016D068
:10B1E000D95309E189EC30F0760EF66E380EF76E21
:10B1F00074EC30F00BD0D9517F0808E189EC30F0C5
:10B20000880EF66E380EF76E74EC30F0E869B9D738
:10B210009551040849E150EC34F09551050844E19A
:10B22000D93D09D068EC30F09A0EF66E380EF76E04
:10B2300074EC30F016D0D95309E168EC30F0AC0E64
:10B24000F66E380EF76E74EC30F00BD0D9517F08E3
:10B2500008E168EC30F0BE0EF66E380EF76E74EC56
:10B2600030F0D93D09D089EC30F0D00EF66E380EB2
:10B27000F76E74EC30F016D0D95309E189EC30F058
:10B28000E20EF66E380EF76E74EC30F00BD0D9513A
:10B290007F0808E189EC30F0F40EF66E380EF76E98
:10B2A00074EC30F0E86BB9D71DD741EC43F0952D25
:10B2B0001CD0D250006ED29E3901E16B150EE06FAA
:10B2C0006000A3F3E3F9E59DE59FE585550EE66F84
:10B2D000AA0EE66FE583E5B3FED7E595E59DE58F1C
:10B2E0000050D2120AD006D000019551040803E1A3
:10B2F000390103D00001D9D739010001A82B5ED351
:10B30000F92D05D0FA51030802E1A82B57D350ECD0
:10B3100034F068EC30F0060EF66E390EF76E74EC11
:10B3200030F089EC30F0180EF66E390EF76E080E1C
:10B330000101956F0001A0EC34F07F0E0101A16FB7
:10B34000000130EC2EF0220EF66E390EF76E050E6F
:10B350000101956F0001A0EC34F07E0E0101A16F98
:10B36000000130EC2EF0200E0101A16F000130EC45
:10B370002EF09551040801E1A82B952D07D0A807C0
:10B38000F92D04D0FA51030801E1A807A85302E1FE
:10B39000010EA86F95510308D8A4C5D068EC30F011
:10B3A0002C0EF66E390EF76E74EC30F089EC30F03E
:10B3B0003E0EF66E390EF76E74EC30F050EC34F051
:10B3C0009551030805E1952D03D09551040862E0DD
:10B3D00068EC30F0500EF66E390EF76E74EC30F00B
:10B3E00089EC30F0620EF66E390EF76E74EC30F0C8
:10B3F0009551030819E150EC34F09551050814E11A
:10B4000068EC30F0740EF66E390EF76E74EC30F0B6
:10B4100089EC30F0860EF66E390EF76E74EC30F073
:10B420007F0ED96F37D0E9D7952D18D050EC34F076
:10B430009551050813E168EC30F0980EF66E390E60
:10B44000F76E74EC30F089EC30F0AA0EF66E390E1F
:10B45000F76E74EC30F0D96B1DD0EAD79551040823
:10B4600018E150EC34F09551050813E168EC30F028
:10B47000BC0EF66E390EF76E74EC30F089EC30F0DD
:10B48000CE0EF66E390EF76E74EC30F0D96902D03C
:10B49000EAD796D7080E0101916FFA0ECE6F000120
:10B4A00005EC2EF00101912FF8D7000141EC43F09B
:10B4B000952D1CD0D250006ED29E3901E16B3C0E0E
:10B4C000E06F600067F3E3F9E59DE59FE585550EC4
:10B4D000E66FAA0EE66FE583E5B3FED7E595E59D39
:10B4E000E58F0050D2121DD019D0000195510408EB
:10B4F00016E16F0048FF91F1D29E3901E16B3C0EDD
:10B50000E06FE59DE59FE581E351E59DE58F010154
:10B5100091BFD28E0001D96F390103D00001C6D787
:10B5200039010001A82B4AD250EC34F0D93D31D07A
:10B5300068EC30F0E00EF66E390EF76E74EC30F019
:10B5400089EC30F0F20EF66E390EF76E080E01013E
:10B55000956F0001A0EC34F07F0E0101A16F000196
:10B5600030EC2EF0FC0EF66E390EF76E050E010172
:10B57000956F0001A0EC34F07E0E0101A16F000177
:10B5800030EC2EF0200E0101A16F000130EC2EF006
:10B5900066D0D95331E168EC30F0060EF66E3A0E03
:10B5A000F76E74EC30F089EC30F0180EF66E3A0E4F
:10B5B000F76E080E0101956F0001A0EC34F07F0ECC
:10B5C0000101A16F000130EC2EF0220EF66E3A0E52
:10B5D000F76E050E0101956F0001A0EC34F07E0EB0
:10B5E0000101A16F000130EC2EF0200E0101A16FCE
:10B5F000000130EC2EF033D0D9517F0830E168ECF7
:10B6000030F02C0EF66E3A0EF76E74EC30F089ECDA
:10B6100030F03E0EF66E3A0EF76E080E0101956F91
:10B620000001A0EC34F07F0E0101A16F000130ECAD
:10B630002EF0480EF66E3A0EF76E050E0101956F6C
:10B640000001A0EC34F07E0E0101A16F000130EC8E
:10B650002EF0200E0101A16F000130EC2EF095516B
:10B66000040801E1A82B952D01D0A80795510308E6
:10B67000D8A4F9D050EC34F095510308D8B4C7D011
:10B68000D93D11D068EC30F0520EF66E3A0EF76EDE
:10B6900074EC30F089EC30F0640EF66E3A0EF76E12
:10B6A00074EC30F026D0D95311E168EC30F0760E0E
:10B6B000F66E3A0EF76E74EC30F089EC30F0880ECE
:10B6C000F66E3A0EF76E74EC30F013D0D9517F0855
:10B6D00010E168EC30F09A0EF66E3A0EF76E74ECEC
:10B6E00030F089EC30F0AC0EF66E3A0EF76E74EC7A
:10B6F00030F095510308D8B4B6D0952D42D050EC17
:10B7000034F0955105083DE1D93D11D068EC30F099
:10B71000BE0EF66E3A0EF76E74EC30F089EC30F037
:10B72000D00EF66E3A0EF76E74EC30F026D0D95388
:10B7300011E168EC30F0E20EF66E3A0EF76E74EC42
:10B7400030F089EC30F0F40EF66E3A0EF76E74ECD1
:10B7500030F013D0D9517F0810E168EC30F0060EBC
:10B76000F66E3B0EF76E74EC30F089EC30F0180E8C
:10B77000F66E3B0EF76E74EC30F00101806B000149
:10B78000C0D79551040842E150EC34F095510508BA
:10B790003DE1D93D11D068EC30F02A0EF66E3B0E3B
:10B7A000F76E74EC30F089EC30F03C0EF66E3B0E28
:10B7B000F76E74EC30F026D0D95311E168EC30F01C
:10B7C0004E0EF66E3B0EF76E74EC30F089EC30F0F6
:10B7D000600EF66E3B0EF76E74EC30F013D0D9515C
:10B7E0007F0810E168EC30F0720EF66E3B0EF76EDB
:10B7F00074EC30F089EC30F0840EF66E3B0EF76E90
:10B8000074EC30F0010180690001C0D735D750ECED
:10B8100034F041EC43F0952D1CD0D250006ED29EF6
:10B820003901E16B010EE06F600003F6E3F9E59D7D
:10B83000E59FE585550EE66FAA0EE66FE583E5B355
:10B84000FED7E595E59DE58F0050D2120AD006D0CF
:10B8500000019551040803E1390103D00001D9D753
:10B8600039010001A82B0001A9D050EC34F0D93DDA
:10B8700031D068EC30F0960EF66E3B0EF76E74EC3D
:10B8800030F089EC30F0A80EF66E3B0EF76E080E25
:10B890000101956F0001A0EC34F07F0E0101A16F52
:10B8A000000130EC2EF0B20EF66E3B0EF76E050E78
:10B8B0000101956F0001A0EC34F07E0E0101A16F33
:10B8C000000130EC2EF0200E0101A16F000130ECE0
:10B8D0002EF066D0D95331E168EC30F0BC0EF66E34
:10B8E0003B0EF76E74EC30F089EC30F0CE0EF66E55
:10B8F0003B0EF76E080E0101956F0001A0EC34F0CD
:10B900007F0E0101A16F000130EC2EF0D80EF66E13
:10B910003B0EF76E050E0101956F0001A0EC34F0AF
:10B920007E0E0101A16F000130EC2EF0200E01010E
:10B93000A16F000130EC2EF033D0D9517F0830E1F7
:10B9400068EC30F0E20EF66E3B0EF76E74EC30F001
:10B9500089EC30F0F40EF66E3B0EF76E080E010126
:10B96000956F0001A0EC34F07F0E0101A16F000182
:10B9700030EC2EF0FE0EF66E3B0EF76E050E01015A
:10B98000956F0001A0EC34F07E0E0101A16F000163
:10B9900030EC2EF0200E0101A16F000130EC2EF0F2
:10B9A0009551040802E1010EA86F952D02D00D0EED
:10B9B000A86F95510308D8B403D000D08FEF43F09F
:10B9C000010116B703D016B901D0FF003901988DD7
:10B9D000000199EF5DF00101966B956B946B936B91
:10B9E0009A6B996B986B320E976F0001B9EC30F03F
:10B9F00088918E6BB253D8A4A1D0B353D8A49ED053
:10BA0000B453D8A49BD0B553D8A498D001011697AD
:10BA10001699169B169D000188B14AD0D93D16D0C3
:10BA200068EC30F0080EF66E3C0EF76E74EC30F0F9
:10BA30000A0E0101CE6F000105EC2EF089EC30F00A
:10BA40001A0EF66E3C0EF76E74EC30F0D95316E118
:10BA500068EC30F02C0EF66E3C0EF76E74EC30F0A5
:10BA60000A0E0101CE6F000105EC2EF089EC30F0DA
:10BA70003E0EF66E3C0EF76E74EC30F0D9517F0836
:10BA800016E168EC30F0500EF66E3C0EF76E74EC7A
:10BA900030F00A0E0101CE6F000105EC2EF089ECAA
:10BAA00030F0620EF66E3C0EF76E74EC30F037D06C
:10BAB000D93D10D068EC30F0740EF66E3C0EF76E87
:10BAC00074EC30F089EC30F0860EF66E3C0EF76EBA
:10BAD00074EC30F0D95310E168EC30F0980EF66E4B
:10BAE0003C0EF76E74EC30F089EC30F0AA0EF66E76
:10BAF0003C0EF76E74EC30F0D9517F0810E168EC21
:10BB000030F0BC0EF66E3C0EF76E74EC30F089EC43
:10BB100030F0CE0EF66E3C0EF76E74EC30F0B25391
:10BB200006E1B35304E1B45302E1B553D8A47FEF67
:10BB300043F095510208D8A401D05CD7F0530DE131
:10BB40000101966B956B946B936B9A6B996B986BE9
:10BB5000E2C097F10001B9EC30F066EC2EF0120073
:10BB6000010192BF12D00F0E006E913900160A0E1D
:10BB7000005C03E2300E002602D09251002600C085
:10BB8000A1F1000130EC2EF001010F0E91170A0E09
:10BB9000915D02E2300E02D0929F9251912791C1A5
:10BBA000A1F1000130EC2EF01200010E656F91C181
:10BBB00092F1100E0101936F946B956B966B0E0EC4
:10BBC000976F1C0E986FB96BB9510A0846E3D8906D
:10BBD000B935070F036A920F016E010E032203C0ED
:10BBE000BBF1D890B935036A1B0FE96E010E032033
:10BBF000EA6E6F00B0FFBDF1ED526F00BCFFBCF10B
:10BC00006000EFF6EAFF600007F0E9FF6000F7F67A
:10BC1000EFFFD890B935080F036A920F016E010E3D
:10BC2000032203C0BBF1D890B935036A1B0FE96E3C
:10BC3000010E0320EA6E6F00B0FFBDF1ED526F0000
:10BC4000BCFFBCF16000EFF6EAFF600007F0E9FF1F
:10BC50006000F3F6EFFFB92BB7D7AF6B1BC0B0F1A5
:10BC6000B16B1DC0B2F1B36B1FC0B4F1010ECF6F49
:10BC7000920ECE6F230ED06F0001E6EC30F002C0C2
:10BC8000B8F101C0B7F1B7C1B5F10101B851B66F54
:10BC9000BB843D01F98F0101B96BB951240811E34F
:10BCA000036AB951920FE96E010E0320EA6E6F002C
:10BCB000BCFFBAF1BA5100011BEC31F00101B92B04
:10BCC000ECD73D01F9AFFED7F98FBB94000112000C
:10BCD00069A308D00101916B000167DF69A302D05D
:10BCE0006993FCD7120068EC30F0C00EF66E220E9D
:10BCF000F76E030E0101956F0001A0EC34F09FC0B8
:10BD0000A1F130EC2EF0A0C0A1F130EC2EF0A1C0DA
:10BD1000A1F130EC2EF0A2C0A1F130EC2EF0A3C0C6
:10BD2000A1F130EC2EF0A4C0A1F130EC2EF0A5C0B2
:10BD3000A1F130EC2EF0A6C0A1F130EC2EF0D30E24
:10BD4000F66E220EF76E050E0101956F0001A0EC54
:10BD500034F01200F55322E101011053D8A402D0AF
:10BD600000011CD0000168EC30F0BA0EF66E420EF5
:10BD7000F76E74EC30F089EC30F0CC0EF66E420EBB
:10BD8000F76E74EC30F0BC96BC94BC92BC90010190
:10BD900016971699169B169D0001DCD71200FE53CC
:10BDA00003E02F0E966F02D07C0E966F01010053B8
:10BDB00005E02F0E0001976F04D001017C0E0001F9
:10BDC000976F0101025305E02F0E0001986F04D018
:10BDD00001017C0E0001986F0101045305E02F0E54
:10BDE0000001996F04D001017C0E0001996F0101DF
:10BDF000065305E02F0E00019A6F04D001017C0E5E
:10BE000000019A6F0101085305E02F0E00019B6F9E
:10BE100004D001017C0E00019B6F01010A5305E073
:10BE20002F0E00019C6F04D001017C0E00019C6F5D
:10BE300001010C5305E02F0E00019D6F04D001019C
:10BE40007C0E00019D6FCBAE03D02F0E9E6F02D0F3
:10BE50007C0E9E6FF63D55D0F4AF03D07C0E9F6FE5
:10BE600002D02F0E9F6F010116A105D07C0E00019C
:10BE7000A06F04D001012F0E0001A06F010116A3D5
:10BE800005D07C0E0001A16F04D001012F0E00012E
:10BE9000A16F010116A505D07C0E0001A26F04D090
:10BEA00001012F0E0001A26F010116A705D07C0E23
:10BEB0000001A36F04D001012F0E0001A36F010147
:10BEC00016A905D07C0E0001A46F04D001012F0E2D
:10BED0000001A46F010116AB05D07C0E0001A56F17
:10BEE00004D001012F0E0001A56F010116AD05D090
:10BEF0007C0E0001A66F04D001012F0E0001A66F79
:10BF000054D0F4AF03D07C0E9F6F02D02F0E9F6FE2
:10BF1000010116A105D07C0E0001A06F04D0010123
:10BF20002F0E0001A06F010116A305D07C0E0001A9
:10BF3000A16F04D001012F0E0001A16F010116A510
:10BF400005D07C0E0001A26F04D001012F0E00016C
:10BF5000A26F010116A705D07C0E0001A36F04D0CB
:10BF600001012F0E0001A36F010116A905D07C0E5F
:10BF70000001A46F04D001012F0E0001A46F010184
:10BF800016AB05D07C0E0001A56F04D001012F0E69
:10BF90000001A56F010116AD05D07C0E0001A66F52
:10BFA00004D001012F0E0001A66F120089EC30F0C1
:10BFB000DA0EF66E220EF76E030E0101956F000188
:10BFC000A0EC34F096C0A1F130EC2EF097C0A1F1B6
:10BFD00030EC2EF098C0A1F130EC2EF099C0A1F118
:10BFE00030EC2EF09AC0A1F130EC2EF09BC0A1F104
:10BFF00030EC2EF09CC0A1F130EC2EF09DC0A1F1F0
:10C0000030EC2EF0ED0EF66E220EF76E050E0101ED
:10C01000956F0001A0EC34F01200952D74D069A941
:10C020003BD089EC30F0DE0EF66E420EF76E030E5A
:10C030000101956F0001A0EC34F096C0A1F130EC45
:10C040002EF097C0A1F130EC2EF098C0A1F130ECA9
:10C050002EF099C0A1F130EC2EF09AC0A1F130EC95
:10C060002EF09BC0A1F130EC2EF09CC0A1F130EC81
:10C070002EF09DC0A1F130EC2EF0F10EF66E420EC6
:10C08000F76E040E0101956F0001A0EC34F09EC024
:10C09000A1F130EC2EF036D089EC30F0F80EF66ECF
:10C0A000420EF76E030E0101956F0001A0EC34F013
:10C0B00096C0A1F130EC2EF097C0A1F130EC2EF03B
:10C0C00098C0A1F130EC2EF099C0A1F130EC2EF027
:10C0D0009AC0A1F130EC2EF09BC0A1F130EC2EF013
:10C0E0009CC0A1F130EC2EF09DC0A1F130EC2EF0FF
:10C0F0000B0EF66E430EF76E050E0101956F0001F3
:10C10000A0EC34F0F0DD706B716BFE53D8B4BDD091
:10C11000D6C093F1D5C092F10101956B0A0E946FD0
:10C1200000019FEC2EF002C092F101C091F10101DB
:10C13000966B956B946B936B9A6B996B02C098F1AD
:10C1400001C097F10001B9EC30F004DE010116974F
:10C150001699169B169D0001F487952D01D090D05D
:10C16000D93D23D0772D11D068EC30F0120EF66E49
:10C17000430EF76E74EC30F089EC30F0240EF66E5E
:10C18000430EF76E74EC30F010D068EC30F0360EE1
:10C19000F66E430EF76E74EC30F089EC30F0480E1A
:10C1A000F66E430EF76E74EC30F0D95310E168EC84
:10C1B00030F05A0EF66E430EF76E74EC30F089ECE8
:10C1C00030F06C0EF66E430EF76E74EC30F0D95111
:10C1D0007F0810E168EC30F07E0EF66E430EF76ECD
:10C1E00074EC30F089EC30F0900EF66E430EF76E82
:10C1F00074EC30F00101916B0001D7DC320E0101CB
:10C20000CE6F000105EC2EF001017FA737D0050E9F
:10C21000AC6FAE6B030EAD6F010EAF6FB16B780EEE
:10C22000B06F000122EC31F00152D8A402D001011C
:10C2300025D079C076F078C077F0772D1ED0D25017
:10C24000006ED29E3901E16B020EE06FE36BE59D5B
:10C25000E59FE585550EE66FAA0EE66FE583E5B32B
:10C26000FED7E595E59DE58F0050D212640E0101E1
:10C27000CE6F000105EC2EF0FF00010104D000019B
:10C280008EDD31DD93DE000140D71200E95001015F
:10C29000996F3B0EA06F9A0E9F6FCA0E9E6F9D6B9B
:10C2A0000A0E9B6FD882010EEA6E950EE96E196A2E
:10C2B000D2BE198ED29E98C1DEF197C1DDF196C132
:10C2C000DCF195C1DBF1A0C1E2F19FC1E1F19EC1BA
:10C2D000E0F19DC1DFF100010CEC25F019BED28E1A
:10C2E0000150005213E101019B51010AD8A402D070
:10C2F00000010CD099510CE00F0B9B5D01E010E2A6
:10C3000099BF0ED099BD04D0200E03D00101996BC6
:10C31000300E002600C0A1F1000130EC2EF001012A
:10C32000D892196AD2BE198ED29EA0C1DEF19FC1E9
:10C33000DDF19EC1DCF19DC1DBF1E26BE16BE06BF5
:10C340000A0EDF6F00010CEC25F019BED28E03C07F
:10C35000A0F102C09FF101C09EF100C09DF101015A
:10C360009B2FA0D7000112000101168700011200C7
:10C37000EF5215E06F00A8FF92F16F00A4FF91F15A
:10C380006F00BCFFA1F130EC2EF060004BF6EAFF2D
:10C39000600047F6E9FFE92AD8B4EA2AE9D7120093
:10C3A000016A026A006A036A0101965102E195512D
:10C3B00018E0100E976FD8909337943700360336F5
:10C3C0009651035C02E19551005C07E39551005ED4
:10C3D000D8A003069651035ED88001360236972F07
:10C3E000EAD7000112006F00A8FF9BF16F00A4FFC5
:10C3F0009AF101019439F009966F9627E20F976F31
:10C40000320F996F94510F0B972797279927E90FB0
:10C41000986F9827982793390F0B98279927983763
:10C420009937991F993793510F0B99279637070E14
:10C43000956F0A0E98079927FDE397079827FDE364
:10C4400096079727FDE395079627FDE3010EEA6E11
:10C45000950EE96E070E9A159A9DE926000EEA22BE
:10C46000E950990803E1EA2C01D09A8DEF50006E53
:10C4700008E19ABD06D09AB91AD09AB702D0200E18
:10C4800003D09A879A99300E00266F00A8FF94F186
:10C490006F00A4FF93F100C0A1F1000130EC2EF079
:10C4A000600053F6EAFF60004FF6E9FF0101EE502D
:10C4B0009AADD6D7000112008F6B95510308D8A40E
:10C4C00061EF66F087898F51080801E28F6B0101E7
:10C4D00016971699169B169D0001878F8F5118E0AD
:10C4E000010A42E0030AD8B491D0010AD8B458D165
:10C4F000070AD8B4BAD1010AD8B42AD2030AD8B4E8
:10C50000ABD2010AD8B41BD30F0AD8B43ED36ED332
:10C5100068EC30F0A40EF66E450EF76E74EC30F059
:10C52000D93D11D089EC30F0B60EF66E450EF76E9F
:10C530000B0E0101956F0001A0EC34F0EA6A1B0EAE
:10C54000E96E16DF10D089EC30F0C40EF66E450EA1
:10C55000F76E0B0E0101956F0001A0EC34F0EA6A52
:10C560001B0EE96E05DF42D3D9517F0809E168EC63
:10C5700030F0D20EF66E450EF76E74EC30F008D047
:10C5800068EC30F0E40EF66E450EF76E74EC30F0A9
:10C59000D93D12D088B989EC30F0F60EF66E450E12
:10C5A000F76E74EC30F088A989EC30F0080EF66E66
:10C5B000460EF76E74EC30F0D95312E188B989EC6D
:10C5C00030F01A0EF66E460EF76E74EC30F088A955
:10C5D00089EC30F02C0EF66E460EF76E74EC30F0EF
:10C5E000D9517F0812E188B989EC30F03E0EF66E21
:10C5F000460EF76E74EC30F088A989EC30F0500EDE
:10C60000F66E460EF76E74EC30F0F0D2D9517F081A
:10C6100009E168EC30F0620EF66E460EF76E74ECCF
:10C6200030F008D068EC30F0740EF66E460EF76EFF
:10C6300074EC30F0D93D3AD089EC30F0D6C093F1AB
:10C64000D5C092F10101956B0A0E946F00019FEC29
:10C650002EF002C092F101C091F102C094F101C02C
:10C6600093F10101966B0A0E956F000199DE02C0ED
:10C6700092F101C091F1860EF66E460EF76E0A0E2B
:10C680000101956F0001A0EC34F0030EE96E92C138
:10C6900094F191C193F1A7DE940EF66E460EF76EFB
:10C6A000040E0101956F0001A0EC34F0D9533AE17A
:10C6B00089EC30F0D6C093F1D5C092F10101956BB1
:10C6C0000A0E946F00019FEC2EF002C092F101C09F
:10C6D00091F102C094F101C093F10101966B0A0E31
:10C6E000956F00015DDE02C092F101C091F19A0EDA
:10C6F000F66E460EF76E0A0E0101956F0001A0EC72
:10C7000034F0030EE96E92C194F191C193F16BDEA6
:10C71000A80EF66E460EF76E040E0101956F00012D
:10C72000A0EC34F0D9517F083AE189EC30F0D6C062
:10C7300093F1D5C092F10101956B0A0E946F00013F
:10C740009FEC2EF002C092F101C091F102C094F171
:10C7500001C093F10101966B0A0E956F000120DE76
:10C7600002C092F101C091F1AE0EF66E460EF76E68
:10C770000A0E0101956F0001A0EC34F0030EE96E82
:10C7800092C194F191C193F12EDEBC0EF66E460E6D
:10C79000F76E040E0101956F0001A0EC34F026D273
:10C7A000D93D1FD068EC30F0C20EF66E460EF76E23
:10C7B00074EC30F089EC30F0D40EF66E460EF76E65
:10C7C0000B0E0101956F0001A0EC34F0050EE96E2F
:10C7D000CDC098F1CCC097F1CBC096F1CAC095F10D
:10C7E00055DDD9531FE168EC30F0E40EF66E460ECD
:10C7F000F76E74EC30F089EC30F0F60EF66E460E03
:10C80000F76E0B0E0101956F0001A0EC34F0050EE0
:10C81000E96ECDC098F1CCC097F1CBC096F1CAC0FB
:10C8200095F134DDD9517F081FE168EC30F0060E38
:10C83000F66E470EF76E74EC30F089EC30F0180E9F
:10C84000F66E470EF76E0B0E0101956F0001A0EC1E
:10C8500034F0050EE96ECDC098F1CCC097F1CBC095
:10C8600096F1CAC095F112DDC1D1F05337E1D93D3F
:10C8700010D068EC30F0280EF66E470EF76E74ECB0
:10C8800030F089EC30F03A0EF66E470EF76E74EC2D
:10C8900030F0D95310E168EC30F04C0EF66E470ED4
:10C8A000F76E74EC30F089EC30F05E0EF66E470EE9
:10C8B000F76E74EC30F0D9517F0810E168EC30F07D
:10C8C000700EF66E470EF76E74EC30F089EC30F0B7
:10C8D000820EF66E470EF76E74EC30F0F03D37D0F6
:10C8E000D93D10D068EC30F0940EF66E470EF76E1E
:10C8F00074EC30F089EC30F0A60EF66E470EF76E51
:10C9000074EC30F0D95310E168EC30F0B80EF66EEC
:10C91000470EF76E74EC30F089EC30F0CA0EF66E0C
:10C92000470EF76E74EC30F0D9517F0810E168ECD7
:10C9300030F0DC0EF66E470EF76E74EC30F089ECDA
:10C9400030F0EE0EF66E470EF76E74EC30F04ED10E
:10C9500069B901D04BD1CBAE7ED0EDC0EEF0ED5138
:10C96000FF0AEE6F0101946BEEC093F10001B2EC8F
:10C970002EF003C0A1F102C0A0F101C09FF100C0E0
:10C980009EF1550E0101A56FC10EA46F480EA36F55
:10C990007D0EA26F00017DEC2FF003C0ECF002C011
:10C9A000EBF001C0EAF000C0E9F0D9517F082AE1BC
:10C9B00068EC30F0000EF66E480EF76E74EC30F056
:10C9C00089EC30F0120EF66E480EF76E0D0E010176
:10C9D000956F0001A0EC34F0010EE96EECC094F10B
:10C9E000EBC093F1EAC092F1E9C091F10101956BBE
:10C9F00000019EEC3DF0250E0101A16F000130EC1D
:10CA00002EF029D068EC30F0280EF66E480EF76E46
:10CA100074EC30F089EC30F03A0EF66E480EF76E9A
:10CA20000D0E0101956F0001A0EC34F0010EE96ECE
:10CA3000ECC094F1EBC093F1EAC092F1E9C091F13E
:10CA40000101956B00019EEC3DF0250E0101A16FE7
:10CA5000000130EC2EF0CAD0F15337E1D93D10D0AF
:10CA600068EC30F0500EF66E480EF76E74EC30F055
:10CA700089EC30F0620EF66E480EF76E74EC30F012
:10CA8000D95310E168EC30F0740EF66E480EF76E74
:10CA900074EC30F089EC30F0860EF66E480EF76ECE
:10CAA00074EC30F0D9517F0810E168EC30F0980E4A
:10CAB000F66E480EF76E74EC30F089EC30F0AA0E8A
:10CAC000F66E480EF76E74EC30F0F13D37D0D93D7C
:10CAD00010D068EC30F0BC0EF66E480EF76E74ECB9
:10CAE00030F089EC30F0CE0EF66E480EF76E74EC36
:10CAF00030F0D95310E168EC30F0E00EF66E480EDD
:10CB0000F76E74EC30F089EC30F0F20EF66E480EF1
:10CB1000F76E74EC30F0D9517F0810E168EC30F01A
:10CB2000040EF66E490EF76E74EC30F089EC30F0BE
:10CB3000160EF66E490EF76E74EC30F057D0F553C2
:10CB400011E168EC30F0280EF66E490EF76E74ECC9
:10CB500030F089EC30F03A0EF66E490EF76E74EC58
:10CB600030F012D0F53D10D068EC30F04C0EF66E7F
:10CB7000490EF76E74EC30F089EC30F05E0EF66E14
:10CB8000490EF76E74EC30F031D0D93D16D001016A
:10CB900017BF02D0000111D0000168EC30F0700E18
:10CBA000F66E490EF76E74EC30F089EC30F0820EC0
:10CBB000F66E490EF76E74EC30F0D95316E10101B0
:10CBC00017BF02D0000111D0000168EC30F0940EC4
:10CBD000F66E490EF76E74EC30F089EC30F0A60E6C
:10CBE000F66E490EF76E74EC30F000D00101966BD2
:10CBF000956B946B936B9A6B996B986B0A0E976F0E
:10CC00000001B9EC30F0B2530FE1B3530DE1B4536E
:10CC10000BE1B55309E195510308D8A405D03901BA
:10CC20005B5104000001EFD78F5107082EE068EC3C
:10CC300030F0B80EF66E490EF76E74EC30F089ECF9
:10CC400030F0CA0EF66E490EF76E74EC30F001014A
:10CC5000966B956B946B936B9A6B996B986B050EB7
:10CC6000976F0001B9EC30F0B2530FE1B3530DE10F
:10CC7000B4530BE1B55309E195510308D8A405D08D
:10CC800039015B5104000001EFD78F2B69B904D043
:10CC90008F51050801E18F2BF0530DE10101966BD7
:10CCA000956B946B936B9A6B996B986BE2C097F151
:10CCB0000001B9EC30F095510308D8A402D05DEF23
:10CCC00062F012000101045308E10001F53D01D0BA
:10CCD00002D0010102D00AD001010E53D8B4D2D043
:10CCE0000001F553D8B402D00101CCD0F4AF05D087
:10CCF000F53D03D00101C6D00001F5531DE101014E
:10CD00000E5318E0000168EC30F0A20EF66E430EF0
:10CD1000F76E74EC30F089EC30F0B40EF66E430E22
:10CD2000F76E74EC30F0010116971699169B169D5C
:10CD30001785E8D7A6D000010101169716990001C2
:10CD4000CFEC5EF0FE5309E10101105303E0000156
:10CD5000F55303E00001952D02D00DEC60F09551E4
:10CD6000020802E1EBEC5CF0952D01D003D0955167
:10CD7000070841E169A93BD089EC30F0C60EF66E98
:10CD8000430EF76E030E0101956F0001A0EC34F025
:10CD900096C0A1F130EC2EF097C0A1F130EC2EF04E
:10CDA00098C0A1F130EC2EF099C0A1F130EC2EF03A
:10CDB0009AC0A1F130EC2EF09BC0A1F130EC2EF026
:10CDC0009CC0A1F130EC2EF09DC0A1F130EC2EF012
:10CDD000D90EF66E430EF76E040E0101956F000139
:10CDE000A0EC34F09EC0A1F130EC2EF002D0D6ECD5
:10CDF0005FF073EC5EF0952D03D09551070840E08D
:10CE0000D93D13D0952D01D010D068EC30F0E00E54
:10CE1000F66E430EF76E74EC30F089EC30F0F20EE3
:10CE2000F66E430EF76E74EC30F0D95313E1952D86
:10CE300001D010D068EC30F0040EF66E440EF76EA0
:10CE400074EC30F089EC30F0160EF66E440EF76E8E
:10CE500074EC30F0D9517F0813E1952D01D010D03A
:10CE600068EC30F0280EF66E440EF76E74EC30F07D
:10CE700089EC30F03A0EF66E440EF76E74EC30F03A
:10CE8000010121D700011200D93D08D089EC30F012
:10CE9000840EF66E420EF76E74EC30F0D95308E152
:10CEA00089EC30F0960EF66E420EF76E74EC30F0B0
:10CEB000D9517F0808E189EC30F0A80EF66E420ED9
:10CEC000F76E74EC30F01200FEC015F10101025152
:10CED000010A006ED8900036005015130635006E1A
:10CEE0000036FC0E0016005015130835006E003693
:10CEF0000036F80E0016005015130A39006EF00EB9
:10CF0000001600501513000169A90ED0000ECBBE0B
:10CF1000010E010A006E003A0036E00E00160050C5
:10CF20000101151303D000010101159B159D159FEB
:10CF30001551000A0001D8B4BED0010AD8B4B6D148
:10CF4000030AD8B4BDD1010AD8B4C4D1070AD8B4F1
:10CF5000CBD1010AD8B4D2D1030AD8B4D9D1010AAD
:10CF6000D8B4E7D10F0AD8B4EED1010AD8B4F5D1BC
:10CF7000030AD8B4FCD1010AD8B403D2070AD8B442
:10CF80000AD2010AD8B411D2030AD8B418D2010ABD
:10CF9000D8B41FD21F0AD8B426D2010AD8B42DD2D1
:10CFA000030AD8B434D2010AD8B43BD2070AD8B4A1
:10CFB00042D2010AD8B449D2030AD8B450D2010AE5
:10CFC000D8B457D20F0AD8B45ED2010AD8B465D209
:10CFD000030AD8B46CD2010AD8B473D2070AD8B401
:10CFE0007AD2010AD8B481D2030AD8B488D2010A0D
:10CFF000D8B48FD23F0AD8B496D2010AD8B49DD201
:10D00000030AD8B4A4D2010AD8B4ABD2070AD8B460
:10D01000B2D2010AD8B4B9D2030AD8B4C0D2010A34
:10D02000D8B4C7D20F0AD8B4CED2010AD8B4D5D258
:10D03000030AD8B4DCD2010AD8B4E3D2070AD8B4C0
:10D04000EAD2010AD8B4F1D2030AD8B4F8D2010A5C
:10D05000D8B4FFD21F0AD8B406D3010AD8B40DD36E
:10D06000030AD8B415D3010AD8B41DD3070AD8B41B
:10D0700025D3010AD8B42DD3030AD8B435D3010A75
:10D08000D8B43DD30F0AD8B445D3010AD8B44DD390
:10D09000030AD8B455D3010AD8B45DD3070AD8B46B
:10D0A00065D3010AD8B46DD3030AD8B475D3010A85
:10D0B000D8B47DD387D3D93D51D068EC30F07C0E05
:10D0C000F66E3D0EF76E74EC30F089EC30F0AA513C
:10D0D000AE5D0101916F0001AB51AF590101926F3B
:10D0E0000001AC51B0590101936F0001AD51B1592C
:10D0F0000101946FD892196AD2BE198ED29EDE6F4A
:10D1000093C1DDF192C1DCF191C1DBF1E26BE16B26
:10D11000E06B0A0EDF6F00010CEC25F019BED28E19
:10D1200003C094F102C093F101C092F100C091F1EB
:10D130008E0EF66E3D0EF76E0D0E0101956F00011D
:10D14000A0EC34F0030EE96E94C198F193C197F10D
:10D1500092C196F191C195F146EC61F0D95351E13C
:10D1600068EC30F0A00EF66E3D0EF76E74EC30F009
:10D1700089EC30F0AA51AE5D0101916F0001AB5115
:10D18000AF590101926F0001AC51B0590101936F89
:10D190000001AD51B1590101946FD892196AD2BE04
:10D1A000198ED29EDE6F93C1DDF192C1DCF191C187
:10D1B000DBF1E26BE16BE06B0A0EDF6F00010CEC60
:10D1C00025F019BED28E03C094F102C093F101C0C4
:10D1D00092F100C091F1B20EF66E3D0EF76E0D0E9B
:10D1E0000101956F0001A0EC34F0030EE96E94C1CB
:10D1F00098F193C197F192C196F191C195F146ECE6
:10D2000061F0D9517F0851E168EC30F0C40EF66E40
:10D210003D0EF76E74EC30F089EC30F0AA51AE5D43
:10D220000101916F0001AB51AF590101926F0001F3
:10D23000AC51B0590101936F0001AD51B1590101D9
:10D24000946FD892196AD2BE198ED29EDE6F93C1A6
:10D25000DDF192C1DCF191C1DBF1E26BE16BE06BDE
:10D260000A0EDF6F00010CEC25F019BED28E03C050
:10D2700094F102C093F101C092F100C091F1D60E79
:10D28000F66E3D0EF76E0D0E0101956F0001A0ECDC
:10D2900034F0030EE96E94C198F193C197F192C1F5
:10D2A00096F191C195F146EC61F0A8D268EC30F0AE
:10D2B000E80EF66E3D0EF76E74EC30F0E5DD9ED2B2
:10D2C00068EC30F0FA0EF66E3D0EF76E74EC30F04E
:10D2D000DBDD94D268EC30F00C0EF66E3E0EF76E8D
:10D2E00074EC30F0D1DD8AD268EC30F01E0EF66EB0
:10D2F0003E0EF76E74EC30F0C7DD80D268EC30F093
:10D30000300EF66E3E0EF76E74EC30F0BDDD76D268
:10D3100068EC30F0420EF66E3E0EF76E74EC30F0B4
:10D3200089EC30F0540EF66E3E0EF76E74EC30F071
:10D3300065D268EC30F0660EF66E3E0EF76E74EC59
:10D3400030F0A2DD5BD268EC30F0780EF66E3E0E67
:10D35000F76E74EC30F098DD51D268EC30F08A0E44
:10D36000F66E3E0EF76E74EC30F08EDD47D268EC50
:10D3700030F09C0EF66E3E0EF76E74EC30F084DDED
:10D380003DD268EC30F0AE0EF66E3E0EF76E74ECE9
:10D3900030F07ADD33D268EC30F0C00EF66E3E0E1F
:10D3A000F76E74EC30F070DD29D268EC30F0D20EFC
:10D3B000F66E3E0EF76E74EC30F066DD1FD268EC50
:10D3C00030F0E40EF66E3E0EF76E74EC30F05CDD7D
:10D3D00015D268EC30F0F60EF66E3E0EF76E74EC79
:10D3E00030F052DD0BD268EC30F0080EF66E3F0ED6
:10D3F000F76E74EC30F048DD01D268EC30F01A0EB4
:10D40000F66E3F0EF76E74EC30F03EDDF7D168EC4F
:10D4100030F02C0EF66E3F0EF76E74EC30F034DD0B
:10D42000EDD168EC30F03E0EF66E3F0EF76E74EC08
:10D4300030F02ADDE3D168EC30F0500EF66E3F0E8E
:10D44000F76E74EC30F020DDD9D168EC30F0620E6C
:10D45000F66E3F0EF76E74EC30F016DDCFD168EC4F
:10D4600030F0740EF66E3F0EF76E74EC30F00CDD9B
:10D47000C5D168EC30F0860EF66E3F0EF76E74EC98
:10D4800030F002DDBBD168EC30F0980EF66E3F0E46
:10D49000F76E74EC30F0F8DCB1D168EC30F0AA0E25
:10D4A000F66E3F0EF76E74EC30F0EEDCA7D168EC50
:10D4B00030F0BC0EF66E3F0EF76E74EC30F0E4DC2C
:10D4C0009DD168EC30F0CE0EF66E3F0EF76E74EC28
:10D4D00030F0DADC93D168EC30F0E00EF66E3F0EFF
:10D4E000F76E74EC30F0D0DC89D168EC30F0F20EDD
:10D4F000F66E3F0EF76E74EC30F0C6DC7FD168EC50
:10D5000030F0040EF66E400EF76E74EC30F0BCDCBA
:10D5100075D168EC30F0160EF66E400EF76E74ECB6
:10D5200030F0B2DC6BD168EC30F0280EF66E400EB5
:10D53000F76E74EC30F0A8DC61D168EC30F03A0E94
:10D54000F66E400EF76E74EC30F09EDC57D168EC4E
:10D5500030F04C0EF66E400EF76E74EC30F094DC4A
:10D560004DD168EC30F05E0EF66E400EF76E74EC46
:10D5700030F08ADC43D168EC30F0700EF66E400E6D
:10D58000F76E74EC30F080DC39D168EC30F0820E4C
:10D59000F66E400EF76E74EC30F076DC2FD168EC4E
:10D5A00030F0940EF66E400EF76E74EC30F06CDCDA
:10D5B00025D168EC30F0A60EF66E400EF76E74ECD6
:10D5C00030F062DC1BD168EC30F0B80EF66E400E25
:10D5D000F76E74EC30F058DC11D168EC30F0CA0E04
:10D5E000F66E400EF76E74EC30F04EDC07D168EC4E
:10D5F00030F0DC0EF66E400EF76E74EC30F044DC6A
:10D60000FDD068EC30F0EE0EF66E400EF76E74EC66
:10D6100030F03ADCF3D068EC30F0000EF66E410EDC
:10D62000F76E74EC30F030DCE9D068EC30F0120EBC
:10D63000F66E410EF76E74EC30F026DCDFD068EC4D
:10D6400030F0240EF66E410EF76E74EC30F01CDCF8
:10D65000D5D068EC30F0360EF66E410EF76E74ECF5
:10D6600030F012DCCBD068EC30F0480EF66E410E94
:10D67000F76E74EC30F008DCC1D068EC30F05A0E74
:10D68000F66E410EF76E74EC30F044EC67F0B6D0F5
:10D6900068EC30F06C0EF66E410EF76E74EC30F004
:10D6A00044EC67F0ABD068EC30F07E0EF66E410EC5
:10D6B000F76E74EC30F044EC67F0A0D068EC30F01A
:10D6C000900EF66E410EF76E74EC30F044EC67F09D
:10D6D00095D068EC30F0A20EF66E410EF76E74EC49
:10D6E00030F044EC67F08AD068EC30F0AE0EF66EA5
:10D6F000410EF76E74EC30F044EC67F07FD068ECCC
:10D7000030F0C00EF66E410EF76E74EC30F044EC63
:10D7100067F074D068EC30F0D20EF66E410EF76E02
:10D7200074EC30F044EC67F069D068EC30F0E40E53
:10D73000F66E410EF76E74EC30F044EC67F05ED09C
:10D7400068EC30F0F60EF66E410EF76E74EC30F0C9
:10D7500044EC67F053D068EC30F0080EF66E420EE1
:10D76000F76E74EC30F044EC67F048D068EC30F0C1
:10D770001A0EF66E420EF76E74EC30F044EC67F061
:10D780003DD068EC30F02C0EF66E420EF76E74EC65
:10D7900030F044EC67F032D068EC30F03E0EF66EBC
:10D7A000420EF76E74EC30F044EC67F027D068EC72
:10D7B00030F04E0EF66E420EF76E74EC30F044EC24
:10D7C00067F01CD068EC30F0600EF66E420EF76E1B
:10D7D00074EC30F089EC30F015C192F1110E0101BA
:10D7E000936F0001D0EC34F0750EF66E420EF76EBA
:10D7F0000E0E0101956F0001A0EC34F01200010142
:10D80000168900011200CA51906FCBC091F0CCC0B4
:10D8100092F0CDC093F0D250006ED29E3901E16BF0
:10D820000F0EE06F600043F2E3F9E59DE59FE585AB
:10D83000550EE66FAA0EE66FE583E5B3FED7E595D4
:10D84000E59DE58F0050D212D250006ED29EE16B62
:10D85000100EE06F600047F2E3F9E59DE59FE58576
:10D86000550EE66FAA0EE66FE583E5B3FED7E595A4
:10D87000E59DE58F0050D212D250006ED29EE16B32
:10D88000110EE06F60004BF2E3F9E59DE59FE58541
:10D89000550EE66FAA0EE66FE583E5B3FED7E59574
:10D8A000E59DE58F0050D212D250006ED29EE16B02
:10D8B000120EE06F60004FF2E3F9E59DE59FE5850C
:10D8C000550EE66FAA0EE66FE583E5B3FED7E59544
:10D8D000E59DE58F0050D212000187EF7DF0390100
:10D8E000E58FE59DF86AD29A078E0E01550E3A0132
:10D8F000BF6FAA0EBF6FBF910B0EE56F080EE86FEA
:10D90000130E096F160E1E6F550EBF6FAA0EBF6F56
:10D91000BF813901DE6BDB6BDD6B050EDF6F600EE7
:10D92000D96F1A6A3D01F39FC392BB82300EF26F2A
:10D93000F66B330EF56FF46BF38FDB9FC59CBD8CDC
:10D94000340EDA6FDE6B330EDD6FDC6BDB8FC39C66
:10D95000BB8C0001626B616B646B636B6991699353
:10D9600001017F937F957F97816B8C6B8B6B3A0165
:10D97000406B506B606B706B806B3E01BD6BBE6B20
:10D98000BF6BBC6BB96BBA6BBB6BB86B330E1B6EEA
:10D990002E0E1C6E310E1D6E2E0E1E6E300E1F6E64
:10D9A000206A0101846B856B3F0EC26EB90EC36E97
:10D9B000800EC46E700EC56EC690C692C694C686A2
:10D9C000800E3A01616F300E716F000E3E01FD6FE7
:10D9D0003A01406F506F606F706F806F3E01BD6B9A
:10D9E000070EBE6FBF6FBC6BB96BBA6FBB6FB86B06
:10D9F000BD9EBB94B8A802D0CF0EB76E2C0EB66EEB
:10DA0000900EB86E450EB96E010EB56E370EB26E41
:10DA1000B36AB46A3C0EB16EB00EB06E0000010E77
:10DA20009D6E070E9A6E9B6A9C6A630E996EC00E7D
:10DA3000986E0000010EA96E370EA66EA76AA86A3E
:10DA40003C0EA56EB00EA46E00000101196B186BA0
:10DA5000179BBE90BE92BE94BA9EBC96BC94BC92DC
:10DA6000BC9016971699169B169D0001F49F010114
:10DA7000169116931695000167EF2DF0010117938B
:10DA80001795000166EC2EF06CEC2EF088936F0079
:10DA900048FF91F1D29E3901E16B300EE06FE59DB8
:10DAA000E59FE581E351E59DE58F010191BFD28EB0
:10DAB0000001F56F6F0048FF91F1D29E3901E16BD3
:10DAC0003C0EE06FE59DE59FE581E351E59DE58F27
:10DAD000010191BFD28E0001D96F6F0048FF91F113
:10DAE000D29E3901E16B140EE06FE59DE59FE58163
:10DAF000E351E59DE58F010191BFD28E016E0001DA
:10DB0000889901B088896F0048FF91F1D29E390150
:10DB1000E16B320EE06FE59DE59FE581E351E59D08
:10DB2000E58F010191BFD28E0001FB6F6F0048FFAE
:10DB300091F1D29E3901E16B330EE06FE59DE59FD7
:10DB4000E581E351E59DE58F010191BFD28E000192
:10DB5000FD6FFF0EFD1B6F0048FF91F1D29E390152
:10DB6000E16B2F0EE06FE59DE59FE581E351E59DBB
:10DB7000E58F010191BFD28E0001F16F6F0048FF68
:10DB800091F1D29E3901E16B380EE06FE59DE59F82
:10DB9000E581E351E59DE58F010191BFD28E000142
:10DBA000F26F6F0048FF91F1D29E3901E16B310EA7
:10DBB000E06FE59DE59FE581E351E59DE58F01017E
:10DBC00091BFD28E0001EF6F6F0048FF91F1D29E9E
:10DBD0003901E16B2D0EE06FE59DE59FE581E35195
:10DBE000E59DE58F010191BFD28E0001F06F6F00BE
:10DBF00048FF91F1D29E3901E16B050EE06FE59D82
:10DC0000E59FE581E351E59DE58F010191BFD28E4E
:10DC10000001CE6FCE515A0802E2050ECE6F6F00A2
:10DC200048FF91F1D29E3901E16B3D0EE06FE59D19
:10DC3000E59FE581E351E59DE58F010191BFD28E1E
:10DC40000001E26F0101936BE2C092F1020E956F49
:10DC5000580E946F00019FEC2EF0E66BE56B02C04E
:10DC6000E4F001C0E3F0D66BCEC0D5F06F0048FF02
:10DC700091F1D29E3901E16B3A0EE06FE59DE59F8F
:10DC8000E581E351E59DE58F010191BFD28E926F51
:10DC90006F0048FF93F1D29E3901E16B390EE06FBE
:10DCA000E59DE59FE581E351E59DE58F010193BF8A
:10DCB000D28E946F92C1C9F094C1C8F00001C83DE2
:10DCC00006D0C93D04D0010EC96F2C0EC86F6F007D
:10DCD00048FF91F1D29E3901E16B070EE06FE59D9F
:10DCE000E59FE581E351E59DE58F010191BFD28E6E
:10DCF000926F6F0048FF93F1D29E3901E16B060EDF
:10DD0000E06FE59DE59FE581E351E59DE58F01012C
:10DD100093BFD28E946F92C1B7F094C1B6F06F00EA
:10DD200048FF91F1D29E3901E16B290EE06FE59D2C
:10DD3000E59FE581E351E59DE58F010191BFD28E1D
:10DD4000926F6F0048FF93F1D29E3901E16B280E6C
:10DD5000E06FE59DE59FE581E351E59DE58F0101DC
:10DD600093BFD28E946F92C1B9F094C1B8F06F0096
:10DD700048FF91F1D29E3901E16B090EE06FE59DFC
:10DD8000E59FE581E351E59DE58F010191BFD28ECD
:10DD9000926F6F0048FF93F1D29E3901E16B080E3C
:10DDA000E06FE59DE59FE581E351E59DE58F01018C
:10DDB00093BFD28E946F92C1BBF094C1BAF06F0042
:10DDC00048FF91F1D29E3901E16B150EE06FE59DA0
:10DDD000E59FE581E351E59DE58F010191BFD28E7D
:10DDE0000001E86F6F0048FF91F1D29E3901E16BAD
:10DDF000010EE06FE59DE59FE581E351E59DE58F2F
:10DE0000010191BFD28E806F6F0048FF91F1D29EC9
:10DE10003901E16B370EE06FE59DE59FE581E35148
:10DE2000E59DE58F010191BFD28E0001F66FF76B82
:10DE30006F0048FF91F1D29E3901E16B0D0EE06F4A
:10DE4000E59DE59FE581E351E59DE58F010191BFEA
:10DE5000D28E0001F76F0101926BF7C091F10001C2
:10DE60001AEC30F002C0DBF001C0DAF0F86B6F00A2
:10DE700048FF91F1D29E3901E16B0B0EE06FE59DF9
:10DE8000E59FE581E351E59DE58F010191BFD28ECC
:10DE90000001F86F0101926BF8C091F100011AECDA
:10DEA00030F002C0DDF001C0DCF0889B686B6F00D1
:10DEB00048FF91F1D29E3901E16B0C0EE06FE59DB8
:10DEC000E59FE581E351E59DE58F010191BFD28E8C
:10DED0000001ED6FC492BC9268EC30F0D20EF66E89
:10DEE000540EF76E74EC30F089EC30F0E40EF66E00
:10DEF000540EF76E74EC30F001018E6B8D6B8E5109
:10DF0000130818E303E18D51870814E3CBAE05D065
:10DF10000001698901010ED003D000016999010156
:10DF2000010ECE6F000105EC2EF001018D2BD8B44F
:10DF30008E2BE5D7000166EC2EF06CEC2EF0010183
:10DF4000906B8F6B905359E18F51630856E300013A
:10DF500069A929D0EDC091F196EC30F0D9517F0834
:10DF600011E168EC30F0F60EF66E540EF76E74ECBC
:10DF700030F089EC30F0080EF66E550EF76E74EC4A
:10DF800030F010D068EC30F01A0EF66E550EF76EC9
:10DF900074EC30F089EC30F02C0EF66E550EF76E06
:10DFA00074EC30F025D06999D9517F0811E168EC03
:10DFB00030F03E0EF66E550EF76E74EC30F089ECD4
:10DFC00030F0500EF66E550EF76E74EC30F010D047
:10DFD00068EC30F0620EF66E550EF76E74EC30F0B1
:10DFE00089EC30F0740EF66E550EF76E74EC30F06E
:10DFF00001018F2BD8B4902BA5D700016997DF6B57
:10E00000E06B956B88858897896B8A6BDC51BA25A4
:10E01000C06FDD51BB21C16FDA51B65DBC6FDB5102
:10E02000B759BD6FDA51B85DBE6FDB51B959BF6FDB
:10E03000889DD76B8C6B8D6B8B6BD86B0101126BD2
:10E040000001E16BF493FC6B699B9551020802E1BE
:10E05000EBEC5CF0010116971699020E916FFA0E27
:10E06000CE6F000105EC2EF00101912FF8D7169725
:10E0700016990001F499F49BF49D0101169F00018B
:10E08000F4910101178717990001889501011A6B16
:10E09000179D816B179F7F910001656B699166ECFD
:10E0A0002EF0C00ED212D9517F0811E168EC30F089
:10E0B000860EF66E550EF76E74EC30F089EC30F08B
:10E0C000980EF66E550EF76E74EC30F023D0D953DF
:10E0D00011E168EC30F0AA0EF66E550EF76E74EC96
:10E0E00030F089EC30F0BC0EF66E550EF76E74EC25
:10E0F00030F010D068EC30F0CE0EF66E550EF76EA4
:10E1000074EC30F089EC30F0E00EF66E550EF76EE0
:10E1100074EC30F06B6B6A6B6D6B6C6B6F6B6E6B72
:10E12000040E0101AC6FAE6B140EAD6F030EAF6F3A
:10E13000B16B6A0EB06F000122EC31F001524CE07D
:10E1400001017F8500016BC070F06AC071F06DC085
:10E1500072F06CC073F06FC074F06EC075F089EC33
:10E1600030F0F20EF66E550EF76E030E0101956F4C
:10E170000001A0EC34F070C091F1370E0101926FF4
:10E180000001B0EC5DF071C091F1370E0101926FAA
:10E190000001B0EC5DF072C091F1370E0101926F99
:10E1A0000001B0EC5DF073C091F1370E0101926F88
:10E1B0000001B0EC5DF074C091F1370E0101926F77
:10E1C0000001B0EC5DF075C091F1370E0101926F66
:10E1D0000001B0EC5DF008D089EC30F00E0EF66E68
:10E1E000560EF76E74EC30F001018053D8A4C6D0FF
:10E1F00000016B6B6A6B6D6B6C6B6F6B6E6B050EFE
:10E200000101AC6FAE6B140EAD6F030EAF6FB16B4F
:10E210006A0EB06F000122EC31F001524CE00101B6
:10E220007F8700016BC070F06AC071F06DC072F042
:10E230006CC073F06FC074F06EC075F068EC30F0B5
:10E24000200EF66E560EF76E030E0101956F00015B
:10E25000A0EC34F070C091F1370E0101926F000113
:10E26000B0EC5DF071C091F1370E0101926F0001C9
:10E27000B0EC5DF072C091F1370E0101926F0001B8
:10E28000B0EC5DF073C091F1370E0101926F0001A7
:10E29000B0EC5DF074C091F1370E0101926F000196
:10E2A000B0EC5DF075C091F1370E0101926F000185
:10E2B000B0EC5DF008D068EC30F03C0EF66E560E17
:10E2C000F76E74EC30F0080E0101916FFA0ECE6F0C
:10E2D000000105EC2EF00101912FF8D700016B6BC6
:10E2E0006A6B010E0101AC6F030EAE6FE80EAD6FED
:10E2F000010EAF6FB16B6A0EB06F000122EC31F00E
:10E30000015214E001017F83000168EC30F04E0EF1
:10E31000F66E560EF76E74EC30F089EC30F0600E4D
:10E32000F66E560EF76E74EC30F010D068EC30F0EC
:10E33000720EF66E560EF76E74EC30F089EC30F01B
:10E34000840EF66E560EF76E74EC30F0040E01017A
:10E35000916FFA0ECE6F000105EC2EF00101912FA6
:10E36000F8D70001CBEC32F0140E0101CE6F0001A2
:10E3700005EC2EF0B4EC33F00CD00101040E916FDB
:10E38000FA0ECE6F000105EC2EF00101912FF8D7A7
:10E390000001C00ED21239019685938F9481988D19
:10E3A000968DBD9E0001699168EC5EF00DEC60F009
:10E3B000AAEC5EF0879F0101065311E00001FB3DCE
:10E3C00003D001010CD00001F4A502D0010107D057
:10E3D000FC2BFC51FB5D01E2F483F485010100019B
:10E3E00088A702D0F493FC6B88A501D0F495CBBE2E
:10E3F00075D069A973D0F499F49B6F0048FF91F12F
:10E40000D29E3901E16B070EE06FE59DE59FE58146
:10E41000E351E59DE58F010191BFD28E926F6F00B0
:10E4200048FF93F1D29E3901E16B060EE06FE59D46
:10E43000E59FE581E351E59DE58F010193BFD28E14
:10E44000946F92C1B7F094C1B6F06F0048FF91F19C
:10E45000D29E3901E16B090EE06FE59DE59FE581F4
:10E46000E351E59DE58F010191BFD28E926F6F0060
:10E4700048FF93F1D29E3901E16B080EE06FE59DF4
:10E48000E59FE581E351E59DE58F010193BFD28EC4
:10E49000946F92C1BBF094C1BAF0926BF7C091F146
:10E4A00000011AEC30F002C0DBF001C0DAF0DA5102
:10E4B000B65DBC6FDB51B759BD6F0101926BF8C0FF
:10E4C00091F100011AEC30F002C0DDF001C0DCF087
:10E4D000DC51BA25C06FDD51BB21C16FF4AB74D0E4
:10E4E000EF5372E1F49B6F0048FF91F1D29E390126
:10E4F000E16B070EE06FE59DE59FE581E351E59D4A
:10E50000E58F010191BFD28E926F6F0048FF93F1AA
:10E51000D29E3901E16B060EE06FE59DE59FE58136
:10E52000E351E59DE58F010193BFD28E946F92C1B7
:10E53000B7F094C1B6F06F0048FF91F1D29E390157
:10E54000E16B090EE06FE59DE59FE581E351E59DF7
:10E55000E58F010191BFD28E926F6F0048FF93F15A
:10E56000D29E3901E16B080EE06FE59DE59FE581E4
:10E57000E351E59DE58F010193BFD28E946F92C167
:10E58000BBF094C1BAF0926BF7C091F100011AECA4
:10E5900030F002C0DBF001C0DAF0DA51B65DBC6FDA
:10E5A000DB51B759BD6F0101926BF8C091F10001C9
:10E5B0001AEC30F002C0DDF001C0DCF0DC51BA250D
:10E5C000C06FDD51BB21C16FF4BD31D0010116A96F
:10E5D00002D000012CD00001F4A929D0EF5327E18B
:10E5E000F499B9C0B7F0B8C0B6F00101926BF7C0AA
:10E5F00091F100011AEC30F002C0DBF001C0DAF05A
:10E60000DA51B65DBC6FDB51B759BD6F0101926B3A
:10E61000F8C091F100011AEC30F002C0DDF001C049
:10E62000DCF0DC51BA25C06FDD51BB21C16F88A57C
:10E6300001D0F49DEF3D02D0F499F49BAAEC5EF07A
:10E6400088A70AD088B508D0010116A702D000011A
:10E6500003D0045315E1000188A7B8EF76F088B520
:10E66000B8EF76F0010116A702D0000181D3005364
:10E67000D8B402D000017CD30001F53D79D301016B
:10E68000005308E10001F53D01D002D0010102D0A4
:10E690000DD001010253D8A402D0000107D0CBBE97
:10E6A00052D1000169B902D001014DD18E6BF53D07
:10E6B0000DD00101966B956B946B936B9A6B996B74
:10E6C000986B020E976F0001B9EC30F0B2530BE17A
:10E6D000B35309E1B45307E1B55305E139015B5187
:10E6E00004000001F3D701010453D8B49ED0000107
:10E6F000F48F010116910001F4AF03D001011681DE
:10E700000001F15305E1F25303E1CBBE01D0698B67
:10E71000FD3D01D0FD6BFD510A0DF3500101916FDC
:10E72000966B956B946B936B9A6B996B986B976FD9
:10E730000001B9EC30F0B2536EE1B3536CE1B45365
:10E740006AE1B55368E1D93D20D068EC30F0960E0F
:10E75000F66E560EF76E74EC30F089EC30F0A80EC1
:10E76000F66E560EF76E070E0101956F0001A0ECD4
:10E7700034F0090EE96ECDC098F1CCC097F1CBC052
:10E7800096F1CAC095F146EC61F0D95320E168ECEE
:10E7900030F0B40EF66E560EF76E74EC30F089EC75
:10E7A00030F0C60EF66E560EF76E070E0101956F2D
:10E7B0000001A0EC34F0090EE96ECDC098F1CCC098
:10E7C00097F1CBC096F1CAC095F146EC61F0D951F2
:10E7D0007F0820E168EC30F0D20EF66E560EF76E30
:10E7E00074EC30F089EC30F0E40EF66E560EF76EF5
:10E7F000070E0101956F0001A0EC34F0090EE96EDF
:10E80000CDC098F1CCC097F1CBC096F1CAC095F1BC
:10E8100046EC61F090D7B4EC61F0F4A703D00101AD
:10E82000168B000169978DD001010001FD3D01D0DB
:10E83000FD6BFD510A0DF3500101916F966B956BC5
:10E84000946B936B9A6B996B986B976F0001B9EC13
:10E8500030F0B2536EE1B3536CE1B4536AE1B55397
:10E8600068E1D93D20D068EC30F0F00EF66E560E1F
:10E87000F76E74EC30F089EC30F0020EF66E570E45
:10E88000F76E070E0101956F0001A0EC34F0090E40
:10E89000E96ECDC098F1CCC097F1CBC096F1CAC05B
:10E8A00095F146EC61F0D95320E168EC30F00E0EA2
:10E8B000F66E570EF76E74EC30F089EC30F0200EE7
:10E8C000F66E570EF76E070E0101956F0001A0EC72
:10E8D00034F0090EE96ECDC098F1CCC097F1CBC0F1
:10E8E00096F1CAC095F146EC61F0D9517F0820E15C
:10E8F00068EC30F02C0EF66E570EF76E74EC30F0BC
:10E9000089EC30F03E0EF66E570EF76E070E0101E1
:10E91000956F0001A0EC34F0090EE96ECDC098F1BE
:10E92000CCC097F1CBC096F1CAC095F146EC61F02E
:10E9300090D7B4EC61F0F4A703D00101168B00016D
:10E9400069978E6B01010053D8B413D20001F53DD5
:10E9500001D002D001010DD2F053D8A409D2F49F06
:10E96000E15310E10101966B956B946B936BE6C0DC
:10E970009AF1E5C099F1E4C098F1E3C097F1000184
:10E98000B9EC30F0B253D8A4C1D1B353D8A4BED19E
:10E99000B453D8A4BBD1B553D8A4B8D1CFEC5EF052
:10E9A000FE5309E10101105303E00001F55303E0B8
:10E9B0000001952D02D00DEC60F09551020802E1A6
:10E9C000EBEC5CF095510308D8B45CEC62F0952D4B
:10E9D00001D03FD1D93D68D068EC30F0AA51AE5D8E
:10E9E0000101916F0001AB51AF590101926F00011C
:10E9F000AC51B0590101936F0001AD51B159010102
:10EA0000946FD892196AD2BE198ED29EDE6F93C1CE
:10EA1000DDF192C1DCF191C1DBF1E26BE16B020E41
:10EA2000E06F580EDF6F00010CEC25F019BED28E9E
:10EA300003C094F102C093F101C092F100C091F1C2
:10EA4000010E01019127000E9223932394234A0E75
:10EA5000F66E570EF76E0D0E956F0001A0EC34F0B8
:10EA6000030EE96E94C198F193C197F192C196F1AA
:10EA700091C195F146EC61F089EC30F05C0EF66ED8
:10EA8000570EF76E070E0101956F0001A0EC34F0F0
:10EA9000090EE96ECDC098F1CCC097F1CBC096F1CC
:10EAA000CAC095F146EC61F0D95368E168EC30F0EA
:10EAB000AA51AE5D0101916F0001AB51AF59010147
:10EAC000926F0001AC51B0590101936F0001AD513B
:10EAD000B1590101946FD892196AD2BE198ED29E93
:10EAE000DE6F93C1DDF192C1DCF191C1DBF1E26B2C
:10EAF000E16B020EE06F580EDF6F00010CEC25F0A9
:10EB000019BED28E03C094F102C093F101C092F1FC
:10EB100000C091F1010E01019127000E9223932371
:10EB20009423680EF66E570EF76E0D0E956F00016A
:10EB3000A0EC34F0030EE96E94C198F193C197F103
:10EB400092C196F191C195F146EC61F089EC30F0FB
:10EB50007A0EF66E570EF76E070E0101956F0001E3
:10EB6000A0EC34F0090EE96ECDC098F1CCC097F15D
:10EB7000CBC096F1CAC095F146EC61F0D9517F083F
:10EB800068E168EC30F0AA51AE5D0101916F0001BF
:10EB9000AB51AF590101926F0001AC51B059010165
:10EBA000936F0001AD51B1590101946FD892196A68
:10EBB000D2BE198ED29EDE6F93C1DDF192C1DCF11F
:10EBC00091C1DBF1E26BE16B020EE06F580EDF6F7B
:10EBD00000010CEC25F019BED28E03C094F102C0E6
:10EBE00093F101C092F100C091F1010E0101912752
:10EBF000000E922393239423860EF66E570EF76E23
:10EC00000D0E956F0001A0EC34F0030EE96E94C177
:10EC100098F193C197F192C196F191C195F146ECAB
:10EC200061F089EC30F0980EF66E570EF76E070E15
:10EC30000101956F0001A0EC34F0090EE96ECDC022
:10EC400098F1CCC097F1CBC096F1CAC095F146ECD3
:10EC500061F00101005308E10001F53D01D002D04F
:10EC6000010102D00DD001010253D8A402D000014D
:10EC700007D0CBBE45D0000169B902D0010140D018
:10EC80000101178900018E6B0101966B956B946BE6
:10EC9000936B9A6B996B986B020E976F0001B9ECAE
:10ECA00030F0B2530BE1B35309E1B45307E1B5536C
:10ECB00005E139015B5104000001F3D70101005364
:10ECC00014E00001F53D01D002D001010ED0010198
:10ECD000045307E00001B4EC61F0F4A703D0010194
:10ECE000168B000169970AD001010001B4EC61F0B4
:10ECF000F4A703D00101168B000169978E6B010107
:10ED0000010E0001E16F68EC5EF03CD6E12D30D0E1
:10ED1000F48F0101966B956B946B936B9A6B996B67
:10ED2000986B020E976F0001B9EC30F0B2530BE113
:10ED3000B35309E1B45307E1B55305E139015B5120
:10ED400004000001F3D70101045303E00001B4EC17
:10ED500061F00001F4A703D00101168B000101014D
:10ED600017B902D0168B01D01799000169978E6BE5
:10ED70000101000162EC66F088B759D088B557D020
:10ED8000010116A702D0000152D016B902D000012D
:10ED90004ED0005308E10001F53D01D002D0010141
:10EDA00002D01ED001010253D8A402D0000118D015
:10EDB000CBBE04D0000169B913D001010853D8B407
:10EDC00002D000010DD00A53D8B402D0000108D0FF
:10EDD00006532EE00001F03D01D002D0010128D001
:10EDE0000101169B169D16971699966B956B946B61
:10EDF000936B9A6B996B986B0A0E976F0001B9EC45
:10EE000030F0B2530BE1B35309E1B45307E1B5530A
:10EE100005E139015B5104000001F3D78E6BB4ECBE
:10EE200061F0F4A703D00101168B0001699701017D
:10EE3000000188B70ED088B50CD0010116A702D00A
:10EE4000000107D016A902D0000103D0045313E13A
:10EE5000000188B730D088B52ED0010116A702D0A6
:10EE6000000129D016A902D0000125D00053D8B442
:10EE700002D0000120D0005308E10001F53D01D08F
:10EE800002D0010102D00DD001010253D8A402D05A
:10EE9000000107D0CBBE10D0000169B902D001013A
:10EEA0000BD0B4EC61F0F4A703D00101168B000184
:10EEB000F48F69978E6B010100010DEC60F087996A
:10EEC000010116B955D20001E83D6BD188A569D181
:10EED000AD6BAC6BAB6BAA6BDE6BB56BB46BB36B32
:10EEE000B26BD6C093F1D5C092F10101956B0A0EB9
:10EEF000946F00019FEC2EF002C092F101C091F1DD
:10EF00000101966B956B946B936B9A6B996B02C036
:10EF100098F101C097F10001B9EC30F0F49DB253C3
:10EF2000D8A42AD1B353D8A427D1B453D8A424D178
:10EF3000B553D8A421D10DEC60F0AAEC5EF0F553E6
:10EF4000D8B462EC66F039015B510400010116A9E6
:10EF500003D0000111D101010001CFEC5EF0955109
:10EF6000020829E1EBEC5CF0AD6BAC6BAB6BAA6B10
:10EF7000DE6BB56BB46BB36BB26BD6C093F1D5C01F
:10EF800092F10101956B0A0E946F00019FEC2EF037
:10EF900002C092F101C091F10101966B956B946BE7
:10EFA000936B9A6B996B02C098F101C097F10001C5
:10EFB000B9EC30F0D4D7952D01D003D09551070886
:10EFC00041E169A93BD089EC30F0A40EF66E570EF2
:10EFD000F76E030E0101956F0001A0EC34F096C0AE
:10EFE000A1F130EC2EF097C0A1F130EC2EF098C0DA
:10EFF000A1F130EC2EF099C0A1F130EC2EF09AC0C6
:10F00000A1F130EC2EF09BC0A1F130EC2EF09CC0B1
:10F01000A1F130EC2EF09DC0A1F130EC2EF0B70E36
:10F02000F66E570EF76E040E0101956F0001A0EC0D
:10F0300034F09EC0A1F130EC2EF002D0D6EC5FF09F
:10F0400073EC5EF00101005323E00001F53D01D0B7
:10F0500002D001011DD0F4B302D0010119D068EC37
:10F0600030F0BE0EF66E570EF76E74EC30F089EC91
:10F0700030F0CC0EF66E570EF76E74EC30F00101E6
:10F0800016971699169B169D0001FC6BDBD70101A4
:10F090000001F493952D01D007D09551070804E0A5
:10F0A00064EC67F05CEC62F00101005308E10001E0
:10F0B000F53D01D002D0010102D02FD00101025351
:10F0C000D8A402D0000129D00853D8B402D000013E
:10F0D00024D00A53D8B402D000011FD0065307E051
:10F0E0000001F03D01D002D0010101D016D0000195
:10F0F000FE5313E10101105303E00001F5530DE04D
:10F10000000187B90AD09551040807E09551070816
:10F1100004E0CBBE25D069A923D0010ECE5D01014C
:10F12000216F226BD6C093F1D5C092F1956B0A0E78
:10F13000946F00019FEC2EF002C092F101C091F19A
:10F140000101966B956B946B936B9A6B996B02C0F4
:10F1500098F101C097F10001B9EC30F0879907D020
:10F160000101005305E1226B216B000105D0010173
:10F17000000168EC5EF0D3D669978E6B8893FFEC44
:10F180006BF00101169B168D966B956B946B936BD0
:10F190009A6B996B986B976B0001B9EC30F0878D87
:10F1A000E16BE853D8A4E3D088A5E1D0010116B9FA
:10F1B000D2D00001F49DF553D8B462EC66F00101A1
:10F1C000005323E00001F53D01D002D001011DD024
:10F1D000F4B302D0010119D068EC30F0DE0EF66E07
:10F1E000570EF76E74EC30F089EC30F0EC0EF66EE2
:10F1F000570EF76E74EC30F0010116971699169BB6
:10F20000169D0001FC6BDBD701010001F4939551C1
:10F21000020803E09551050855E19551020802E105
:10F22000EBEC5CF0955105084CE10101005308E15D
:10F230000001F53D01D002D0010102D02AD0010128
:10F240000853D8B402D0000124D00A53D8B402D055
:10F2500000011FD0065307E00001F03D01D002D0AD
:10F26000010101D016D00001FE5313E1010110533A
:10F2700003E00001F5530DE0000187B90AD0955174
:10F28000040807E09551070804E0CBBE05D069A942
:10F2900003D064EC67F015D001010253D8B45BD001
:10F2A000000168EC30F0FE0EF66E570EF76E74EC4F
:10F2B00030F089EC30F0100EF66E580EF76E74ECEC
:10F2C00030F043D0CFEC5EF069A93BD089EC30F050
:10F2D000220EF66E580EF76E030E0101956F0001B7
:10F2E000A0EC34F096C0A1F130EC2EF097C0A1F163
:10F2F00030EC2EF098C0A1F130EC2EF099C0A1F1C5
:10F3000030EC2EF09AC0A1F130EC2EF09BC0A1F1B0
:10F3100030EC2EF09CC0A1F130EC2EF09DC0A1F19C
:10F3200030EC2EF0350EF66E580EF76E040E01011D
:10F33000956F0001A0EC34F09EC0A1F130EC2EF0EE
:10F3400002D0D6EC5FF073EC5EF00DEC60F0AAEC4E
:10F350005EF02CD701010001FFEC6BF00101169B60
:10F36000168D000169978E6B8893878DE16B010183
:10F370000001CFEC5EF0010116A702D016AB04D05D
:10F3800016A97CD016BB7AD00001952D3FD069A973
:10F390003BD089EC30F03C0EF66E580EF76E030E43
:10F3A0000101956F0001A0EC34F096C0A1F130ECA2
:10F3B0002EF097C0A1F130EC2EF098C0A1F130EC06
:10F3C0002EF099C0A1F130EC2EF09AC0A1F130ECF2
:10F3D0002EF09BC0A1F130EC2EF09CC0A1F130ECDE
:10F3E0002EF09DC0A1F130EC2EF04F0EF66E580EAF
:10F3F000F76E040E0101956F0001A0EC34F09EC081
:10F40000A1F130EC2EF002D0D6EC5FF0952D01D0BA
:10F4100034D0D9517F0819E189EC30F0560EF66EE0
:10F42000580EF76E070E0101956F0001A0EC34F045
:10F43000090EE96ECDC098F1CCC097F1CBC096F122
:10F44000CAC095F146EC61F018D089EC30F0620E3C
:10F45000F66E580EF76E070E0101956F0001A0ECD5
:10F4600034F0090EE96ECDC098F1CCC097F1CBC055
:10F4700096F1CAC095F146EC61F00101000188A740
:10F48000B4D0010116A702D00001AFD00001F49F53
:10F49000952D41D069A93BD089EC30F06E0EF66E07
:10F4A000580EF76E030E0101956F0001A0EC34F0C9
:10F4B00096C0A1F130EC2EF097C0A1F130EC2EF007
:10F4C00098C0A1F130EC2EF099C0A1F130EC2EF0F3
:10F4D0009AC0A1F130EC2EF09BC0A1F130EC2EF0DF
:10F4E0009CC0A1F130EC2EF09DC0A1F130EC2EF0CB
:10F4F000810EF66E580EF76E040E0101956F000135
:10F50000A0EC34F09EC0A1F130EC2EF002D0D6EC8D
:10F510005FF073EC5EF0952D01D067D0D93D20D01F
:10F5200068EC30F0880EF66E580EF76E74EC30F022
:10F5300089EC30F09A0EF66E580EF76E070E010148
:10F54000956F0001A0EC34F0090EE96ECDC098F182
:10F55000CCC097F1CBC096F1CAC095F146EC61F0F2
:10F56000D95320E168EC30F0A60EF66E580EF76E17
:10F5700074EC30F089EC30F0B80EF66E580EF76E81
:10F58000070E0101956F0001A0EC34F0090EE96E41
:10F59000CDC098F1CCC097F1CBC096F1CAC095F11F
:10F5A00046EC61F0D9517F0820E168EC30F0C40EE0
:10F5B000F66E580EF76E74EC30F089EC30F0D60E23
:10F5C000F66E580EF76E070E0101956F0001A0EC64
:10F5D00034F0090EE96ECDC098F1CCC097F1CBC0E4
:10F5E00096F1CAC095F146EC61F0010116B9B9D0A7
:10F5F00016B7B7D0000188A702D00101B2D088A504
:10F6000002D00101AED0952D41D069A93BD089EC43
:10F6100030F0E20EF66E580EF76E030E0101956F94
:10F620000001A0EC34F096C0A1F130EC2EF097C0B0
:10F63000A1F130EC2EF098C0A1F130EC2EF099C081
:10F64000A1F130EC2EF09AC0A1F130EC2EF09BC06D
:10F65000A1F130EC2EF09CC0A1F130EC2EF09DC059
:10F66000A1F130EC2EF0F50EF66E580EF76E040E8A
:10F670000101956F0001A0EC34F09EC0A1F130ECC7
:10F680002EF002D0D6EC5FF073EC5EF0952D01D039
:10F6900067D0D93D20D068EC30F0FC0EF66E580EE5
:10F6A000F76E74EC30F089EC30F00E0EF66E590EF9
:10F6B000F76E070E0101956F0001A0EC34F0090E02
:10F6C000E96ECDC098F1CCC097F1CBC096F1CAC01D
:10F6D00095F146EC61F0D95320E168EC30F01A0E58
:10F6E000F66E590EF76E74EC30F089EC30F02C0E9B
:10F6F000F66E590EF76E070E0101956F0001A0EC32
:10F7000034F0090EE96ECDC098F1CCC097F1CBC0B2
:10F7100096F1CAC095F146EC61F0D9517F0820E11D
:10F7200068EC30F0380EF66E590EF76E74EC30F06F
:10F7300089EC30F04A0EF66E590EF76E070E010195
:10F74000956F0001A0EC34F0090EE96ECDC098F180
:10F75000CCC097F1CBC096F1CAC095F146EC61F0F0
:10F7600001010001CFEC5EF0010116A79BD0000162
:10F77000952D41D069A93BD089EC30F0560EF66E3C
:10F78000590EF76E030E0101956F0001A0EC34F0E5
:10F7900096C0A1F130EC2EF097C0A1F130EC2EF024
:10F7A00098C0A1F130EC2EF099C0A1F130EC2EF010
:10F7B0009AC0A1F130EC2EF09BC0A1F130EC2EF0FC
:10F7C0009CC0A1F130EC2EF09DC0A1F130EC2EF0E8
:10F7D000690EF66E590EF76E040E0101956F000169
:10F7E000A0EC34F09EC0A1F130EC2EF002D0D6ECAB
:10F7F0005FF073EC5EF0952D01D01FD0D93D08D09D
:10F8000068EC30F0700EF66E590EF76E74EC30F056
:10F81000D95308E168EC30F0820EF66E590EF76E9F
:10F8200074EC30F0D9517F0808E168EC30F0940EA8
:10F83000F66E590EF76E74EC30F0BDAF03D0C3AF67
:10F840000AD002D0C3BF2DD0BD51C35D2AE303E16E
:10F85000C251BC5D26E2952D02D073EC5EF0952D71
:10F8600001D01FD0D93D08D089EC30F0A60EF66E3D
:10F87000590EF76E74EC30F0D95308E189EC30F092
:10F88000B80EF66E590EF76E74EC30F0D9517F0851
:10F8900008E189EC30F0CA0EF66E590EF76E74EC82
:10F8A00030F0010116A99ED00001952D41D069A923
:10F8B0003BD089EC30F0DC0EF66E590EF76E030E7D
:10F8C0000101956F0001A0EC34F096C0A1F130EC7D
:10F8D0002EF097C0A1F130EC2EF098C0A1F130ECE1
:10F8E0002EF099C0A1F130EC2EF09AC0A1F130ECCD
:10F8F0002EF09BC0A1F130EC2EF09CC0A1F130ECB9
:10F900002EF09DC0A1F130EC2EF0EF0EF66E590EE8
:10F91000F76E040E0101956F0001A0EC34F09EC05B
:10F92000A1F130EC2EF002D0D6EC5FF073EC5EF07B
:10F93000952D01D01FD0D93D08D068EC30F0F60EDF
:10F94000F66E590EF76E74EC30F0D95308E168EC9E
:10F9500030F0080EF66E5A0EF76E74EC30F0D95196
:10F960007F0808E168EC30F01A0EF66E5A0EF76E5A
:10F9700074EC30F0C3AF03D0C1AF0AD002D0C1BF26
:10F9800032D0C351C15D2FE303E1C051C25D2BE210
:10F99000952D02D073EC5EF0952D01D01FD0D93D8E
:10F9A00008D089EC30F02C0EF66E5A0EF76E74EC1F
:10F9B00030F0D95308E189EC30F03E0EF66E5A0E65
:10F9C000F76E74EC30F0D9517F0808E189EC30F023
:10F9D000500EF66E5A0EF76E74EC30F0010116A759
:10F9E00001D0169D0001010116B702D016A978D0EA
:10F9F000000169A72ED0010116971699169B169D36
:10FA0000000168EC30F0620EF66E5A0EF76E74EC80
:10FA100030F089EC30F0740EF66E5A0EF76E74EC1E
:10FA200030F0640E0101CE6F000105EC2EF0CC8C9D
:10FA3000640E0101CE6F000105EC2EF0CC9C640E2B
:10FA40000101CE6F000105EC2EF001011783D4D720
:10FA50000001E051080845E2010116971699169B2E
:10FA6000169DCCBC13D0000168EC30F0860EF66E0B
:10FA70005A0EF76E74EC30F089EC30F0980EF66E9A
:10FA80005A0EF76E74EC30F012D00101000168ECF0
:10FA900030F0AA0EF66E5A0EF76E74EC30F089EC68
:10FAA00030F0BC0EF66E5A0EF76E74EC30F0640E49
:10FAB0000101CE6F000105EC2EF0CC8C640E01012B
:10FAC000CE6F000105EC2EF0CC9C640E0101CE6FD0
:10FAD000000105EC2EF0E06BCC9C01011783BDD733
:10FAE00000015CEC62F0010116A716D0000187BD91
:10FAF00002D0010111D0010ECA27D8B0CB2BD8B447
:10FB0000CC2BD8B4CD2B879D8E6B03EF6CF066ECBD
:10FB10002EF06CEC2EF0010100019551020802E17B
:10FB2000EBEC5CF0DF510A0805E266EC2EF06CECC1
:0AFB30002EF0DF6BC9EF71F0030047
:00000001FF
